:04070000BCEFFAF060
:08070800056ED8CF06F0E0CF2A
:1007100007F00001E9CF0DF0EACF08F0E1CF09F0D2
:10072000E2CF0AF0D9CF0BF0DACF0CF0F3CF14F010
:10073000F4CF15F0FACF16F0FBCF17F000C00FF092
:1007400001C010F002C011F003C012F004C013F099
:100750009DAAAEEF03F09EBA8BEF28F0F2AAB4EF99
:1007600003F0F2B4EDEF25F0A3AABAEF03F0A4BAB8
:10077000E6EF28F09DA0C0EF03F09EB0E0EF24F07C
:10078000F0AAC6EF03F0F0B4B9EF24F0F0A8CCEF74
:1007900003F0F0B297EF24F0F0A6D2EF03F0F0B040
:1007A000A8EF24F0F2A8D8EF03F0F2B286EF24F01D
:1007B000A0A2DEEF03F0A1B2F8EF26F00FC000F028
:1007C00010C001F011C002F012C003F013C004F019
:1007D0000DC0E9FF08C0EAFF088E09C0E1FF0AC0AA
:1007E000E2FF0BC0D9FF0CC0DAFF14C0F3FF15C045
:1007F000F4FF16C0FAFF17C0FBFF055007C0E0FF6B
:1008000006C0D8FF1000F2CF0EF0F29EF76A240F58
:10081000F66E080EF722000EF86E0900F5500EBEB7
:10082000F28E1200280C0106F2CF0EF0F29EF76A4B
:10083000460FF66E080EF722000EF86E0900F5500E
:100840000EBEF28E12004C6F6164205072657365AB
:1008500074206B3D254C58200A0D0000F2CF0EF09D
:10086000F29EF76A7A0FF66E080EF722000EF86E07
:100870000900F5500EBEF28E12005265616420250B
:1008800032782025327820254C5820254C582025B8
:100890004C5820254C5820254C580A0D0000F2CF0A
:1008A0000EF0F29EF76ABC0FF66E080EF722000EED
:1008B000F86E0900F5500EBEF28E12005361766597
:1008C00020507265736574206B3D254C58200A0DCD
:1008D0000000F2CF0EF0F29EF76AF00FF66E080EEF
:1008E000F722000EF86E0900F5500EBEF28E1200CF
:1008F00053617665202532782025327820254C58A2
:1009000020254C5820254C5820254C5820254C5843
:100910000A0D0000F2CF0EF0F29EF76A320FF66E6B
:10092000090EF722000EF86E0900F5500EBEF28E89
:100930001200536F6E79204556492D4433302020E4
:10094000202020202000F2CF0EF0F29EF76A640FE4
:10095000F66E090EF722000EF86E0900F5500EBE75
:10096000F28E1200536F6E79204556492D44333074
:100970002F44333120202000F2CF0EF0F29EF76A90
:10098000960FF66E090EF722000EF86E0900F5506C
:100990000EBEF28E120056616464696F2041646479
:1009A0002D612D43616D20202000F2CF0EF0F29ECC
:1009B000F76AC80FF66E090EF722000EF86E0900EE
:1009C000F5500EBEF28E1200536F6E7920455649D7
:1009D0002D4431303020202020202000F2CF0EF096
:1009E000F29EF76AFA0FF66E090EF722000EF86E05
:1009F0000900F5500EBEF28E1200536F6E7920453D
:100A000056492D4437302020202020202000F2CFCE
:100A10000EF0F29EF76A2C0FF66E0A0EF722000E09
:100A2000F86E0900F5500EBEF28E1200536F6E790B
:100A3000204252432D33303020202020202020001F
:100A4000F2CF0EF0F29EF76A5E0FF66E0A0EF722F4
:100A5000000EF86E0900F5500EBEF28E1200536FB4
:100A60006E79204252432D483730302020202020FC
:100A70002000F2CF0EF0F29EF76A900FF66E0A0E8B
:100A8000F722000EF86E0900F5500EBEF28E12002D
:100A9000536F6E79204252432D5A37303020202038
:100AA00020202000F2CF0EF0F29EF76AC20FF66E01
:100AB0000A0EF722000EF86E0900F5500EBEF28EF7
:100AC0001200536F6E79204556492D48443120203D
:100AD000202020202000F2CF0EF0F29EF76AF40FC3
:100AE000F66E0A0EF722000EF86E0900F5500EBEE3
:100AF000F28E120056616464696F2048442D3138CB
:100B00002020202020202000F2CF0EF0F29EF76A55
:100B1000260FF66E0B0EF722000EF86E0900F55048
:100B20000EBEF28E120056616464696F20436569DF
:100B30006C696E67564945572000F2CF0EF0F29E61
:100B4000F76A580FF66E0B0EF722000EF86E0900CA
:100B5000F5500EBEF28E120043616E6E6F6E20561F
:100B6000432D43353069202020202000F2CF0EF0A5
:100B7000F29EF76A8A0FF66E0B0EF722000EF86EE1
:100B80000900F5500EBEF28E120050616E61736F57
:100B90006E69632048453130302020202000F2CF9C
:100BA0000EF0F29EF76ABC0FF66E0B0EF722000EE7
:100BB000F86E0900F5500EBEF28E12004E6F7420D2
:100BC000466F756E642020202020202020202000E9
:100BD000F2CF0EF0F29EF76AEE0FF66E0B0EF722D2
:100BE000000EF86E0900F5500EBEF28E1200546928
:100BF0006C7420446972656374696F6E3A20496E43
:100C0000766572740000F2CF0EF0F29EF76A240F40
:100C1000F66E0C0EF722000EF86E0900F5500EBEAF
:100C2000F28E120054696C742044697265637469B1
:100C30006F6E3A204E6F726D616C0000F2CF0EF055
:100C4000F29EF76A5A0FF66E0C0EF722000EF86E3F
:100C50000900F5500EBEF28E12005A6F6F6D2044DF
:100C60006972656374696F6E3A20496E7665727455
:100C70000000F2CF0EF0F29EF76A900FF66E0C0EA7
:100C8000F722000EF86E0900F5500EBEF28E12002B
:100C90005A6F6F6D20446972656374696F6E3A2094
:100CA0004E6F726D616C0000F2CF0EF0F29EF76A2B
:100CB000C60FF66E0C0EF722000EF86E0900F55006
:100CC0000EBEF28E120050616E204469726563742C
:100CD000696F6E3A20496E7665727400F2CF0EF03D
:100CE000F29EF76AFA0FF66E0C0EF722000EF86EFF
:100CF0000900F5500EBEF28E120050616E2044695C
:100D000072656374696F6E3A204E6F726D616C002C
:100D1000F2CF0EF0F29EF76A2E0FF66E0D0EF7224E
:100D2000000EF86E0900F5500EBEF28E1200486FEC
:100D300073742053657269616C20496E7075743AE2
:100D400020456E61626C65640000F2CF0EF0F29E89
:100D5000F76A680FF66E0D0EF722000EF86E0900A6
:100D6000F5500EBEF28E1200486F737420536572F8
:100D700069616C20496E7075743A204469736162D0
:100D80006C656400F2CF0EF0F29EF76AA20FF66E69
:100D90000D0EF722000EF86E0900F5500EBEF28E11
:100DA000120053657269616C204563686F3A204593
:100DB0006E61626C65640000F2CF0EF0F29EF76A1D
:100DC000D60FF66E0D0EF722000EF86E0900F550E4
:100DD0000EBEF28E120053657269616C2045636825
:100DE0006F3A2044697361626C656400F2CF0EF063
:100DF000F29EF76A0A0FF66E0E0EF722000EF86EDC
:100E00000900F5500EBEF28E1200537769746368C4
:100E1000696E67204D6F64653A2053656C20466F9C
:100E20006C6C6F772045585420410000F2CF0EF0D3
:100E3000F29EF76A4A0FF66E0E0EF722000EF86E5B
:100E40000900F5500EBEF28E120053776974636884
:100E5000696E67204D6F64653A204D616E75616CF7
:100E60000000F2CF0EF0F29EF76A800FF66E0E0EC3
:100E7000F722000EF86E0900F5500EBEF28E120039
:100E80000000F2CF0EF0F29EF76AA00FF66E0E0E83
:100E9000F722000EF86E0900F5500EBEF28E120019
:100EA000537769746368696E67204D6F64653A2093
:100EB00053656C20466F6C6C6F7720455854204208
:100EC0000000F2CF0EF0F29EF76AE00FF66E0E0E03
:100ED000F722000EF86E0900F5500EBEF28E1200D9
:100EE0004E6F7420466F756E6400F2CF0EF0F29E66
:100EF000F76A080FF66E0F0EF722000EF86E090063
:100F0000F5500EBEF28E1200446961676E6F737405
:100F10006963204D6F64653A204F6E00F2CF0EF08A
:100F2000F29EF76A3A0FF66E0F0EF722000EF86E79
:100F30000900F5500EBEF28E1200446961676E6FB3
:100F400073746963204D6F64653A204F66660000D4
:100F5000F2CF0EF0F29EF76A6E0FF66E0F0EF722CA
:100F6000000EF86E0900F5500EBEF28E12005365A9
:100F70007269616C20496E666F3A204F6E00F2CF45
:100F80000EF0F29EF76A9C0FF66E0F0EF722000E1F
:100F9000F86E0900F5500EBEF28E120053657269AC
:100FA000616C20496E666F3A204F66660000F2CF92
:100FB0000EF0F29EF76ACC0FF66E0F0EF722000EBF
:100FC000F86E0900F5500EBEF28E12004C4344201C
:100FD000446973706C61793A204F6E00F2CF0EF065
:100FE000F29EF76AFA0FF66E0F0EF722000EF86EF9
:100FF0000900F5500EBEF28E12004C4344204469A5
:1010000073706C61793A204F66660000F2CF0EF083
:10101000F29EF76A2A0FF66E100EF722000EF86E97
:101020000900F5500EBEF28E120054616C6C7920EE
:1010300049646C65204C6576656C3A204869676840
:101040000000F2CF0EF0F29EF76A600FF66E100EFF
:10105000F722000EF86E0900F5500EBEF28E120057
:1010600054616C6C792049646C65204C6576656CC4
:101070003A204C6F7700F2CF0EF0F29EF76A940F91
:10108000F66E100EF722000EF86E0900F5500EBE37
:10109000F28E1200446973706C6179205669646540
:1010A0006F2053656C65637465643A204368616EB4
:1010B0006E656C204100F2CF0EF0F29EF76AD40FFD
:1010C000F66E100EF722000EF86E0900F5500EBEF7
:1010D000F28E1200446973706C6179205669646500
:1010E0006F2053656C65637465643A204368616E74
:1010F0006E656C204200F2CF0EF0F29EF76A140F7C
:10110000F66E110EF722000EF86E0900F5500EBEB5
:10111000F28E1200446F46696E64416374697665AD
:101120005072657365747320506F7274202564204B
:101130006261640A0D00F2CF0EF0F29EF76A540F5E
:10114000F66E110EF722000EF86E0900F5500EBE75
:10115000F28E1200506F7274202564204550524F59
:101160004D204C6F636174696F6E20254C580A0DD9
:101170000000F2CF0EF0F29EF76A900FF66E110E9D
:10118000F722000EF86E0900F5500EBEF28E120026
:1011900020202053797374656D204D656E75202075
:1011A0002000F2CF0EF0F29EF76AC00FF66E110E1D
:1011B000F722000EF86E0900F5500EBEF28E1200F6
:1011C000202053657269616C20496E70757420200F
:1011D0002000F2CF0EF0F29EF76AF00FF66E110EBD
:1011E000F722000EF86E0900F5500EBEF28E1200C6
:1011F000202053657269616C204563686F20202050
:101200002000F2CF0EF0F29EF76A200FF66E120E5B
:10121000F722000EF86E0900F5500EBEF28E120095
:101220002020436C656172204D656D6F72792020BE
:101230002000F2CF0EF0F29EF76A500FF66E120EFB
:10124000F722000EF86E0900F5500EBEF28E120065
:101250002020436C65617220507265736574732041
:101260002000F2CF0EF0F29EF76A800FF66E120E9B
:10127000F722000EF86E0900F5500EBEF28E120035
:1012800020202053657269616C20496E666F2020B2
:101290002000F2CF0EF0F29EF76AB00FF66E120E3B
:1012A000F722000EF86E0900F5500EBEF28E120005
:1012B0002020506F776572205570205072657365DD
:1012C0007400F2CF0EF0F29EF76AE00FF66E120E87
:1012D000F722000EF86E0900F5500EBEF28E1200D5
:1012E0002020507265736574204C6F636174696F60
:1012F0006E00F2CF0EF0F29EF76A100FF66E130E2C
:10130000F722000EF86E0900F5500EBEF28E1200A4
:10131000202052657475726E20746F204D61696E65
:101320002000F2CF0EF0F29EF76A400FF66E130E19
:10133000F722000EF86E0900F5500EBEF28E120074
:1013400020202050616E20446972204D656E75200A
:101350002000F2CF0EF0F29EF76A700FF66E130EB9
:10136000F722000EF86E0900F5500EBEF28E120044
:101370002020202020416C6C20506F72747320203C
:101380002000F2CF0EF0F29EF76AA00FF66E130E59
:10139000F722000EF86E0900F5500EBEF28E120014
:1013A000202020202020506F7274203031202020F7
:1013B0002000F2CF0EF0F29EF76AD00FF66E130EF9
:1013C000F722000EF86E0900F5500EBEF28E1200E4
:1013D000202020202020506F7274203032202020C6
:1013E0002000F2CF0EF0F29EF76A000FF66E140E98
:1013F000F722000EF86E0900F5500EBEF28E1200B4
:10140000202020202020506F727420303320202094
:101410002000F2CF0EF0F29EF76A300FF66E140E37
:10142000F722000EF86E0900F5500EBEF28E120083
:10143000202020202020506F727420303420202063
:101440002000F2CF0EF0F29EF76A600FF66E140ED7
:10145000F722000EF86E0900F5500EBEF28E120053
:10146000202020202020506F727420303520202032
:101470002000F2CF0EF0F29EF76A900FF66E140E77
:10148000F722000EF86E0900F5500EBEF28E120023
:10149000202020202020506F727420303620202001
:1014A0002000F2CF0EF0F29EF76AC00FF66E140E17
:1014B000F722000EF86E0900F5500EBEF28E1200F3
:1014C000202054696C7420446972204D656E75202B
:1014D0002000F2CF0EF0F29EF76AF00FF66E140EB7
:1014E000F722000EF86E0900F5500EBEF28E1200C3
:1014F00020202052657363616E2043616D657261C7
:101500007300F2CF0EF0F29EF76A200FF66E150E02
:10151000F722000EF86E0900F5500EBEF28E120092
:101520002020205363616E2050616E61736F6E697D
:101530006300F2CF0EF0F29EF76A500FF66E150EB2
:10154000F722000EF86E0900F5500EBEF28E120062
:1015500020202044656661756C742043616D65725E
:101560006100F2CF0EF0F29EF76A800FF66E150E54
:10157000F722000EF86E0900F5500EBEF28E120032
:1015800020202044656661756C7420507265736517
:101590007400F2CF0EF0F29EF76AB00FF66E150EE1
:1015A000F722000EF86E0900F5500EBEF28E120002
:1015B00020202050616E53656E736974697669747A
:1015C0007900F2CF0EF0F29EF76AE00FF66E150E7C
:1015D000F722000EF86E0900F5500EBEF28E1200D2
:1015E000202054696C7453656E73697469766974EC
:1015F0007900F2CF0EF0F29EF76A100FF66E160E1B
:10160000F722000EF86E0900F5500EBEF28E1200A1
:10161000202020202050616E2053706565642020BA
:101620002000F2CF0EF0F29EF76A400FF66E160E13
:10163000F722000EF86E0900F5500EBEF28E120071
:10164000202020202020537461727400F2CF0EF00D
:10165000F29EF76A6A0FF66E160EF722000EF86E0B
:101660000900F5500EBEF28E12002020202020200E
:10167000204F66660000F2CF0EF0F29EF76A940FDC
:10168000F66E160EF722000EF86E0900F5500EBE2B
:10169000F28E1200202020202020204F6E200000FB
:1016A000F2CF0EF0F29EF76ABE0FF66E160EF7221C
:1016B000000EF86E0900F5500EBEF28E12002020CA
:1016C000202020204E6F726D616C0000F2CF0EF072
:1016D000F29EF76AEA0FF66E160EF722000EF86E0B
:1016E0000900F5500EBEF28E12002020202020208E
:1016F000496E766572740000F2CF0EF0F29EF76AC2
:10170000160FF66E170EF722000EF86E0900F55050
:101710000EBEF28E12002020202020204E6F6E651B
:10172000202020200000F2CF0EF0F29EF76A440F36
:10173000F66E170EF722000EF86E0900F5500EBE79
:10174000F28E12002020202020457874726F6E20C7
:1017500020200000F2CF0EF0F29EF76A720FF66EB4
:10176000170EF722000EF86E0900F5500EBEF28E2D
:101770001200202020416E616C6F67205761792034
:101780000000F2CF0EF0F29EF76AA00FF66E170E71
:10179000F722000EF86E0900F5500EBEF28E120010
:1017A0002020456469726F6C2D34482C3253000040
:1017B000F2CF0EF0F29EF76ACE0FF66E170EF722FA
:1017C000000EF86E0900F5500EBEF28E12002020B9
:1017D000456469726F6C2D34532C32480000F2CF8F
:1017E0000EF0F29EF76AFC0FF66E170EF722000E4F
:1017F000F86E0900F5500EBEF28E120020204564EE
:1018000069726F6C2D33532C33480000F2CF0EF009
:10181000F29EF76A2A0FF66E180EF722000EF86E87
:101820000900F5500EBEF28E1200202020496E6E87
:101830006F766174696F6E200000F2CF0EF0F29E39
:10184000F76A580FF66E180EF722000EF86E0900B0
:10185000F5500EBEF28E12002020202020204F7462
:101860006865722020200000F2CF0EF0F29EF76A29
:10187000860FF66E180EF722000EF86E0900F5506E
:101880000EBEF28E1200202020202020204D616EFE
:1018900075616C00F2CF0EF0F29EF76AB20FF66E31
:1018A000180EF722000EF86E0900F5500EBEF28EEB
:1018B000120020202020466F6C6C6F772045585412
:1018C00020410000F2CF0EF0F29EF76AE20FF66EB2
:1018D000180EF722000EF86E0900F5500EBEF28EBB
:1018E000120020202020466F6C6C6F7720455854E2
:1018F00020420000F2CF0EF0F29EF76A120FF66E51
:10190000190EF722000EF86E0900F5500EBEF28E89
:101910001200202020416374697665204869676859
:101920000000F2CF0EF0F29EF76A400FF66E190E2D
:10193000F722000EF86E0900F5500EBEF28E12006E
:10194000202020416374697665204C6F7720000069
:10195000F2CF0EF0F29EF76A6E0FF66E190EF722B6
:10196000000EF86E0900F5500EBEF28E1200202017
:1019700020202020205965730000F2CF0EF0F29E47
:10198000F76A980FF66E190EF722000EF86E09002E
:10199000F5500EBEF28E12002020202020202020A4
:1019A0004E6F0000F2CF0EF0F29EF76AC20FF66E95
:1019B000190EF722000EF86E0900F5500EBEF28ED9
:1019C00012002020202020486F6D652043616D6546
:1019D00072612000F2CF0EF0F29EF76AF20FF66EFF
:1019E000190EF722000EF86E0900F5500EBEF28EA9
:1019F000120020202020205072657365742031323F
:101A000020202000F2CF0EF0F29EF76A220FF66E31
:101A10001A0EF722000EF86E0900F5500EBEF28E77
:101A200012002020202020416C6C204C6F63616CE0
:101A300020202000F2CF0EF0F29EF76A520FF66ED1
:101A40001A0EF722000EF86E0900F5500EBEF28E47
:101A5000120020203620496E43616D2036204C6FE5
:101A600063616C00F2CF0EF0F29EF76A820FF66EA1
:101A70001A0EF722000EF86E0900F5500EBEF28E17
:101A80001200536561726368696E6720666F722029
:101A900041747461636865642043616D657261734C
:101AA0000D0A0000F2CF0EF0F29EF76AC20FF66E3A
:101AB0001A0EF722000EF86E0900F5500EBEF28ED7
:101AC0001200506F72742025643A20200000F2CF7B
:101AD0000EF0F29EF76AEC0FF66E1A0EF722000E69
:101AE000F86E0900F5500EBEF28E1200204E6F20E7
:101AF00043616D20202020506F7274203000F2CF9F
:101B00000EF0F29EF76A1C0FF66E1B0EF722000E07
:101B1000F86E0900F5500EBEF28E120020484531D5
:101B200030302020202020506F7274203000F2CFFF
:101B30000EF0F29EF76A4C0FF66E1B0EF722000EA7
:101B4000F86E0900F5500EBEF28E120050616E6103
:101B5000736F6E69632044657465637465640D0A10
:101B60000000F2CF0EF0F29EF76A800FF66E1B0EA9
:101B7000F722000EF86E0900F5500EBEF28E12002C
:101B80002056432D43353069202020506F72742039
:101B90003000F2CF0EF0F29EF76AB00FF66E1B0E19
:101BA000F722000EF86E0900F5500EBEF28E1200FC
:101BB00043616E6F6E2044657465637465640D0ADD
:101BC0000000F2CF0EF0F29EF76AE00FF66E1B0EE9
:101BD000F722000EF86E0900F5500EBEF28E1200CC
:101BE0000D0A2057616974466565644261636B2024
:101BF00054696D656F7574203230303020286D73F4
:101C0000290D0A00F2CF0EF0F29EF76A220FF66E4F
:101C10001C0EF722000EF86E0900F5500EBEF28E73
:101C200012000D0A2057616974466565644261635C
:101C30006B200000F2CF0EF0F29EF76A520FF66EA4
:101C40001C0EF722000EF86E0900F5500EBEF28E43
:101C500012000A0D2043616D657261547970652030
:101C60000000F2CF0EF0F29EF76A800FF66E1C0EA7
:101C7000F722000EF86E0900F5500EBEF28E12002B
:101C800054696D656F75740A0D200000F2CF0EF077
:101C9000F29EF76AAA0FF66E1C0EF722000EF86E7F
:101CA0000900F5500EBEF28E12000D0A536F6E79C8
:101CB000204556492D4433302F3331200D0A000082
:101CC000F2CF0EF0F29EF76ADE0FF66E1C0EF722D0
:101CD000000EF86E0900F5500EBEF28E120020457F
:101CE00056492D4433302F3331506F7274203000F9
:101CF000F2CF0EF0F29EF76A0E0FF66E1D0EF7226F
:101D0000000EF86E0900F5500EBEF28E12000D0A9C
:101D1000536F6E79204556492D4433300D0A00002B
:101D2000F2CF0EF0F29EF76A3E0FF66E1D0EF7220E
:101D3000000EF86E0900F5500EBEF28E120020451E
:101D400056492D443330202020506F7274203000CB
:101D5000F2CF0EF0F29EF76A6E0FF66E1D0EF722AE
:101D6000000EF86E0900F5500EBEF28E12000D0A3C
:101D700056616464696F204164642D412D43616D37
:101D80000D0A0000F2CF0EF0F29EF76AA20FF66E77
:101D90001D0EF722000EF86E0900F5500EBEF28EF1
:101DA0001200204164642D412D43616D20506F72FB
:101DB00074203000F2CF0EF0F29EF76AD20FF66E6A
:101DC0001D0EF722000EF86E0900F5500EBEF28EC1
:101DD00012000D0A536F6E79204556492D4431305B
:101DE000300D0A00F2CF0EF0F29EF76A020FF66E87
:101DF0001E0EF722000EF86E0900F5500EBEF28E90
:101E00001200204556492D443130302020506F7249
:101E100074203000F2CF0EF0F29EF76A320FF66EA9
:101E20001E0EF722000EF86E0900F5500EBEF28E5F
:101E300012000D0A536F6E79204556492D443730F4
:101E40000D0A0000F2CF0EF0F29EF76A620FF66EF6
:101E50001E0EF722000EF86E0900F5500EBEF28E2F
:101E60001200204556492D443730202020506F72F3
:101E700074203000F2CF0EF0F29EF76A920FF66EE9
:101E80001E0EF722000EF86E0900F5500EBEF28EFF
:101E900012000D0A536F6E7920425243482D37309D
:101EA000300D0A00F2CF0EF0F29EF76AC20FF66E06
:101EB0001E0EF722000EF86E0900F5500EBEF28ECF
:101EC000120020425243482D3730302020506F728C
:101ED00074203000F2CF0EF0F29EF76AF20FF66E29
:101EE0001E0EF722000EF86E0900F5500EBEF28E9F
:101EF00012000D0A456C6D6F2043616D6572610DB6
:101F00000A00F2CF0EF0F29EF76A200FF66E1F0E57
:101F1000F722000EF86E0900F5500EBEF28E120088
:101F200020456C6D6F202020202020506F7274207F
:101F30003000F2CF0EF0F29EF76A500FF66E1F0ED1
:101F4000F722000EF86E0900F5500EBEF28E120058
:101F50000D0A536F6E79204252432D3330300D0AF3
:101F60000000F2CF0EF0F29EF76A800FF66E1F0EA1
:101F7000F722000EF86E0900F5500EBEF28E120028
:101F8000204252432D333030202020506F72742075
:101F90003000F2CF0EF0F29EF76AB00FF66E1F0E11
:101FA000F722000EF86E0900F5500EBEF28E1200F8
:101FB0000D0A536F6E79204252432D5A3730300D3F
:101FC0000A00F2CF0EF0F29EF76AE00FF66E1F0ED7
:101FD000F722000EF86E0900F5500EBEF28E1200C8
:101FE000204252432D5A3730302020506F727420D7
:101FF0003000F2CF0EF0F29EF76A100FF66E200E50
:10200000F722000EF86E0900F5500EBEF28E120097
:102010000D0A56616464696F2048442D31380D0AF9
:102020000000F2CF0EF0F29EF76A400FF66E200E1F
:10203000F722000EF86E0900F5500EBEF28E120067
:10204000202048442D3138202020506F72742030D9
:102050000000F2CF0EF0F29EF76A700FF66E200EBF
:10206000F722000EF86E0900F5500EBEF28E120037
:102070000D0A536F6E79204556492D4844310D0A9B
:102080000000F2CF0EF0F29EF76AA00FF66E200E5F
:10209000F722000EF86E0900F5500EBEF28E120007
:1020A000204556492D484431202020506F7274201D
:1020B0003000F2CF0EF0F29EF76AD00FF66E200ECF
:1020C000F722000EF86E0900F5500EBEF28E1200D7
:1020D0000D0A56616464696F204365696C696E67B7
:1020E000564945570D0A0000F2CF0EF0F29EF76AEE
:1020F000060FF66E210EF722000EF86E0900F5505D
:102100000EBEF28E12002043562F43564D50202013
:1021100020506F7274203000F2CF0EF0F29EF76AFA
:10212000360FF66E210EF722000EF86E0900F550FC
:102130000EBEF28E1200496E76616C6964204361B6
:102140006D6572610D0A0000F2CF0EF0F29EF76A23
:10215000660FF66E210EF722000EF86E0900F5509C
:102160000EBEF28E120020496E76616C69642043C7
:10217000616D65726100F2CF0EF0F29EF76A940F06
:10218000F66E210EF722000EF86E0900F5500EBE15
:10219000F28E12000D0A536F6E79204556492D4478
:1021A00033302872290D0A00F2CF0EF0F29EF76A42
:1021B000C60FF66E210EF722000EF86E0900F550DC
:1021C0000EBEF28E1200204556492D44333028723F
:1021D00029506F7274203000F2CF0EF0F29EF76A31
:1021E000F60FF66E210EF722000EF86E0900F5507C
:1021F0000EBEF28E12000A0D2041542F4D445F4D49
:102200006F6465496E712000F2CF0EF0F29EF76A9E
:10221000260FF66E220EF722000EF86E0900F5501A
:102220000EBEF28E12002054696D656F75740A0D32
:102230002000F2CF0EF0F29EF76A500FF66E220EDB
:10224000F722000EF86E0900F5500EBEF28E120055
:102250000D0A2057616974536F6E7941636B205486
:10226000696D656F757420256C6420286D73290D68
:102270000A00F2CF0EF0F29EF76A900FF66E220E71
:10228000F722000EF86E0900F5500EBEF28E120015
:102290000D0A2057616974536F6E7941636B28256D
:1022A0006C6429200000F2CF0EF0F29EF76AC40F92
:1022B000F66E220EF722000EF86E0900F5500EBEE3
:1022C000F28E12000D0A2057616974536F6E7920E7
:1022D00054696D656F757420256C6420286D7329B1
:1022E0000D0A0000F2CF0EF0F29EF76A020FF66EB2
:1022F000230EF722000EF86E0900F5500EBEF28E86
:1023000012000D0A2057616974536F6E7920000026
:10231000F2CF0EF0F29EF76A2E0FF66E230EF72222
:10232000000EF86E0900F5500EBEF28E1200205419
:10233000696D656F757420256C6420286D73290D97
:102340000A00F2CF0EF0F29EF76A600FF66E230ECF
:10235000F722000EF86E0900F5500EBEF28E120044
:102360000A0D2042616420436F6D6D616E640A0D39
:102370000000F2CF0EF0F29EF76A900FF66E230E79
:10238000F722000EF86E0900F5500EBEF28E120014
:102390000D0A205761697443616E6F6E2054696D38
:1023A000656F757420256C6420286D73290D0A00F3
:1023B000F2CF0EF0F29EF76ACE0FF66E230EF722E2
:1023C000000EF86E0900F5500EBEF28E12000D0AD6
:1023D000205761697443616E6F6E2000F2CF0EF07A
:1023E000F29EF76AFA0FF66E230EF722000EF86ED1
:1023F0000900F5500EBEF28E12000D0A20576169D9
:102400007443616E6F6E41636B2054696D656F75C7
:102410007420256C6420286D73290D0A0000F2CF0A
:102420000EF0F29EF76A3C0FF66E240EF722000EB5
:10243000F86E0900F5500EBEF28E12000D0A2057FC
:1024400061697443616E6F6E41636B200000F2CF6F
:102450000EF0F29EF76A6C0FF66E240EF722000E55
:10246000F86E0900F5500EBEF28E120057616974C5
:1024700043616E6F6E41636B202532782C25327874
:102480002028253278290D0A0000F2CF0EF0F29EA6
:10249000F76AA80FF66E240EF722000EF86E0900F8
:1024A000F5500EBEF28E1200446F55706461746573
:1024B00043616D65726153746174653A2053746150
:1024C0007465466C61673D202532582C204C617341
:1024D000743D2532582C204163746976653D253260
:1024E000580A0D3E0000F2CF0EF0F29EF76A040F7C
:1024F000F66E250EF722000EF86E0900F5500EBE9E
:10250000F28E1200446F55706461746543616D65AD
:10251000726153746174653A2044696666657265D8
:102520006E63653D2532780A0D00F2CF0EF0F29E03
:10253000F76A480FF66E250EF722000EF86E0900B6
:10254000F5500EBEF28E1200446F557064617465D2
:1025500043616D65726153746174653A20546F20F4
:102560004D616E75616C0A0D3E00F2CF0EF0F29E69
:10257000F76A880FF66E250EF722000EF86E090036
:10258000F5500EBEF28E1200446F55706461746592
:1025900043616D65726153746174653A205265736D
:1025A0006574204272696768746E657320746F2069
:1025B00064656661756C740A0D3E0000F2CF0EF022
:1025C000F29EF76ADA0FF66E250EF722000EF86E0D
:1025D0000900F5500EBEF28E1200446F5570646112
:1025E000746543616D65726153746174653A20541A
:1025F0006F204175746F0A0D3E00F2CF0EF0F29E0F
:10260000F76A180FF66E260EF722000EF86E090014
:10261000F5500EBEF28E12000D0A205761697450FB
:10262000616E61736F6E69632054696D656F757457
:1026300020256C6420286D73290D0A00F2CF0EF05E
:10264000F29EF76A5A0FF66E260EF722000EF86E0B
:102650000900F5500EBEF28E12000D0A2057616976
:102660007450616E61736F6E69632000F2CF0EF07B
:10267000F29EF76A8A0FF66E260EF722000EF86EAB
:102680000900F5500EBEF28E12000D0A2057616946
:102690007450616E61736F6E69635265737020541C
:1026A000696D656F757420256C6420286D73290D24
:1026B0000A00F2CF0EF0F29EF76AD00FF66E260EE9
:1026C000F722000EF86E0900F5500EBEF28E1200D1
:1026D0000D0A205761697450616E61736F6E696392
:1026E000526573702000F2CF0EF0F29EF76A040F6D
:1026F000F66E270EF722000EF86E0900F5500EBE9A
:10270000F28E12000A0D50726F64756374204E6170
:102710006D653A20257325730A0D0000F2CF0EF087
:10272000F29EF76A3A0FF66E270EF722000EF86E49
:102730000900F5500EBEF28E120020202020436FBB
:102740006D70696C65643A2025732061742025736F
:102750000A0D0000F2CF0EF0F29EF76A720FF66ECD
:10276000270EF722000EF86E0900F5500EBEF28E0D
:10277000120031352D4A616E2D313000F2CF0EF04E
:10278000F29EF76A9A0FF66E270EF722000EF86E89
:102790000900F5500EBEF28E120031363A30323A50
:1027A00031300000F2CF0EF0F29EF76AC20FF66EE3
:1027B000270EF722000EF86E0900F5500EBEF28EBD
:1027C00012000D0A53797374656D20536574746932
:1027D0006E67733A0A0D0A0D44656661756C742064
:1027E00043616D6572613A2025640A0D4465666136
:1027F000756C74205072657365743A2025640A0DF7
:102800000000F2CF0EF0F29EF76A200FF66E280E4F
:10281000F722000EF86E0900F5500EBEF28E12007F
:102820000D0A54696C745370656564202050616EA4
:10283000537065656420205A6F6F6D5370656564D1
:10284000202050616E656C204C69676874730A0DB6
:102850000000F2CF0EF0F29EF76A700FF66E280EAF
:10286000F722000EF86E0900F5500EBEF28E12002F
:1028700020202025642020202020202020202564C6
:1028800020202020202020202564202020202020FF
:102890002020202025640A0D0A0D0000F2CF0EF042
:1028A000F29EF76ABA0FF66E280EF722000EF86E47
:1028B0000900F5500EBEF28E12000D0A4A6F7973B0
:1028C0007469636B2053656E736974697669747992
:1028D000202050616E202054696C742049646C651E
:1028E000205A6F6E650A0D00F2CF0EF0F29EF76A65
:1028F000060FF66E290EF722000EF86E0900F5504D
:102900000EBEF28E12002020202020202020202029
:10291000202020202020202020202020202564206E
:1029200020202564202020202020202025640A0D3E
:102930000A0D0000F2CF0EF0F29EF76A520FF66E0B
:10294000290EF722000EF86E0900F5500EBEF28E29
:1029500012000A0D507265736574733A0A0D0A0D00
:102960000000F2CF0EF0F29EF76A800FF66E290E8D
:10297000F722000EF86E0900F5500EBEF28E12001E
:1029800043616D20507265204D6F64656C2020207E
:1029900020202020202020202020202020205061C6
:1029A0006E20202054696C7420205A6F6F6D204671
:1029B0006F63757320204272696768746E65737304
:1029C0000000F2CF0EF0F29EF76AE00FF66E290ECD
:1029D000F722000EF86E0900F5500EBEF28E1200BE
:1029E000205B4272696768742C466F6375732C4173
:1029F00057422C424C435D0A0D0A0D00F2CF0EF0F7
:102A0000F29EF76A1A0FF66E2A0EF722000EF86E83
:102A10000900F5500EBEF28E120020256420202001
:102A2000253264202531387320253258254C582012
:102A300020254C582020254C582020254C5820205B
:102A4000202020254C580000F2CF0EF0F29EF76AAD
:102A5000660FF66E2A0EF722000EF86E0900F5508A
:102A60000EBEF28E12002020202020202000F2CF67
:102A70000EF0F29EF76A8C0FF66E2A0EF722000E09
:102A8000F86E0900F5500EBEF28E12004F6E202037
:102A9000202020200000F2CF0EF0F29EF76AB40F43
:102AA000F66E2A0EF722000EF86E0900F5500EBEE3
:102AB000F28E12004F666620202020200000F2CF08
:102AC0000EF0F29EF76ADC0FF66E2A0EF722000E69
:102AD000F86E0900F5500EBEF28E12004F6E2020E7
:102AE00020200000F2CF0EF0F29EF76A020FF66E81
:102AF0002B0EF722000EF86E0900F5500EBEF28E76
:102B000012004F66662020200000F2CF0EF0F29EE9
:102B1000F76A280FF66E2B0EF722000EF86E0900EA
:102B2000F5500EBEF28E12004F6E20202000F2CF24
:102B30000EF0F29EF76A4C0FF66E2B0EF722000E87
:102B4000F86E0900F5500EBEF28E12004F66662038
:102B50002000F2CF0EF0F29EF76A700FF66E2B0E89
:102B6000F722000EF86E0900F5500EBEF28E12002C
:102B70004F6E0000F2CF0EF0F29EF76A920FF66EE3
:102B80002B0EF722000EF86E0900F5500EBEF28EE5
:102B900012004F666600F2CF0EF0F29EF76AB40F95
:102BA000F66E2B0EF722000EF86E0900F5500EBEE1
:102BB000F28E12000A0D436F6D6D616E6420436FDB
:102BC0006D706C6574650A0D3E00F2CF0EF0F29EDA
:102BD000F76AE80FF66E2B0EF722000EF86E09006A
:102BE000F5500EBEF28E12000A0D43616D204D6F3E
:102BF00064656C0A0D00F2CF0EF0F29EF76A140FB6
:102C0000F66E2C0EF722000EF86E0900F5500EBE7F
:102C1000F28E120020256420204E6F2043616D65E6
:102C200072610A0D0000F2CF0EF0F29EF76A440FB7
:102C3000F66E2C0EF722000EF86E0900F5500EBE4F
:102C4000F28E12003E2573204E6F7420466F756E13
:102C5000640A0D3E0000F2CF0EF0F29EF76A740F88
:102C6000F66E2C0EF722000EF86E0900F5500EBE1F
:102C7000F28E12000A0D0A0D52656164204932433A
:102C80002055256420416464726573733D25325874
:102C90002052656769737465723D2532582052650C
:102CA00073706F6E73653D2532580A0D0000F2CFC8
:102CB0000EF0F29EF76ACC0FF66E2C0EF722000E85
:102CC000F86E0900F5500EBEF28E12000A0D0A0DC4
:102CD0005265616420493243205525642041646473
:102CE000726573733D253258205265676973746548
:102CF000723D25325820526573706F6E73653D25A5
:102D00004C580A0D0000F2CF0EF0F29EF76A240F25
:102D1000F66E2D0EF722000EF86E0900F5500EBE6D
:102D2000F28E12000A0D0A0D52656164205365632C
:102D30006F6E6461727920493243205525642041C9
:102D40006464726573733D253258205265676973F8
:102D50007465723D25325820526573706F6E7365CD
:102D60003D2532580A0D0000F2CF0EF0F29EF76AB0
:102D7000860FF66E2D0EF722000EF86E0900F55044
:102D80000EBEF28E12000A0D0A0D526561642053C8
:102D900065636F6E64617279204932432055256402
:102DA00020416464726573733D2532582052656713
:102DB00069737465723D25325820526573706F6E69
:102DC00073653D254C580A0D0000F2CF0EF0F29EBF
:102DD000F76AE80FF66E2D0EF722000EF86E090066
:102DE000F5500EBEF28E12000A0D0A0D577269746C
:102DF000652055256420416464726573733D2532F6
:102E0000582C52656769737465723D2532582C449D
:102E10006174613D253258200A0D0000F2CF0EF09A
:102E2000F29EF76A3A0FF66E2E0EF722000EF86E3B
:102E30000900F5500EBEF28E12000A0D0A0D5772EF
:102E40006974652055256420416464726573733D1F
:102E50002532582C52656769737465723D25325866
:102E60002C446174613D254C58200A0D0000F2CFBE
:102E70000EF0F29EF76A8C0FF66E2E0EF722000E01
:102E8000F86E0900F5500EBEF28E12000A0D0A0D02
:102E90005772697465205365636F6E64617279203F
:102EA00055256420416464726573733D2532582C46
:102EB00052656769737465723D2532582C4461749C
:102EC000613D253258200A0D0000F2CF0EF0F29E2F
:102ED000F76AE80FF66E2E0EF722000EF86E090064
:102EE000F5500EBEF28E12000A0D0A0D577269746B
:102EF00065205365636F6E64617279205525642087
:102F0000416464726573733D2532582C526567695C
:102F1000737465723D2532582C446174613D254CB3
:102F200058200A0D0000F2CF0EF0F29EF76A440F0F
:102F3000F66E2F0EF722000EF86E0900F5500EBE49
:102F4000F28E12000A0D3E2043616D6572612025EC
:102F500064204E6F7420617661696C61626C650AF1
:102F60000D3E2000F2CF0EF0F29EF76A820FF66E51
:102F70002F0EF722000EF86E0900F5500EBEF28EED
:102F800012000A0D3E204A6F79737469636B204EFC
:102F900065757472616C205A6F6E65202564200A15
:102FA0000D3E2000F2CF0EF0F29EF76AC20FF66ED1
:102FB0002F0EF722000EF86E0900F5500EBEF28EAD
:102FC00012004F6E2043616D65726120496E697415
:102FD0002C2073656E6420486F6D6520636F6D6D86
:102FE000616E640A0D3E2000F2CF0EF0F29EF76A89
:102FF000060FF66E300EF722000EF86E0900F5503F
:103000000EBEF28E12004F6E2043616D657261201C
:10301000496E69742C2073656E6420507265736507
:103020007420313220636F6D6D616E642073657141
:1030300075656E63650A0D3E2000F2CF0EF0F29EBC
:10304000F76A580FF66E300EF722000EF86E090080
:10305000F5500EBEF28E12000A0D3E204A6F7973B3
:103060007469636B2050616E2053656E7369746977
:1030700076697479202564200A0D3E200000F2CF85
:103080000EF0F29EF76A9C0FF66E300EF722000EDD
:10309000F86E0900F5500EBEF28E12000A0D3E5376
:1030A000657444656661756C74202564200A0D3E64
:1030B0002000F2CF0EF0F29EF76AD00FF66E300EBF
:1030C000F722000EF86E0900F5500EBEF28E1200C7
:1030D0000A0D3E44656661756C7443616D2025641C
:1030E000200A0D3E2000F2CF0EF0F29EF76A040F88
:1030F000F66E310EF722000EF86E0900F5500EBE86
:10310000F28E120045787465726E616C205472699B
:1031100067676572732061726520416374697665C3
:1031200020486967680A0D00F2CF0EF0F29EF76A38
:10313000460FF66E310EF722000EF86E0900F550BC
:103140000EBEF28E120045787465726E616C20546A
:103150007269676765727320617265204163746983
:103160007665204C6F770A0D0000F2CF0EF0F29ECC
:10317000F76A880FF66E310EF722000EF86E09001E
:10318000F5500EBEF28E120050726F63657373209D
:1031900055313420254C5820254C580A0D00F2CFCB
:1031A0000EF0F29EF76ABC0FF66E310EF722000E9B
:1031B000F86E0900F5500EBEF28E12002563494EDE
:1031C000503A25643B00F2CF0EF0F29EF76AE40F0E
:1031D000F66E310EF722000EF86E0900F5500EBEA5
:1031E000F28E12002020204578742043544C204158
:1031F000203020202000F2CF0EF0F29EF76A140F4C
:10320000F66E320EF722000EF86E0900F5500EBE73
:10321000F28E120043544C204125640A0D3E0000FA
:10322000F2CF0EF0F29EF76A3E0FF66E320EF722E4
:10323000000EF86E0900F5500EBEF28E1200342A10
:1032400030230000F2CF0EF0F29EF76A620FF66EA6
:10325000320EF722000EF86E0900F5500EBEF28E07
:1032600012002563494E503A25643B256354414B77
:103270003A25642E25643B00F2CF0EF0F29EF76AE9
:10328000960FF66E320EF722000EF86E0900F5501A
:103290000EBEF28E12002020204578742043544C3C
:1032A0002042203020202000F2CF0EF0F29EF76A5C
:1032B000C60FF66E320EF722000EF86E0900F550BA
:1032C0000EBEF28E120043544C204225640A0D3E7D
:1032D0000000F2CF0EF0F29EF76AF00FF66E320E9B
:1032E000F722000EF86E0900F5500EBEF28E1200A5
:1032F00056616C69646174652043757272656E74A1
:1033000053746174652E43616D6572615B25645D04
:10331000202532580A0D0000F2CF0EF0F29EF76A17
:10332000360FF66E330EF722000EF86E0900F550D8
:103330000EBEF28E12004E6F2D56616C6964617480
:10334000652043757272656E7453746174652E43A3
:10335000616D6572615B25645D202532580A0D0040
:10336000F2CF0EF0F29EF76A7E0FF66E330EF72262
:10337000000EF86E0900F5500EBEF28E12004C6F72
:10338000616420507265736574732043616D2025FC
:10339000640A0D00F2CF0EF0F29EF76AB20FF66EDD
:1033A000330EF722000EF86E0900F5500EBEF28EB5
:1033B0001200202020202043616D2053656C2030B6
:1033C00020202000F2CF0EF0F29EF76AE20FF66E98
:1033D000330EF722000EF86E0900F5500EBEF28E85
:1033E000120043616D6572612025640A0D3E000084
:1033F000F2CF0EF0F29EF76A0E0FF66E340EF72241
:10340000000EF86E0900F5500EBEF28E1200204339
:10341000616D2053656C2030204E6F2043616D003C
:10342000F2CF0EF0F29EF76A3E0FF66E340EF722E0
:10343000000EF86E0900F5500EBEF28E12005072AA
:103440006F636573732055313520254C5820254C0A
:10345000580A0D00F2CF0EF0F29EF76A720FF66E68
:10346000340EF722000EF86E0900F5500EBEF28EF3
:10347000120020496E2043616D2053746F726520E5
:1034800030300000F2CF0EF0F29EF76AA20FF66E17
:10349000340EF722000EF86E0900F5500EBEF28EC3
:1034A0001200496E43616D2053746F72652025646C
:1034B0000A0D3E00F2CF0EF0F29EF76AD20FF66EC2
:1034C000340EF722000EF86E0900F5500EBEF28E93
:1034D0001200202052656164696E672043616D654A
:1034E00072610000F2CF0EF0F29EF76A020FF66EE4
:1034F000350EF722000EF86E0900F5500EBEF28E62
:103500001200202053746F72696E672050726573C9
:1035100065740000F2CF0EF0F29EF76A320FF66E7D
:10352000350EF722000EF86E0900F5500EBEF28E31
:1035300012002053746F7265203030205072657312
:1035400065740000F2CF0EF0F29EF76A620FF66E1D
:10355000350EF722000EF86E0900F5500EBEF28E01
:10356000120053746F72652025640A0D3E00F2CF7D
:103570000EF0F29EF76A8C0FF66E350EF722000EF3
:10358000F86E0900F5500EBEF28E12002053746FD3
:103590007265203030204661696C65640000F2CFAE
:1035A0000EF0F29EF76ABC0FF66E350EF722000E93
:1035B000F86E0900F5500EBEF28E120020496E2002
:1035C00043616D20507265736574203030200000B7
:1035D000F2CF0EF0F29EF76AEE0FF66E350EF7227E
:1035E000000EF86E0900F5500EBEF28E12005072F9
:1035F000657365742025640A0D3E0000F2CF0EF05D
:10360000F29EF76A1A0FF66E360EF722000EF86E6B
:103610000900F5500EBEF28E120050616E61736F9C
:103620006E696320466F6375733A20546F2041754D
:10363000746F0A0D3E00F2CF0EF0F29EF76A540F3F
:10364000F66E360EF722000EF86E0900F5500EBE2B
:10365000F28E120050616E61736F6E696320466F67
:103660006375733A20546F204D616E75616C0A0D5D
:103670003E00F2CF0EF0F29EF76A900FF66E360E15
:10368000F722000EF86E0900F5500EBEF28E120001
:1036900050616E61736F6E6963204272696768740E
:1036A0003A20546F204175746F0A0D3E0000F2CF2E
:1036B0000EF0F29EF76ACC0FF66E360EF722000E71
:1036C000F86E0900F5500EBEF28E120050616E6168
:1036D000736F6E6963204272696768743A20546F31
:1036E000204D616E75616C0A0D3E0000F2CF0EF048
:1036F000F29EF76A0A0FF66E370EF722000EF86E8A
:103700000900F5500EBEF28E120020204C6F61644D
:10371000696E67205072657365740000F2CF0EF019
:10372000F29EF76A3A0FF66E370EF722000EF86E29
:103730000900F5500EBEF28E120020202050726556
:10374000736574203030202020200000F2CF0EF06E
:10375000F29EF76A6A0FF66E370EF722000EF86EC9
:103760000900F5500EBEF28E120020202050726526
:10377000736574203030204261640000F2CF0EF097
:10378000F29EF76A9A0FF66E370EF722000EF86E69
:103790000900F5500EBEF28E12002020204E6F2040
:1037A000507265736574203030200000F2CF0EF047
:1037B000F29EF76ACA0FF66E370EF722000EF86E09
:1037C0000900F5500EBEF28E1200202045787420BC
:1037D000566964656F2041204F6E0000F2CF0EF0F5
:1037E000F29EF76AFA0FF66E370EF722000EF86EA9
:1037F0000900F5500EBEF28E1200446973706C61C0
:103800007920434841204F6E0A0D3E00F2CF0EF062
:10381000F29EF76A2A0FF66E380EF722000EF86E47
:103820000900F5500EBEF28E12002020204469736C
:10383000706C6179204F66660000F2CF0EF0F29E48
:10384000F76A580FF66E380EF722000EF86E090070
:10385000F5500EBEF28E1200446973706C617920CF
:103860004F66660A0D3E0000F2CF0EF0F29EF76A38
:10387000860FF66E380EF722000EF86E0900F5502E
:103880000EBEF28E120020204578742056696465C1
:103890006F2042204F6E0000F2CF0EF0F29EF76ACA
:1038A000B60FF66E380EF722000EF86E0900F550CE
:1038B0000EBEF28E1200446973706C617920434829
:1038C00042204F6E0A0D3E00F2CF0EF0F29EF76AD4
:1038D000E60FF66E380EF722000EF86E0900F5506E
:1038E0000EBEF28E120050726F63657373205531F5
:1038F0003620254C5820254C580A0D00F2CF0EF0EA
:10390000F29EF76A1A0FF66E390EF722000EF86E65
:103910000900F5500EBEF28E1200204261636B4C1E
:1039200069676874436D70204F666600F2CF0EF0D1
:10393000F29EF76A4A0FF66E390EF722000EF86E05
:103940000900F5500EBEF28E1200424C43204F6625
:10395000660A0D3E0000F2CF0EF0F29EF76A740F79
:10396000F66E390EF722000EF86E0900F5500EBE05
:10397000F28E1200204261636B4C69676874436D7C
:1039800070204F6E2000F2CF0EF0F29EF76AA40F67
:10399000F66E390EF722000EF86E0900F5500EBED5
:1039A000F28E1200424C43204F6E0A0D3E00F2CFC1
:1039B0000EF0F29EF76ACC0FF66E390EF722000E6B
:1039C000F86E0900F5500EBEF28E120020424C43F4
:1039D000204E6F20537570706F7274202000F2CFEC
:1039E0000EF0F29EF76AFC0FF66E390EF722000E0B
:1039F000F86E0900F5500EBEF28E1200506F77651A
:103A000072204F66660A0D3E0000F2CF0EF0F29E65
:103A1000F76A280FF66E3A0EF722000EF86E0900CC
:103A2000F5500EBEF28E1200506F776572204F6E09
:103A30000A0D3E00F2CF0EF0F29EF76A520FF66EBC
:103A40003A0EF722000EF86E0900F5500EBEF28E07
:103A5000120020204272696768746E657373205586
:103A600070202000F2CF0EF0F29EF76A820FF66E01
:103A70003A0EF722000EF86E0900F5500EBEF28ED7
:103A800012004272696768742055700A0D3E00008A
:103A9000F2CF0EF0F29EF76AAE0FF66E3A0EF722F4
:103AA000000EF86E0900F5500EBEF28E12002020B6
:103AB0004272696768746E65737320446E202000DB
:103AC000F2CF0EF0F29EF76ADE0FF66E3A0EF72294
:103AD000000EF86E0900F5500EBEF28E1200427212
:103AE0006967687420446F776E0A0D3E0000F2CF5C
:103AF0000EF0F29EF76A0C0FF66E3B0EF722000EE8
:103B0000F86E0900F5500EBEF28E120020204272AF
:103B1000696768746E657373204175746F00F2CFC6
:103B20000EF0F29EF76A3C0FF66E3B0EF722000E87
:103B3000F86E0900F5500EBEF28E120042726967EF
:103B40006874204175746F0A0D3E0000F2CF0EF0CC
:103B5000F29EF76A6A0FF66E3B0EF722000EF86EC1
:103B60000900F5500EBEF28E1200202042726967E5
:103B700068746E657373204D616E2000F2CF0EF095
:103B8000F29EF76A9A0FF66E3B0EF722000EF86E61
:103B90000900F5500EBEF28E120042726967687419
:103BA000204D616E75616C0A0D3E0000F2CF0EF083
:103BB000F29EF76ACA0FF66E3B0EF722000EF86E01
:103BC0000900F5500EBEF28E120020202020466F14
:103BD000637573204E65617220202000F2CF0EF0D5
:103BE000F29EF76AFA0FF66E3B0EF722000EF86EA1
:103BF0000900F5500EBEF28E1200466F63757320F9
:103C00004E6561720A0D3E00F2CF0EF0F29EF76A29
:103C1000260FF66E3C0EF722000EF86E0900F550E6
:103C20000EBEF28E120020202020466F6375732096
:103C30004661722020200000F2CF0EF0F29EF76A5B
:103C4000560FF66E3C0EF722000EF86E0900F55086
:103C50000EBEF28E1200466F637573204661720AC3
:103C60000D3E0000F2CF0EF0F29EF76A820FF66E64
:103C70003C0EF722000EF86E0900F5500EBEF28ED3
:103C8000120020202020466F637573204175746FE9
:103C900020200000F2CF0EF0F29EF76AB20FF66E0F
:103CA0003C0EF722000EF86E0900F5500EBEF28EA3
:103CB000120020202020466F637573204D616E75C1
:103CC000616C0000F2CF0EF0F29EF76AE20FF66E22
:103CD0003C0EF722000EF86E0900F5500EBEF28E73
:103CE0001200466F637573204175746F0A0D3E00B4
:103CF000F2CF0EF0F29EF76A0E0FF66E3D0EF7222F
:103D0000000EF86E0900F5500EBEF28E1200204132
:103D100075746F576869746542616C204F66660000
:103D2000F2CF0EF0F29EF76A3E0FF66E3D0EF722CE
:103D3000000EF86E0900F5500EBEF28E12004157CB
:103D400042204F66660A0D3E0000F2CF0EF0F29E52
:103D5000F76A680FF66E3D0EF722000EF86E090046
:103D6000F5500EBEF28E1200204175746F576869CF
:103D7000746542616C204F6E2000F2CF0EF0F29E0F
:103D8000F76A980FF66E3D0EF722000EF86E0900E6
:103D9000F5500EBEF28E1200415742204F6E0A0DB2
:103DA0003E00F2CF0EF0F29EF76AC00FF66E3D0EA7
:103DB000F722000EF86E0900F5500EBEF28E1200CA
:103DC00020415742204E6F20537570706F727420DF
:103DD0002000F2CF0EF0F29EF76AF00FF66E3D0E65
:103DE000F722000EF86E0900F5500EBEF28E12009A
:103DF0002043616D20253258202C20537461746556
:103E0000202532580A0D0000F2CF0EF0F29EF76A1C
:103E1000260FF66E3E0EF722000EF86E0900F550E2
:103E20000EBEF28E12004261642047657420553147
:103E3000342049535220254C5820254C580A0D0057
:103E4000F2CF0EF0F29EF76A5E0FF66E3E0EF7228C
:103E5000000EF86E0900F5500EBEF28E120042619F
:103E60006420476574205531352049535220254C34
:103E70005820254C580A0D00F2CF0EF0F29EF76A3A
:103E8000960FF66E3E0EF722000EF86E0900F55002
:103E90000EBEF28E120042616420476574205531D7
:103EA000362049535220254C5820254C580A0D00E5
:103EB000F2CF0EF0F29EF76ACE0FF66E3E0EF722AC
:103EC000000EF86E0900F5500EBEF28E1200205062
:103ED00072657365742050474D204D6F64652000F6
:103EE000F2CF0EF0F29EF76AFE0FF66E3E0EF7224C
:103EF000000EF86E0900F5500EBEF28E1200204C36
:103F00006F6164696E672050726573657431320049
:103F1000F2CF0EF0F29EF76A2E0FF66E3F0EF722EA
:103F2000000EF86E0900F5500EBEF28E1200204E03
:103F30006F20507265736574313220466F756E6400
:103F40000000F2CF0EF0F29EF76A600FF66E3F0EA1
:103F5000F722000EF86E0900F5500EBEF28E120028
:103F60004D61696E566964656F204572726F72208B
:103F7000506F72743D2532780A0D3E200000F2CF5A
:103F80000EF0F29EF76A9C0FF66E3F0EF722000EBF
:103F9000F86E0900F5500EBEF28E12005072657672
:103FA000696577566964656F204572726F7220503B
:103FB0006F72743D2532780A0D3E2000F2CF0EF06C
:103FC000F29EF76ADA0FF66E3F0EF722000EF86ED9
:103FD0000900F5500EBEF28E1200436F6D31205273
:103FE000656365697665204572726F722873293D35
:103FF0002532780A0D00F2CF0EF0F29EF76A140F08
:10400000F66E400EF722000EF86E0900F5500EBE57
:10401000F28E1200436F6D322052656365697665DA
:10402000204572726F722873293D2532780A0D007F
:10403000F2CF0EF0F29EF76A4E0FF66E400EF722A8
:10404000000EF86E0900F5500EBEF28E12000C50F4
:10405000726F64756374696F6E56696577534A0051
:10406000F2CF0EF0F29EF76A7E0FF66E400EF72248
:10407000000EF86E0900F5500EBEF28E12000A0016
:10408000F2CF0EF0F29EF76A9E0FF66E400EF72208
:10409000000EF86E0900F5500EBEF28E12002020C0
:1040A0005374617274696E67205570202000F2CFDE
:1040B0000EF0F29EF76ACC0FF66E400EF722000E5D
:1040C000F86E0900F5500EBEF28E12000A0D436123
:1040D0006D657261205061737320436F6D706C6504
:1040E00074650A0D3E00F2CF0EF0F29EF76A040FDF
:1040F000F66E410EF722000EF86E0900F5500EBE66
:10410000F28E12005461736B466C616773203078D5
:1041100030662028254C58290A0D0000F2CF0EF0F9
:10412000F29EF76A3A0FF66E410EF722000EF86E15
:104130000900F5500EBEF28E120050726F64756366
:1041400074696F6E56696577534A25730A0D0000CE
:10415000F2CF0EF0F29EF76A6E0FF66E410EF72266
:10416000000EF86E0900F5500EBEF28E120054617A
:10417000736B466C61677320307830663020282579
:104180004C58290A0D00F2CF0EF0F29EF76AA40FE8
:10419000F66E410EF722000EF86E0900F5500EBEC5
:1041A000F28E12002046696E64696E672043616D6D
:1041B000657261730000F2CF0EF0F29EF76AD40FC1
:1041C000F66E410EF722000EF86E0900F5500EBE95
:1041D000F28E12005461736B466C61677320307805
:1041E000306630302028254C58290A0D0000F2CFC7
:1041F0000EF0F29EF76A0C0FF66E420EF722000EDA
:10420000F86E0900F5500EBEF28E120020436C6568
:104210006172696E67205072657365747300F2CFC6
:104220000EF0F29EF76A3C0FF66E420EF722000E79
:10423000F86E0900F5500EBEF28E120020436C6538
:104240006172696E6720416C6C2020200000F2CF03
:104250000EF0F29EF76A6C0FF66E420EF722000E19
:10426000F86E0900F5500EBEF28E12005461736BA9
:10427000466C616773203078663030302028254CDA
:1042800058290A0D0000F2CF0EF0F29EF76AA40F33
:10429000F66E420EF722000EF86E0900F5500EBEC3
:1042A000F28E1200446F44556D700000F2CF0EF094
:1042B000F29EF76ACA0FF66E420EF722000EF86EF3
:1042C0000900F5500EBEF28E1200456E61626C65FB
:1042D0002053657269616C0A0D00F2CF0EF0F29EF8
:1042E000F76AF80FF66E420EF722000EF86E09001C
:1042F000F5500EBEF28E12005461736B466C61670E
:10430000733220307830662028254C58290A0D0059
:10431000F2CF0EF0F29EF76A2E0FF66E430EF722E2
:10432000000EF86E0900F5500EBEF28E12005461B8
:10433000736B466C616773322030783066302028AA
:10434000254C58290A0D0000F2CF0EF0F29EF76AB4
:10435000660FF66E430EF722000EF86E0900F55058
:104360000EBEF28E120020204E6F74206F6E205011
:104370007265736574200000F2CF0EF0F29EF76A4A
:10438000960FF66E430EF722000EF86E0900F550F8
:104390000EBEF28E12005461736B53696D756C61C1
:1043A0007465203078303030662028254C58290A32
:1043B0000D00F2CF0EF0F29EF76AD00FF66E430EAC
:1043C000F722000EF86E0900F5500EBEF28E1200B4
:1043D0005461736B53696D756C617465203078300E
:1043E00066302028254C58290A0D0000F2CF0EF027
:1043F000F29EF76A0A0FF66E440EF722000EF86E70
:104400000900F5500EBEF28E12005461736B5369B1
:104410006D756C61746520307830663030202825E9
:104420004C58290A0D00F2CF0EF0F29EF76A440FA5
:10443000F66E440EF722000EF86E0900F5500EBE1F
:10444000F28E12005461736B53696D756C61746503
:10445000203078663030302028254C58290A0D004D
:10446000F2CF0EF0F29EF76A7E0FF66E440EF72240
:10447000000EF86E0900F5500EBEF28E1200546167
:10448000736B53696D756C617465312030783030B1
:1044900030662028254C58290A0D0000F2CF0EF076
:1044A000F29EF76ABA0FF66E440EF722000EF86E0F
:1044B0000900F5500EBEF28E12005461736B536901
:1044C0006D756C617465312030783030663020282D
:1044D000254C58290A0D0000F2CF0EF0F29EF76A23
:1044E000F60FF66E440EF722000EF86E0900F55036
:1044F0000EBEF28E1200204C6F6164696E6720441C
:10450000656661756C747300F2CF0EF0F29EF76A07
:10451000260FF66E450EF722000EF86E0900F550D4
:104520000EBEF28E12002046696E64696E672045E9
:104530007874726F6E00F2CF0EF0F29EF76A540F2D
:10454000F66E450EF722000EF86E0900F5500EBE0D
:10455000F28E120020466F756E642020204578741C
:10456000726F6E00F2CF0EF0F29EF76A820FF66E57
:10457000450EF722000EF86E0900F5500EBEF28EC1
:10458000120020457874726F6E2057616974203371
:1045900030730000F2CF0EF0F29EF76AB20FF66EA3
:1045A000450EF722000EF86E0900F5500EBEF28E91
:1045B000120020457874726F6E2057616974203242
:1045C00030730000F2CF0EF0F29EF76AE20FF66E43
:1045D000450EF722000EF86E0900F5500EBEF28E61
:1045E000120020457874726F6E2057616974203113
:1045F00030730000F2CF0EF0F29EF76A120FF66EE3
:10460000460EF722000EF86E0900F5500EBEF28E2F
:10461000120020457874726F6E2052657374617257
:104620007400F2CF0EF0F29EF76A400FF66E460E5F
:10463000F722000EF86E0900F5500EBEF28E120041
:1046400020457874726F6E204E6F7420466F756EC1
:104650006400F2CF0EF0F29EF76A700FF66E460E0F
:10466000F722000EF86E0900F5500EBEF28E120011
:104670002046696E6420416E616C6F6757617920D6
:104680002000F2CF0EF0F29EF76AA00FF66E460EF3
:10469000F722000EF86E0900F5500EBEF28E1200E1
:1046A00020466F756E6420416E616C6F675761794B
:1046B0000000F2CF0EF0F29EF76AD00FF66E460EB3
:1046C000F722000EF86E0900F5500EBEF28E1200B1
:1046D00020416E616C6F67576179203330207365BC
:1046E0006300F2CF0EF0F29EF76A000FF66E470EEF
:1046F000F722000EF86E0900F5500EBEF28E120081
:1047000020416E616C6F675761792032302073658C
:104710006300F2CF0EF0F29EF76A300FF66E470E8E
:10472000F722000EF86E0900F5500EBEF28E120050
:1047300020416E616C6F675761792031302073655D
:104740006300F2CF0EF0F29EF76A600FF66E470E2E
:10475000F722000EF86E0900F5500EBEF28E120020
:1047600020416E616C6F6757617920526573747276
:104770007400F2CF0EF0F29EF76A900FF66E470EBD
:10478000F722000EF86E0900F5500EBEF28E1200F0
:1047900020416E616C6F67576179204E6F46696E7C
:1047A0006400F2CF0EF0F29EF76AC00FF66E470E6D
:1047B000F722000EF86E0900F5500EBEF28E1200C0
:1047C0002020506F776572696E6720557020202019
:1047D0000000F2CF0EF0F29EF76AF00FF66E470E71
:1047E000F722000EF86E0900F5500EBEF28E120090
:1047F0000A2020506F776572696E6720446F776E6C
:104800002000C69E9E96F3CCC9FF020EC6BE05D000
:104810009EA6FED7000EC5BC010E016E000CC69C04
:10482000C586C5B6FED700B0C59A00A0C58AC588A2
:10483000C5B8FED7C9CF01F0000C0C01EE6BC580E6
:10484000C5B0FED70A0E006E002EFED700D0EC5188
:10485000FE0BEF6FF36F0001D4DF0A0E006E002E27
:10486000FED700D0EDCCF3FCCCDF0A0E006E002E9C
:10487000FED700D0C582C5B2FED70A0E006E002E4C
:10488000FED700D00C01EC510109EF6FF36F00016E
:10489000B8DF0A0E006E002EFED700D0006ABFDF20
:1048A00001C0EEFC0A0E006E002EFED700D0C584BB
:1048B000C5B4FED70D0E006E002EFED70C01EECC57
:1048C00001F00001000C0C01E86BE96BEA6BE751A9
:1048D000FE0BEB6FE6CCECFCED6F0001AEDF01C030
:1048E000EAFC0C01E7510109EB6FE6CCECFCED6F43
:1048F0000001A3DF01C0E9FC0C01E86BEA51E813F9
:10490000E8CC01F0E9CC02F00001000C0C01E46BF2
:10491000E56B4C80400EE66F080EE76F0001D3DFB9
:1049200002C0E5FC01C0E4FCF292DEEF03F00C01F2
:10493000E46BE56B4C82440EE66F080EE76F0001F6
:10494000C2DF02C0E5FC01C0E4FCF092DEEF03F040
:104950000C01E46BE56B4C84420EE66F080EE76FCA
:104960000001B1DF02C0E5FC01C0E4FCF090DEEF25
:1049700003F00C01E46BE56B4C86460EE66F080E07
:10498000E76F0001A0DF02C0E5FC01C0E4FCF09489
:10499000DEEF03F00C01E751016AE65D03E2E6CCCD
:1049A00000F00CD0006A080EE86FE6370036E751D9
:1049B000005CD8B0006E0136E82FF7D70001000C7C
:1049C0000101A851040DF3500C01E56BE46F036A7B
:1049D0000101B8510C01E425016EE551032201509B
:1049E000AC0FE96E010E0320EA6EC282C2B2FED79E
:1049F000C4CFEFFF0101A851040DF3500C01E56B8A
:104A0000E46F036A0101B8510C01E425016EE55120
:104A100003220150AC0FE96E010E0320EA6EEF5045
:104A20007B0827E20101A851040DF3500C01E56B4E
:104A3000E46F036A0101B8510C01E425016EE551F0
:104A400003220150AC0FE96E010E0320EA6EEF5015
:104A500084080FE3D8900101A835036AB90FE96E05
:104A6000010E0320EA6EEC6AED52800EEF6E77D0F5
:104A70000C01D8900101A835036AB90F016E010E2F
:104A8000032201C0E4FC03C0E5FC0101A851040DB0
:104A9000F3500C01E76BE66FAC0EE625E96E010EF4
:104AA000E721EA6EEF50E76BE66F0101A851040DB4
:104AB000F3500C01E96BE86F010EE825016E000E62
:104AC000E921036E0150AC0FE96E010E0320EA6E7E
:104AD000EF50036AE6270350E7230101A851040DB4
:104AE000F3500C01E96BE86F020EE825016E000E31
:104AF000E921036E0150AC0FE96E010E0320EA6E4E
:104B0000EF50036AE6270350E7230101A851040D83
:104B1000F3500C01E96BE86F030EE825016E000EFF
:104B2000E921036E0150AC0FE96E010E0320EA6E1D
:104B3000EF50036AE6270350E723E731036EE631BF
:104B4000026E033202323F0E0316E5CCEAFFE4CCDC
:104B5000E9FF03C0ECFFED5202C0EFFF0101010EBF
:104B6000B825030BB86F010EA8250C01E56FE66FA1
:104B7000030EE76F00010EDF00C0A8F10101A835A8
:104B8000006E0036FC0E0016C250C30B0010C26E41
:104B90005D2E1FD05C2A5E2A1B0E5D6E5BA80FD0B7
:104BA0000001600760530AE15B98C4C114F2C5C1FB
:104BB00015F2C4C113F24A804A82498C010158BEE1
:104BC00002D05BA006D05E50030803E2589E5B90C3
:104BD000458A9E900001DEEF03F0F294DEEF03F0D1
:104BE000C580C5B0FED70A0E006E002EFED700D0DD
:104BF0000C01EF51FE0BF26FF36F000102DE0A0EA3
:104C0000006E002EFED700D0F0CCF3FCFADD0A0EC9
:104C1000006E002EFED700D0F1CCF3FCF2DD0A0EC0
:104C2000006E002EFED700D0C584C5B4FED70D0E91
:104C3000006E002EFED7000C0C01E9510109EC6F4B
:104C4000EBCCEDFCEE6BEE6BE8CCEFFCF06FEBCC5D
:104C5000F1FC0001C5DF0C01E951FE0BEC6FEACC61
:104C6000EDFCEE6BE8CCEFFCF06FEACCF1FC000160
:104C7000B7DF000C0C01E96BEA6B010EE85DF40F85
:104C800051E20C0F000198EF26F00C01EA6B080EC0
:104C9000E96F48D00C01EA6B040EE96F43D00101C3
:104CA000C1A105D00C01EA6B010EE96F04D00C0123
:104CB000EA6B020EE96F36D00101C1A105D00C01EB
:104CC000EA6B020EE96F04D00C01EA6B010EE96F8A
:104CD00029D0800E0C01EA6FE96B24D0400E0C0144
:104CE000EA6FE96B1FD0200E0C01EA6FE96B1AD056
:104CF000100E0C01EA6FE96B15D0080E0C01EA6F7B
:104D0000E96B10D0040E0C01EA6FE96B0BD0020EB8
:104D10000C01EA6FE96B06D0010E0C01EA6FE96B3A
:104D200001D00C01E9CC01F0EACC02F00001000C4A
:104D300008AE03D0F2CF0EF0F29EE824F76AF73601
:104D4000630FF66E4D0EF722000EF86EFB6E0A0032
:104D5000F550FA6E0800F55008AE02D00EBEF28E85
:104D6000F96E184D0E4D044DFA4CF04CE64CDC4CEF
:104D7000D24CB84C9E4C944C8A4C0C01E96BEA6BBB
:104D8000E85102080EE3010EE85D006E400EE96F87
:104D9000EA6B005205E0D890E937EA37002EFBD7DE
:104DA00021D0E85104080EE3030EE85D006E400ECA
:104DB000EA6FE96B005205E0D890E937EA37002E38
:104DC000FBD710D0E85106080DE3050EE85D006E34
:104DD000400EE96FEA6B005205E0D890E937EA37F8
:104DE000002EFBD7E9CC01F0EACC02F00001000C68
:104DF0000C01E46BE56BE66BE76B58AA03D0589C9B
:104E0000A08281D1A092588C58A060D04F504D14F0
:104E1000E86F50504E14E96FE85304E1E95302E1A2
:104E200058A20BD04D50FF0A006E4E50FF0A036E81
:104E300000504F160350501604D04D504F124E5094
:104E400050125150010A000105E0030A0EE0010A68
:104E50001AE024D04C0E0C01E86FE96B50C0EBFC5B
:104E60004FC0EAFC0001E8DE1BD050C0E8FC0C019A
:104E7000E96BE96B480EEF6F010EF06F50C0F1FC6B
:104E80000001AEDE0DD04A0E0C01E86FE96B50C098
:104E9000EBFC4FC0EAFC0001CFDE02D0588200D00C
:104EA00058A205D0516A506A4F6A5890589258A03B
:104EB00006D0A082589C0C0126D108D0000158B41D
:104EC00006D0589C589458960C011DD1000158A644
:104ED00007D0589458960C01E46B596A14D100011C
:104EE00058A40ED15952D8B40BD10C01E46B59C05F
:104EF000E7FCE7510C080EE3036AE7514D0FE96E3A
:104F0000020E0320EA6EEF5203E1E7CCE4FC02D08C
:104F1000E72BEFD7E45318E1592C01D015D0010E3F
:104F2000596E59C0E7FCE7510C080EE3036AE751DC
:104F30004D0FE96E020E0320EA6EEF5203E1E7CC5B
:104F4000E4FC02D0E72BEFD7E453D8B475D0FF0EC2
:104F5000521A531A300E5216536AE4515A5C02E147
:104F6000587801D0589858B808D0E4CCE8FC000133
:104F700081DE01505212025053120EC2E8FC0001B1
:104F8000FCDE02C0E6FC01C0E5FC02010E51020895
:104F90001AE30C01E5515614E86FE6515714E96F16
:104FA000E8530BE1E95309E1E5515212E65153127E
:104FB000E5515612E651571204D03F0E5216576A69
:104FC000566A27D00201FF0E541A551A54500C018C
:104FD000E515E86F5550E615E96FE8530AE1E95326
:104FE00008E13F0E54165516E5515412E65155127C
:104FF00003D03F0E54165516FF0E541A551A4A0E7A
:10500000E86FE96B55C0EBFC54C0EAFC000114DE0C
:105010000C01FF0E521A531A4C0EE86FE96B53C085
:10502000EBFC52C0EAFC000107DEE4CC5AF0010EB2
:105030000C01E425596E5ED0592C5CD0FF0E521A3B
:10504000531AF00E5216536A0EC2E8FC000195DEA8
:1050500002C0E6FC01C0E5FC02010E51020824E397
:1050600052500C01E515E86F5350E615E96FE8530F
:105070000AE1E95308E1300E5216536AE551521223
:10508000E651531203D0300E5216536AFF0E521AD5
:10509000531A4C0EE86FE96B53C0EBFC52C0EAFCAC
:1050A0000001CADD26D00201FF0E541A551A5450D1
:1050B0000C01E515E86F5550E615E96FE8530AE174
:1050C000E95308E13F0E54165516E5515412E651C6
:1050D000551203D03F0E54165516FF0E541A551A8A
:1050E0004A0EE86FE96B55C0EBFC54C0EAFC0001C6
:1050F000A3DD0C01E7510D0802E2010E596E00011B
:10510000589CA0820C01A1920001DEEF03F09EA842
:10511000FED7AD6E000C0C01E46B9EAAFED7AECF9D
:10512000E4FC036A00016351680FE96E000E03207E
:10513000EA6EE4CCEFFF036A6351680FE96E000E7C
:105140000320EA6EEF500D0801E1652B010E632587
:10515000FF0802E1636B01D0632B5B8E47BC2ED04E
:105160000101C3A92DD00C01E451210806E0E4514E
:10517000220803E0E451300809E10001675180088A
:1051800006E26751890803E30C01E46B00010C019E
:10519000E45108080AE1E4510001B9DF200EB7DF4D
:1051A0000C01E4510001B3DF0C01E4511F0807E2D8
:1051B000E4517E0804E3E4510001A9DF0C01010180
:1051C000E4CC67F09E9A0001DEEF03F00C01E46B83
:1051D000A4AAFED76ECFE4FC47AE05D0E45100018F
:1051E00096DF15D00C01036A00016451680FE96E67
:1051F000010E0320EA6EE4CCEFFF01016781010E8E
:10520000000164253F0802E2646B01D0642BA49A7C
:10521000DEEF03F0080EEA6ED10EE96EEF500EE0FD
:10522000050E016E006A002EFED7012EFBD72E0E52
:10523000006E002EFED700D0EF2EF2D7000C080E25
:10524000EA6ED40EE96EEF500EE0050E016E006AB4
:10525000002EFED7012EFBD72E0E006E002EFED79D
:1052600000D0EF2EF2D7000C0801D939F00B006EF8
:105270000F0E8C1400108C6E00008C80020E006EDD
:10528000002EFED700008C900001000C8350006EB1
:1052900000380F0B016E000C0F0E9514F009956E7F
:1052A0008C8400008C800000F1DF01C0D9F88C9064
:1052B00000008C8000D000D0E9DF01C0D8F88C90CD
:1052C0000F0E9514956E0801D939006EF00E001678
:1052D0000050D811016E000170EF29F08C92DCD7DC
:1052E00001C0D8F8080101AE02D00001F8D78C92B5
:1052F000D6B18C8200008C9400008C90D739D86F86
:105300000F0ED817D8C8D9F80001AEDF0801D75161
:105310000F0BD86FD96F0001A7DF000C0F0E95148B
:10532000956E9590959295948C928C948C900F0E8E
:105330000801D46F000183DF010E0401C16FC15168
:1053400003080DE3030E0801D96F00018DDF050E80
:105350000801D46F000173DF0401C12BF0D7020EE6
:105360000801D96F000180DF0401C16BC15103083E
:1053700014E3036AC151F2CFC2F4F29E000103ECC0
:1053800004F00401C2BFF28EC26F0801D66BD76F62
:105390000001A4DF0401C12BE9D70001BAEFFEF040
:1053A000D1C8D3F8D0C8D2F8D3C803F00801D2C806
:1053B000E9FFD3C8EAFFEF5206E0D22BD8B4D32BD3
:1053C0000001F2D70801D051D25D006ED151D359FE
:1053D000036E00C001F00001000C0801D32D01D0C4
:1053E00003D0400ED46F01D0D46B010ED25DD42710
:1053F000D4518009D56FD66BD76F00016FDF000CD9
:105400000801D1510C0A000105E0060A0FE0020A6A
:1054100015E01BD00801D66B010ED76F00015EDFCF
:10542000020E0801D46F00010ADF17D0010E080137
:10543000D26F020ED36F0001D0DF0FD00801D66B00
:10544000100ED76F00014ADF08D0010E0801D66F99
:10545000D1C8D7F8000142DF00D0000C0801CF6BA3
:10546000CEC8D1F8CDC8D0F800019ADF0152D8B427
:105470008ED0CEC8D1F8CDC8D0F892DF0150080147
:10548000CF5DD8B085D0036ACF51CD25E96ECE511E
:105490000320EA6EEF50010A00010DE0030A26E046
:1054A000010A3FE0080A58E0070A5EE0060A5CE0ED
:1054B000020A5AE059D00801CF5317E1010ED26F0A
:1054C000D36F00018ADF200E0801D16F000198DF41
:1054D000010E0801D26F020ED36F00017EDF200E95
:1054E0000801D16F00018CDF08014ED00801CF53B5
:1054F00017E1010ED26FD36F00016FDF3E0E08017E
:10550000D16F00017DDF010E0801D26F020ED36F53
:10551000000163DF200E0801D16F000171DF080177
:1055200033D00801CF5317E1010ED26FD36F0001C2
:1055300054DF200E0801D16F000162DF010E080167
:10554000D26F020ED36F000148DF3E0E0801D16F0B
:10555000000156DF080118D0010E0801D26FD36F89
:1055600000013BDF080110D0036A0801CF51CD25AF
:10557000E96ECE510320EA6EEFCFD0F8D0C8D1F853
:1055800000013EDF080100D0CF2B000172D70801D7
:105590000001000C010E016EFCEFFEF0196AF2BE74
:1055A000198EF29E4C0E0C01E86F040EE96FEB6B46
:1055B000EA6B00011CEC26F019BEF28E196AF2BEED
:1055C000198EF29E4C0E0C01E86F060EE96FEB6B24
:1055D000EA6B00011CEC26F019BEF28E196AF2BECD
:1055E000198EF29E4C0E0C01EF6F0B0EF06FF16BEB
:1055F0000001F0EC25F019BEF28E196AF2BE198E88
:10560000F29E480E0C01E86F040EE96FEB6BEA6B3B
:1056100000011CEC26F019BEF28E196AF2BE198E3A
:10562000F29E480E0C01E86F060EE96FEB6BEA6B19
:1056300000011CEC26F019BEF28E196AF2BE198E1A
:10564000F29E480E0C01EF6F0A0EF06FF16B000135
:10565000F0EC25F019BEF28E196AF2BE198EF29E98
:105660004A0E0C01E86F040EE96FEB6BEA6B000168
:105670001CEC26F019BEF28E196AF2BE198EF29E4B
:105680004A0E0C01E86F060EE96FEB6BEA6B000146
:105690001CEC26F019BEF28E196AF2BE198EF29E2B
:1056A0004A0E0C01EF6F0A0EF06FF16B0001F0EC87
:1056B00025F019BEF28E196AF2BE198EF29E400EC6
:1056C0000C01E86F040EE96FEB6BEA6B00011CEC58
:1056D00026F019BEF28E196AF2BE198EF29E400EA5
:1056E0000C01E86F060EE96FEB6BEA6B00011CEC36
:1056F00026F019BEF28E196AF2BE198EF29E400E85
:105700000C01EF6F0A0EF06FF16B0001F0EC25F069
:1057100019BEF28E196AF2BE198EF29E440E0C0169
:10572000E86F040EE96FEB6BEA6B00011CEC26F0EE
:1057300019BEF28E196AF2BE198EF29E440E0C0149
:10574000E86F060EE96FFF0EEB6FEA6F00011CECCD
:1057500026F019BEF28E196AF2BE198EF29E440E20
:105760000C01EF6F0A0EF06FF16B0001F0EC25F009
:1057700019BEF28E196AF2BE198EF29E420E0C010B
:10578000E86F040EE96FEB6BEA6B00011CEC26F08E
:1057900019BEF28E196AF2BE198EF29E420E0C01EB
:1057A000E86F060EE96FFF0EEB6FEA6F00011CEC6D
:1057B00026F019BEF28E196AF2BE198EF29E420EC2
:1057C0000C01EF6F0A0EF06FF16B0001F0EC25F0A9
:1057D00019BEF28E196AF2BE198EF29E460E0C01A7
:1057E000E86F040EE96FEB6BEA6B00011CEC26F02E
:1057F00019BEF28E196AF2BE198EF29E460E0C0187
:10580000E86F060EE96FFF0EEB6FEA6F00011CEC0C
:1058100026F019BEF28E196AF2BE198EF29E460E5D
:105820000C01EF6F0A0EF06FF16B0001F0EC25F048
:1058300019BEF28E25EFFFF00401F551010A0001B7
:105840000AE0030AD8B4CFD0010AD8B494D1030A2D
:10585000D8B459D258D2020EEA6E5A0EE96EF2CF7F
:10586000F6F4F29E000EB9EC08F00A000900F550BB
:10587000EE6E0009FBE10401F6BFF28E020EEA6E45
:105880006C0EE96EF2CFF6F4F29E000E0001D1EC40
:1058900008F00A000900F550EE6E0009FBE1040172
:1058A000F6BFF28E020EEA6E7E0EE96EF2CFF6F4CD
:1058B000F29E000E0001E9EC08F00A000900F55024
:1058C000EE6E0009FBE10401F6BFF28E020EEA6EF5
:1058D000900EE96EF2CFF6F4F29E000E000101EC9C
:1058E00009F00A000900F550EE6E0009FBE1040121
:1058F000F6BFF28E020EEA6EA20EE96EF2CFF6F459
:10590000F29E000E000119EC09F00A000900F550A2
:10591000EE6E0009FBE10401F6BFF28E020EEA6EA4
:10592000B40EE96EF2CFF6F4F29E000E000131ECF7
:1059300009F00A000900F550EE6E0009FBE10401D0
:10594000F6BFF28E020EEA6EC60EE96EF2CFF6F4E4
:10595000F29E000E000149EC09F00A000900F55022
:10596000EE6E0009FBE10401F6BFF28E020EEA6E54
:10597000D80EE96EF2CFF6F4F29E000E000161EC53
:1059800009F00A000900F550EE6E0009FBE1040180
:10599000F6BFF28E020EEA6EEA0EE96EF2CFF6F470
:1059A000F29E000E000179EC09F00A000900F550A2
:1059B000EE6E0009FBE10401F6BFF28E010E030159
:1059C000C26F036AC251CB0FE96E030E0320EA6E69
:1059D000080EEF6E036AC251CF0FE96E030E03206B
:1059E000EA6EEF6A45D2020EEA6E5A0EE96EF2CF07
:1059F000F6F4F29E000E91EC09F00A000900F55051
:105A0000EE6E0009FBE10401F6BFF28E020EEA6EB3
:105A10006C0EE96EF2CFF6F4F29E000E0001A9ECD6
:105A200009F00A000900F550EE6E0009FBE10401DF
:105A3000F6BFF28E020EEA6E7E0EE96EF2CFF6F43B
:105A4000F29E000E0001C1EC09F00A000900F550B9
:105A5000EE6E0009FBE10401F6BFF28E020EEA6E63
:105A6000900EE96EF2CFF6F4F29E000E0001D9EC32
:105A700009F00A000900F550EE6E0009FBE104018F
:105A8000F6BFF28E020EEA6EA20EE96EF2CFF6F4C7
:105A9000F29E000E0001F1EC09F00A000900F55039
:105AA000EE6E0009FBE10401F6BFF28E020EEA6E13
:105AB000B40EE96EF2CFF6F4F29E000E000109EC8E
:105AC0000AF00A000900F550EE6E0009FBE104013E
:105AD000F6BFF28E020EEA6EC60EE96EF2CFF6F453
:105AE000F29E000E000121EC0AF00A000900F550B8
:105AF000EE6E0009FBE10401F6BFF28E020EEA6EC3
:105B0000D80EE96EF2CFF6F4F29E000E000139ECE9
:105B10000AF00A000900F550EE6E0009FBE10401ED
:105B2000F6BFF28E020EEA6EEA0EE96EF2CFF6F4DE
:105B3000F29E000E000179EC09F00A000900F55010
:105B4000EE6E0009FBE10401F6BFF28E020E0301C6
:105B5000C26F036AC251CB0FE96E030E0320EA6ED7
:105B6000080EEF6E036AC251CF0FE96E030E0320D9
:105B7000EA6EEF6A7DD1020EEA6E5A0EE96EF2CF3E
:105B8000F6F4F29E000E51EC0AF00A000900F550FE
:105B9000EE6E0009FBE10401F6BFF28E020EEA6E22
:105BA0006C0EE96EF2CFF6F4F29E000E0001A9EC45
:105BB00009F00A000900F550EE6E0009FBE104014E
:105BC000F6BFF28E020EEA6E7E0EE96EF2CFF6F4AA
:105BD000F29E000E0001C1EC09F00A000900F55028
:105BE000EE6E0009FBE10401F6BFF28E020EEA6ED2
:105BF000900EE96EF2CFF6F4F29E000E0001D9ECA1
:105C000009F00A000900F550EE6E0009FBE10401FD
:105C1000F6BFF28E020EEA6EA20EE96EF2CFF6F435
:105C2000F29E000E0001F1EC09F00A000900F550A7
:105C3000EE6E0009FBE10401F6BFF28E020EEA6E81
:105C4000B40EE96EF2CFF6F4F29E000E000109ECFC
:105C50000AF00A000900F550EE6E0009FBE10401AC
:105C6000F6BFF28E020EEA6EC60EE96EF2CFF6F4C1
:105C7000F29E000E000121EC0AF00A000900F55026
:105C8000EE6E0009FBE10401F6BFF28E020EEA6E31
:105C9000D80EE96EF2CFF6F4F29E000E000139EC58
:105CA0000AF00A000900F550EE6E0009FBE104015C
:105CB000F6BFF28E020EEA6EEA0EE96EF2CFF6F44D
:105CC000F29E000E000179EC09F00A000900F5507F
:105CD000EE6E0009FBE10401F6BFF28E030E030134
:105CE000C26F036AC251CB0FE96E030E0320EA6E46
:105CF000080EEF6E036AC251CF0FE96E030E032048
:105D0000EA6EEF6AB5D0020EEA6E5A0EE96EE26AEA
:105D1000320EE16EE752E6CFEEFFFCE1020EEA6ED4
:105D20006C0EE96EE26A200EE16EE752E6CFEEFFFE
:105D3000FCE1020EEA6E7E0EE96EF2CFF6F4F29E00
:105D4000000E69EC0AF00A000900F550EE6E000939
:105D5000FBE10401F6BFF28E020EEA6E900EE96ED0
:105D6000F2CFF6F4F29E000E000181EC0AF00A0078
:105D70000900F550EE6E0009FBE10401F6BFF28E5A
:105D8000020EEA6EA20EE96EF2CFF6F4F29E000E5B
:105D9000000199EC0AF00A000900F550EE6E0009C6
:105DA000FBE10401F6BFF28E020EEA6EB40EE96E5C
:105DB000F2CFF6F4F29E000E0001B1EC0AF00A00F8
:105DC0000900F550EE6E0009FBE10401F6BFF28E0A
:105DD000020EEA6EC60EE96EF2CFF6F4F29E000EE7
:105DE0000001C9EC0AF00A000900F550EE6E000946
:105DF000FBE10401F6BFF28E020EEA6ED80EE96EE8
:105E0000F2CFF6F4F29E000E0001E1EC0AF00A0077
:105E10000900F550EE6E0009FBE10401F6BFF28EB9
:105E2000020EEA6EEA0EE96EF2CFF6F4F29E000E72
:105E30000001F9EC0AF00A000900F550EE6E0009C5
:105E4000FBE10401F6BFF28E0301C26B036AC2518B
:105E5000CB0FE96E030E0320EA6E120EEF6E036A9B
:105E6000C251CF0FE96E030E0320EA6EEF6A00D035
:105E70000001000C0801CE6703D0CF6702D007D025
:105E8000CF2BCDC8EEFFCE2FFCD7CF2FFAD70001F6
:105E9000000CCEC8D3F8CDC8D2F80801D15324E005
:105EA000D0C803F0CFC8E9FFD0C8EAFFEF521CE02A
:105EB000D3C803F0D251D22BD8B4D32BD46F03C0A4
:105EC000D5F8D0C803F0CF51CF2BD8B4D02BE96E82
:105ED00003C0EAFFEFCFD6F8D5C8EAFFD4C8E9FF80
:105EE000D6C8EFFFD107DAD7D1530CE0D3C803F0FF
:105EF000D251D22BD8B4D32BE96E03C0EAFFEF6A9C
:105F0000D107F2D7CDC801F0CEC802F00001000CD5
:105F1000010167B329D0080EEA6EA70EE96E0801E9
:105F2000CD6BCF6B130ECE6F0001A4DF080E0801FE
:105F3000CE6FA70ECD6F020ED06F5A0ECF6F120E1E
:105F4000D16F0001A6DF0C0E0801A76F080ECE6FFF
:105F5000A70ECD6F00012EEC2AF0050E0801D46FBC
:105F600000011FEC29F00101080EEA6EBA0EE96E7D
:105F70000801CD6BCF6B130ECE6F00017BDF080ED7
:105F80000801CE6FBA0ECD6FA6C8D0F8A5C8CFF85D
:105F9000120ED16F00017DDF0A0E0801BA6F080EE4
:105FA000CE6FBA0ECD6F00012EEC2AF0000C04016A
:105FB000D6C4E9FFD7C4EAFFEFCFDAF4D9C403F0BF
:105FC000D8C4E9FFD9C4EAFFEF50DA5D15E1D7C4C0
:105FD00003F0D6C4E9FF03C0EAFFEF5203E1000E6D
:105FE000016E1FD0D7C403F0D651D62BD8B4D72B0F
:105FF000D82BD8B4D92BDCD7D7C403F0D6C4E9FF4B
:10600000D7C4EAFFEFCFDAF4D9C403F0D8C4E9FF6C
:10601000D9C4EAFFEF50DA5D02E2FF0E01D0010EB3
:10602000016E000156EF30F00401C16BC26BC36B0F
:10603000200EC46FC56FC66FC76FC86FC96FCA6FB8
:10604000CB6FCC6FCD6FCE6FCF6FD06FD16FD26F64
:10605000D36FD46B030EC36FE70EC26FC16BC15118
:1060600011081BE3036AC151C40FE96E040E03203B
:10607000EA6EF2CFD8F4F29EC3C4AAFFC2C4A9FF4D
:10608000A69CA69EA680A850D8BFF28EEF6E010EE9
:10609000C227000EC323C12BE2D7040ED76FC40E54
:1060A000D66FD96B320ED86F000181D7015204E14F
:1060B000010E016E04D003D0000E016E00D0A9EFD6
:1060C000FFF00401DC6BDD6BDE6BF2CFDFF4F29EE0
:1060D000030EAA6EFF0EA96EA69CA69EA680A850CF
:1060E000DFBFF28EDE6FDD6BDC6BDD5103081CE37E
:1060F000DDC4AAFFDCC4A9FFFF0EA86EA69CA69E65
:10610000A684F2CF00F0F29E0F01550EA76EAA0EE4
:10611000A76EA682A6B2FED7A6940050F212040182
:10612000DC2BD8B4DD2BE1D7DE51010819E3030ED7
:10613000AA6EFF0EA96EDEC4A8FFA69CA69EA6842A
:10614000F2CF00F0F29E0F01550EA76EAA0EA76EB9
:10615000A682A6B2FED7A6940050F21217D0040170
:10616000030EAA6EFF0EA96EA86AA69CA69EA68420
:10617000F2CF00F0F29E0F01550EA76EAA0EA76E89
:10618000A682A6B2FED7A6940050F21200011BEF21
:1061900031F00401DC6BDD6BDE6BDF6BE06BDD6B24
:1061A000200EDC6FDE6BDE5105082DE3DF6BDF5167
:1061B0000B0827E3E06BE0510B0821E3DDC403F09B
:1061C000DC51DC2BD8B4DD2BE16F03C0E2F403C05B
:1061D000AAFFA96EA86AA69CA69EA684F2CF00F08C
:1061E000F29E0F01550EA76EAA0EA76EA682A6B24A
:1061F000FED7A6940050F2120401E02BDCD7DF2B6F
:10620000D6D7DE2BD0D7DE6BDE510C080AE3036A4B
:10621000DE514D0FE96E020E0320EA6EEF6ADE2BAF
:10622000F3D70001000C0401D76BD86BD96BDA6B84
:10623000DB6B000146D7AA6AA96A010EA86EA69C6C
:10624000A69EA684F2CF00F0F29E0F01550EA76E17
:10625000AA0EA76EA682A6B2FED7A6940050F2128E
:10626000AA6A010EA96EA86EA69CA69EA684F2CF6D
:1062700000F0F29E550EA76EAA0EA76EA682A6B2D9
:10628000FED7A6940050F212AA6A020EA96E0F0E53
:10629000A86EA69CA69EA684F2CF00F0F29E550E94
:1062A000A76EAA0EA76EA682A6B2FED7A69400502D
:1062B000F212AA6A100EA96EA86AA69CA69EA684CF
:1062C000F2CF00F0F29E550EA76EAA0EA76EA68220
:1062D000A6B2FED7A6940050F212AA6A030EA96EC7
:1062E000120EA86EA69CA69EA684F2CF00F0F29E87
:1062F000550EA76EAA0EA76EA682A6B2FED7A694CA
:106300000050F212AA6A0F0EA96EA86AA69CA69E59
:10631000A684F2CF00F0F29E550EA76EAA0EA76ECD
:10632000A682A6B2FED7A6940050F212AA6A040E64
:10633000A96EA86EA69CA69EA684F2CF00F0F29E3F
:10634000550EA76EAA0EA76EA682A6B2FED7A69479
:106350000050F212AA6A050EA96EA86EA69CA69E0F
:10636000A684F2CF00F0F29E550EA76EAA0EA76E7D
:10637000A682A6B2FED7A6940050F212AA6A060E12
:10638000A96E180EA86EA69CA69EA684F2CF00F059
:10639000F29E550EA76EAA0EA76EA682A6B2FED7D3
:1063A000A6940050F212AA6A070EA96E040EA86EF7
:1063B000A69CA69EA684F2CF00F0F29E550EA76E74
:1063C000AA0EA76EA682A6B2FED7A6940050F2121D
:1063D000F2CFDCF4F29E030EAA6EFF0EA96EA69C0D
:1063E000A69EA680A8500401DCBFF28EDD6FAA6ACB
:1063F000080EA96EDDC4A8FFA69CA69EA684F25036
:10640000006EF29E0F01550EA76EAA0EA76EA68211
:10641000A6B2FED7A6940050F212AA6A090EA96E7F
:10642000190EA86EA69CA69EA684F2CF00F0F29E3E
:10643000550EA76EAA0EA76EA682A6B2FED7A69488
:106440000050F212AA6A0A0EA96E180EA86EA69C37
:10645000A69EA684F2CF00F0F29E550EA76EAA0E5D
:10646000A76EA682A6B2FED7A6940050F212AA6A20
:106470000B0EA96E180EA86EA69CA69EA684F2CF3F
:1064800000F0F29E550EA76EAA0EA76EA682A6B2C7
:10649000FED7A6940050F212AA6A0C0EA96E0E0E38
:1064A000A86EA69CA69EA684F2CF00F0F29E550E82
:1064B000A76EAA0EA76EA682A6B2FED7A69400501B
:1064C000F212AA6A0D0EA96EA86AA69CA69EA684C0
:1064D000F2CF00F0F29E550EA76EAA0EA76EA6820E
:1064E000A6B2FED7A6940050F212AA6A0E0EA96EAA
:1064F000A86AA69CA69EA684F2CF00F0F29E550E36
:10650000A76EAA0EA76EA682A6B2FED7A6940050CA
:10651000F212AA6A120EA96EA86AA69CA69EA6846A
:10652000F2CF00F0F29E550EA76EAA0EA76EA682BD
:10653000A6B2FED7A6940050F21200012ADE030E86
:106540000401D86FE70ED76FDB6BDB51110827E32F
:10655000036ADB51320FE96E000E0320EA6EEFCFC3
:10656000DCF4D8C4AAFFD7C4A9FFDCC4A8FFA69C4A
:10657000A69EA684F2CF00F0F29E0F01550EA76EE4
:10658000AA0EA76EA682A6B2FED7A6940050F2125B
:10659000010E0401D727000ED823DB2BD6D7DA6BE8
:1065A000D96BDB6BDB51110843E3036ADB51200F2E
:1065B000E96E000E0320EA6EEFCFDCF4DC512F0809
:1065C00003E2DC51390802E2000E01D0010E01089D
:1065D0002DE1DA532BE1D951050828E3036ADB5199
:1065E000200FE96E000E0320EA6EEFCFDCF4D8C472
:1065F000AAFFD7C4A9FFDCC4A8FFA69CA69EA684B8
:10660000F2CF00F0F29E0F01550EA76EAA0EA76EF4
:10661000A682A6B2FED7A6940050F2120401D92B8E
:10662000D8B4DA2B010ED727000ED823DB2BBAD72C
:106630000001000C0C01DF51E103F3CF01F0F4CFB6
:1066400000F0E203F3500026E051E103F350002094
:10665000026E0001000C0801D6BF10D00F0E006EB4
:10666000D53900160A0E005C03E2300E002602D077
:10667000D651002600509EA8FED7AD6E0F0ED5173E
:106680000A0ED55D02E2300E02D0D69FD651D52734
:10669000D5519EA8FED7AD6E0001000C0501246BFC
:1066A000256B266B225303E02251060804E2000EFC
:1066B000016E13D208D0235303E023510C0803E2E8
:1066C000000E016E0AD2256B900E246F010E225D22
:1066D000036A276F03C028F525C5E0FC24C5DFFC4D
:1066E00003C0E2FCE8CFE1FC0001A4DF02C025F515
:1066F00001C024F5200E05012427000E2523010EDC
:10670000235D0C0DF350036A242703502523010158
:10671000C2A127D00501276B2751000114EC04F01A
:106720000501272B000187EC28F00E0E0501275DDF
:10673000F3E125C5D5F8370E0801D66F00018BDFD0
:1067400024C5D5F8370E0801D66F000184DF200E6E
:1067500087EC28F00A0E87EC28F00D0E87EC28F065
:10676000010105012551036E2451242BD8B4252B9A
:10677000276F03C028F5F2CF29F5F29E28C5AAFF9E
:1067800027C5A9FFA69CA69EA680A85029BFF28E69
:10679000266F2651F00BD8B49DD12651F00B276FF0
:1067A0000101D151F00B0501275DD8A493D126C575
:1067B000D1F12551036E2451242BD8B4252B276FFA
:1067C00003C028F5F2CF29F5F29E28C5AAFF27C5F8
:1067D000A9FFA69CA69EA680A85029BFF28E010103
:1067E000D26F05012551036E2451242BD8B4252BDB
:1067F000276F03C028F5F2CF29F5F29E28C5AAFF1E
:1068000027C5A9FFA69CA69EA680A85029BFF28EE8
:106810000101D46FD36B05012551036E2451242B44
:10682000D8B4252B276F03C028F5F2CF29F5F29EA7
:1068300028C5AAFF27C5A9FFA69CA69EA680A8508A
:1068400029BFF28E0101D31305012551036E245196
:10685000242BD8B4252B276F03C028F5F2CF29F5B8
:10686000F29E28C5AAFF27C5A9FFA69CA69EA680C2
:10687000A85029BFF28E0101D66FD56B05012551B5
:10688000036E2451242BD8B4252B276F03C028F581
:10689000F2CF29F5F29E28C5AAFF27C5A9FFA69C1D
:1068A000A69EA680A85029BFF28E0101D51305012E
:1068B0002551036E2451242BD8B4252B276F03C0F8
:1068C00028F5F2CF29F5F29E28C5AAFF27C5A9FF12
:1068D000A69CA69EA680A85029BFF28E0101D86F63
:1068E000D76B05012551036E2451242BD8B4252BD9
:1068F000276F03C028F5F2CF29F5F29E28C5AAFF1D
:1069000027C5A9FFA69CA69EA680A85029BFF28EE7
:106910000101D71305012551036E2451242BD8B44E
:10692000252B276F03C028F5F2CF29F5F29E28C545
:10693000AAFF27C5A9FFA69CA69EA680A85029BF8E
:10694000F28E0101DA6FD96B05012551036E2451D6
:10695000242BD8B4252B276F03C028F5F2CF29F5B7
:10696000F29E28C5AAFF27C5A9FFA69CA69EA680C1
:10697000A85029BFF28E0101D91305012551036EDC
:106980002451242BD8B4252B276F03C028F5F2CF30
:1069900029F5F29E28C5AAFF27C5A9FFA69CA69E99
:1069A000A680A85029BFF28E0101DC6FDB6BF2CF0D
:1069B00027F5F29E25C5AAFF24C5A9FFA69CA69E81
:1069C000A680A850050127BFF28E0101DB13C2A1EA
:1069D0007CD00501276B275100012EEC04F0050146
:1069E000272B000187EC28F0050E0501275DF3E158
:1069F000D1C1D5F8570E0801D66F00012CDE200E4C
:106A000087EC28F0D2C1D5F8570E0801D66F0001E7
:106A100022DE200E87EC28F0D4C1D5F8370E08010D
:106A2000D66F000118DED3C1D5F8370E0801D66F36
:106A3000000111DE200E87EC28F0D6C1D5F8370E04
:106A40000801D66F000107DED5C1D5F8370E080161
:106A5000D66F000100DE200E87EC28F0D8C1D5F8F3
:106A6000370E0801D66F0001F6DDD7C1D5F8370E15
:106A70000801D66F0001EFDD200E87EC28F0DAC1A7
:106A8000D5F8370E0801D66F0001E5DDD9C1D5F87C
:106A9000370E0801D66F0001DEDD200E87EC28F0EE
:106AA000DCC1D5F8370E0801D66F0001D4DDDBC19B
:106AB000D5F8370E0801D66F0001CDDD0A0E87EC40
:106AC00028F00D0E87EC28F00101010E016E050182
:106AD00004D003D0000E016E00D00001000CF2CFF4
:106AE000EDF4F29EAA6AA96AA69CA69EA680A8506A
:106AF0000401EDBFF28E0101C46FF2CFEDF4F29EFE
:106B0000AA6A010EA96EA69CA69EA680A8500401A2
:106B1000EDBFF28E0101C56FF2CFEDF4F29EAA6ACD
:106B2000020EA96EA69CA69EA680A8500401EDBFE9
:106B3000F28E0101C66FF2CFEDF4F29EAA6A100E3A
:106B4000A96EA69CA69EA680A8500401EDBFF28E59
:106B50000101C96FF2CFEDF4F29EAA6A030EA96E8D
:106B6000A69CA69EA680A8500401EDBFF28E01014E
:106B7000C76FF2CFEDF4F29EAA6A0F0EA96EA69C23
:106B8000A69EA680A8500401EDBFF28E0101C86F39
:106B9000F2CFEDF4F29EAA6A040EA96EA69CA69E00
:106BA000A680A8500401EDBFF28E0101CA6FF2CF9A
:106BB000EDF4F29EAA6A050EA96EA69CA69EA6807A
:106BC000A8500401EDBFF28E0101CB6FF2CFEDF4BE
:106BD000F29EAA6A060EA96EA69CA69EA680A85042
:106BE0000401EDBFF28E0101C36FF2CFEDF4F29E0E
:106BF000AA6A070EA96EA69CA69EA680A8500401AC
:106C0000EDBFF28E0101C26FF2CFEDF4F29EAA6ADF
:106C1000080EA96EA69CA69EA680A8500401EDBFF2
:106C2000F28E0101C16FF2CFEDF4F29EAA6A090E55
:106C3000A96EA69CA69EA680A8500401EDBFF28E68
:106C40000101CC6FF2CFEDF4F29EAA6A0A0EA96E92
:106C5000A69CA69EA680A8500401EDBFF28E01015D
:106C6000CD6FF2CFEDF4F29EAA6A0B0EA96EA69C30
:106C7000A69EA680A8500401EDBFF28E0101CE6F42
:106C8000F2CFEDF4F29EAA6A0C0EA96EA69CA69E07
:106C9000A680A8500401EDBFF28E0101CF6FF2CFA4
:106CA000EDF4F29EAA6A0D0EA96EA69CA69EA68081
:106CB000A8500401EDBFF28E0101BF6FF2CFEDF4D9
:106CC000F29EAA6A0E0EA96EA69CA69EA680A85049
:106CD0000401EDBFF28E0101C06FF2CFEDF4F29E20
:106CE000AA6A120EA96EA69CA69EA680A8500401B0
:106CF000EDBFF28E0101D06FCF51280802E2280EBD
:106D0000CF6FCD51180802E2180ECD6FCE51180882
:106D100002E2140ECE6FC4C122F5C5C123F50001F5
:106D2000BDDC010E016E03EF6FF0036A6151680F65
:106D3000E96E000E0320EA6EEFCF42F50501010E69
:106D4000000161250501446F196AF2BE198EF29E99
:106D5000E8CFE6FCFF0E0C01E76F0001CAEC24F05F
:106D600019BEF28E00C061F06351615D01E15B9E6E
:106D7000050142C501F00001000C0501246B5BAE6A
:106D800006D00001D2DF01C024F50501F8D70001CB
:106D9000656B000C0501276B286B296B25C5EAFF85
:106DA00024C5E9FF0801CD6BCF6B26C5CEF80001E5
:106DB0003AEC2FF00501286B276B2851030814E3E8
:106DC00003E12751E70810E3020E0801D16F00012B
:106DD0000AEC29F0655303E0050106D00001050126
:106DE000272BD8B4282BE9D70001655303E1000E07
:106DF000016E79D00501296B5BAE73D0036A29510E
:106E00002425016E2551032201C02AF503C02BF56C
:106E100000018BDF2BC5EAFF2AC5E9FF01C0EFFFA8
:106E2000036A050129512425E96E25510320EA6EE4
:106E3000EF500D083FE100016507050124C5E9FF9A
:106E400025C5EAFFEF50450818E1010E2425E96E3B
:106E5000000E2521EA6EEF50300809E0010E2425CE
:106E6000E96E000E2521EA6EEF50310806E1000EB2
:106E7000016E000138D008D005012951020805E251
:106E8000010E016E00012FD00501296B320E0801A1
:106E9000D16F00010AEC29F025C5EAFF24C5E9FFFE
:106EA0000801CD6BCF6B26C5CEF800013AEC2FF070
:106EB00016D00501036A29512425E96E25510320C6
:106EC000EA6EEF500A0805E0292B2651295D01E3FF
:106ED000296B0A0E0801D16F00010AEC29F00501A7
:106EE0008BD7000E016E0001000C0501126B126BB6
:106EF00010C5EAFF0FC5E9FF0801CD6BCF6B11C5C7
:106F0000CEF800013AEC2FF06553D8B46CD05BAEEC
:106F10006AD0036A050112510F25016E1051032238
:106F200001C013F503C014F50001FFDE14C5EAFF2C
:106F300013C5E9FF01C0EFFF036A050112510F25D8
:106F4000E96E10510320EA6EEF500D083BE100019D
:106F5000650705010FC5E9FF10C5EAFFEF504508B9
:106F600016E1010E0F25E96E000E1021EA6EEF50BA
:106F7000300809E0010E0F25E96E000E1021EA6EBF
:106F8000EF50310804E1000E016E30D006D01251EE
:106F9000020803E2010E016E29D0126B320E0801C5
:106FA000D16F00010AEC29F010C5EAFF0FC5E9FF17
:106FB0000801CD6BCF6B11C5CEF800013AEC2FF074
:106FC00011D00501036A12510F25E96E10510320FB
:106FD000EA6EEF500A0805E0122B1151125D01E331
:106FE000126B000194D7000E016E05010001000C28
:106FF0000401F06BF191F1B11DD10001BEDE04017D
:10700000F26BF251000110EC19F00401F22B0001B7
:1070100087EC28F0040E0401F25DF3E1EEC425F5DF
:10702000EDC424F5EFC426F50001B4DE015211E1F0
:107030009D9A640E0801D16F00010AEC29F09DDED3
:107040009D8AC00EF212640E0801D16F00010AEC95
:1070500029F0EEC425F5EDC424F5EFC426F59ADE3B
:10706000012CDBD00401EDC4E9FFEEC4EAFFEF50D0
:10707000450816E1010EED25E96E000EEE21EA6EDF
:10708000EF5066080DE1020EED25E96E000EEE21CF
:10709000EA6EEF50660804E1010E016ECDD049D0D2
:1070A000EDC4E9FFEEC4EAFFEF50520842E1010EE1
:1070B000ED25E96E000EEE21EA6EEF50650839E12C
:1070C000020EED25E96E000EEE21EA6EEF50630828
:1070D00030E1030EED25E96E000EEE21EA6EEF5071
:1070E0006F0827E1040EED25E96E000EEE21EA6E31
:1070F000EF506E081EE1050EED25E96E000EEE2143
:10710000EA6EEF50660815E1060EED25E96E000EF9
:10711000EE21EA6EEF5069080CE1070EED25E96EED
:10712000000EEE21EA6EEF50670803E1010E016EDA
:1071300083D0EEC410F5EDC40FF5EFC411F50001D6
:10714000D4DE012C69D00401EDC4E9FFEEC4EAFFEE
:10715000EF50450816E1010EED25E96E000EEE2117
:10716000EA6EEF5066080DE1020EED25E96E000EA5
:10717000EE21EA6EEF50660804E1010E016E5CD06C
:1071800049D0EDC4E9FFEEC4EAFFEF50520842E1F6
:10719000010EED25E96E000EEE21EA6EEF50650856
:1071A00039E1020EED25E96E000EEE21EA6EEF5098
:1071B000630830E1030EED25E96E000EEE21EA6E64
:1071C000EF506F0827E1040EED25E96E000EEE2169
:1071D000EA6EEF506E081EE1050EED25E96E000E19
:1071E000EE21EA6EEF50660815E1060EED25E96E18
:1071F000000EEE21EA6EEF5069080CE1070EED2556
:10720000E96E000EEE21EA6EEF50670803E1010E11
:10721000016E12D08ED700011CD7640E0801D16F09
:1072200000010AEC29F00401F02BF051020801E200
:10723000F181E1D6000E016E0001D6EF6FF0580E1D
:107240000801D16F036A00016251680FE96E010EF7
:107250000320EA6EEFCFD1F80801010E000162258C
:107260003F0B626F6451625D02E1010167910801A9
:10727000D1C801F00001000C640E0801D46F0001B8
:107280001FEC29F00101C2A107D00D0E000187EC0F
:1072900028F00A0E87EC28F000016451625D1AE0C4
:1072A000CEDF01C0EEF40101C2A10DD0EEC4D5F8CD
:1072B000570E0801D66F00012BEC33F0200E87EC3F
:1072C00028F007D00101320E0801D46F00011FEC35
:1072D00029F0E3D7000C200E0801ACA9300EAD6FE9
:1072E000ABC800F0ABAF07D0001E002A00C0ABF85F
:1072F0002D0EAD6FAC8F0150196AF2BE198EF29E41
:10730000ABC8E6FC640E0C01E76F0001CAEC24F088
:1073100019BEF28E00C0ABF8300E01240801AE6F2A
:10732000196AF2BE198EF29EABC8E6FC0A0E0C0179
:10733000E76F0001CAEC24F019BEF28E300E002473
:107340000801B06F300E0124AF6FADC800F0ACA7DC
:1073500002D0ACAFAC95ACB90BD0ACAF22D0ACB5D1
:1073600020D000C0AEF8ACB31CD000C0AFF819D02C
:10737000300EAE5D16E100C0AEF8200EAD6FACA7CA
:1073800004D0AC95AC83ACAFAC93300EAF5D09E1EB
:1073900000C0AFF8200EAE6FACA7F7D7AC93ACAF80
:1073A000AC91ACA504D0AD519EA8FED7AD6EACA3F8
:1073B00004D0AE519EA8FED7AD6EACA104D0AF51A3
:1073C0009EA8FED7AD6EB0519EA8FED7AD6E00014F
:1073D000000CA4A8FED76D6E000C0801D26BD36B15
:1073E000D0C8E9FFD1C8EAFFEFCFD3F8D353D8B460
:1073F00078D00101C2A107D00D0E000187EC28F062
:107400000A0E87EC28F0010E0801D26FD251D35D2D
:1074100068E30101C2A14FD0D139006E0F0E0016F2
:1074200000500D0832E1036A0801D251D025E96EFF
:10743000D1510320EA6EEF501F0812E2036AD251C5
:10744000D025E96ED1510320EA6EEFCFD4F8D451A4
:10745000000187EC28F0200E87EC28F014D00801FA
:10746000036AD251D025E96ED1510320EA6EEFCFE5
:10747000D4F8D4C8D5F8570ED66F00012BEC33F0F2
:10748000200E87EC28F015D00101036A0801D251C3
:10749000D025E96ED1510320EA6EEFCFD4F8D4C8DD
:1074A000D5F8570ED66F00012BEC33F0200E87EC89
:1074B00028F007D00101010E0801D46F00011FEC74
:1074C00029F0036A0801D251D025E96ED151032079
:1074D000EA6EEFCFD4F8D45100017BDF0801D22B44
:1074E00095D70001000CEACFCBF8E9CFCAF8080124
:1074F000C4AF08D0CA8FCAA9CA2BC31FC41FC32BCD
:10750000D8B4C42BC439F009C66FC627E20FC76FC1
:10751000320FC96FC4510F0BC727C727C927E90FFF
:10752000C86FC827C827C3390F0BC827C927C83752
:10753000C937C91FC937C3510F0BC927C637070E33
:10754000C56F0A0EC807C927FDE3C707C827FDE3B3
:10755000C607C727FDE3C507C627FDE3080EEA6E89
:10756000C50EE96E070ECA15CA9DE906CA1507E1E0
:10757000CAB9E92ACAB903D0200E006E1CD0E92688
:10758000C90EE95CD8B4CA8DEF50006E08E1CABDDF
:1075900006D0CAB914D0CAB702D0200E0BD0CAAFD9
:1075A00006D02D0E006EED50CA9DCA9F04D0CA872A
:1075B000CA99300E002600509EA8FED7AD6EEE5040
:1075C000CAADDED70001000C0801BE6BBF6BC06BFB
:1075D000C16BC291010167B151D0C1C8E0FCC0C804
:1075E000DFFC0C01E26B320EE16F00011AEC33F0AC
:1075F00002C0C4F801C0C3F80801B151025C33E312
:1076000003E1B051C35D2FE30101C2A128D00801FD
:10761000C36BC351000119EC11F00801C32B000129
:1076200087EC28F0170E0801C35DF3E1100EE96E38
:10763000B1C8C4F8B0C8C3F8000155DF1A0E08017C
:10764000C36FC351000119EC11F00801C32B0001F5
:1076500087EC28F0210E0801C35DF3E10101000E63
:10766000016EF6D00801320ED46F00011FEC29F034
:107670000801C02BD8B4C12BADD70101080EEA6EAA
:10768000B20EE96E0801CD6BCF6B0C0ECE6F000110
:107690003AEC2FF00101C2A11ED00801C36BC35107
:1076A000000139EC11F00801C32B000187EC28F030
:1076B0000F0E0801C35DF3E1100EE96EB1C8C4F806
:1076C000B0C8C3F800010FDF290E87EC28F0200EA8
:1076D00087EC28F0010167A1BBD00001B0DD01C03B
:1076E000BEF80801C2A167D0BE3D36D00101C2A1DB
:1076F0000CD0BEC8D5F8370E0801D66F00012BECB0
:1077000033F0200E87EC28F001010801B351410845
:1077100003E0B351420806E1010E016E010198D069
:1077200019D00801B351510803E0B35152080EE1DA
:10773000080EEA6EB20EE96ECD6BCF6B0C0ECE6FFB
:1077400000013AEC2FF00801C29105D0000E016E45
:1077500001017ED008012ED0036ABF51B20FE96E3D
:10776000080E0320EA6EBEC8EFFF0101C2A116D0C9
:10777000036A0801BF51B20FE96E080E0320EA6EDA
:10778000EFCFC3F8C3C8D5F8370ED66F00012BEC86
:1077900033F0200E87EC28F007D00101320E0801EB
:1077A000D46F00011FEC29F00801BF2BBF510B085B
:1077B00001E2C29146D0BE51900825E1BF6B036A39
:1077C000BF51B20FE96E080E0320EA6EBEC8EFFF8C
:1077D0000101C2A114D0036A0801BF51B20FE96EC2
:1077E000080E0320EA6EEFCFC3F8C3C8D5F8370EF2
:1077F000D66F00012BEC33F0200E87EC28F0080147
:10780000BF2BC2811ED00101C2A114D05B0E0001AA
:1078100087EC28F0BEC8D5F8370E0801D66F0001F6
:107820002BEC33F05D0E87EC28F0200E87EC28F06F
:1078300007D00101320E0801D46F00011FEC29F0BE
:107840000801320ED46F00011FEC29F0010143D76B
:107850000001000C0801D06B010167A10DD00001EF
:10786000EEDC01C0D0F80A0E0801D16F00010AEC6D
:1078700029F00801F1D701010001000C060E0801F2
:107880009B6F810E9C6F010E9D6F040E9E6F070E05
:107890009F6FA06BFF0EA16F090EA26F810EA36FE9
:1078A000010EA46F060EA56F010EA66FA76BA86B45
:1078B000030EA96FAA6FFF0EAB6FAF6B98517F0BD2
:1078C000AC6F99517F0BAD6F9A517F0BAE6F010179
:1078D000D139006E0F0E001600500B080BE10801A5
:1078E000AE53D8A402D0010105D00101CA517F0BCB
:1078F0000801AE6F0801AC5305E1010EAC6F030E39
:10790000A96F09D09851800B800803E1010EA96F7F
:1079100002D0020EA96FACC8A7F8AD5305E1010E65
:10792000AD6F030EAA6F09D09951800B800803E157
:10793000010EAA6F02D0020EAA6FADC8A8F801010D
:10794000D139006E0F0E001600500A0855E00801EC
:10795000A951030803E1AA51030839E00101DD83BD
:10796000080E0801D16FA20ED06F000136DD0101B3
:10797000D139006E0F0E00160050010807E0D13912
:10798000006E0F0E00160050050809E1030E0801F5
:10799000B16FE80EB06F000117DE16D00101D139CA
:1079A000006E0F0E0016005003080FE1D0530DE0DB
:1079B0000801B16BFA0EB06F000106DED0C1AFF85E
:1079C000AFC8D4F81FEC29F0010114D0080101015F
:1079D000DDA310D0DD93080E0801D16FA20ED06F89
:1079E0000001FBDC030E0801B16FE80EB06F00016F
:1079F000EBDD010100012EDF0801AE5302E1A06BB7
:107A00000DD09A51800B800805E1AE51070B20097B
:107A1000A06F04D0AE51070B3009A06FA05337E020
:107A2000080ED16F9B0ED06F0001D7DC0101DD8104
:107A3000D139006E0F0E00160050010807E0D13951
:107A4000006E0F0E00160050050809E1030E080134
:107A5000B16FE80EB06F0001B7DD16D00101D1396A
:107A6000006E0F0E0016005003080FE1D0530DE01A
:107A70000801B16BFA0EB06F0001A6DDD0C1AFF8FE
:107A8000AFC8D4F81FEC29F0010114D0080101019E
:107A9000DDA110D0DD91080E0801D16F9B0ED06FD3
:107AA00000019BDC030E0801B16FE80EB06F00010E
:107AB0008BDD01010001CEDE000C0801D151090867
:107AC00005E3300ED125016E05D004D0370ED12547
:107AD000016E00D00001000C080E08019B6FFF0E24
:107AE0009C6F300E9D6F9E6F9F6B600EA06F300E6F
:107AF000A16FA26FEF0EA36F070EA46FFF0EA56F0D
:107B0000300EA66FA76FA86BA20EA96F300EAA6FDA
:107B1000EF0EAB6F090EAC6FFF0EAD6F300EAE6F98
:107B2000AF6FB06B500EB16FB26BB36BB46BEF0E47
:107B3000B56F090EB66FFF0EB76F300EB86FB96F25
:107B4000BA6B510EBB6FBC6BBD6BBE6BEF0EBF6FE4
:107B5000080EC06FFF0EC16F300EC26FC36FC46BD3
:107B6000B40EC56F310EC66FC76BEF0EC86F98515C
:107B70007F0BC96F99517F0BCA6F9A517F0BCB6FE7
:107B8000CB5315E1040168513008D8A402D0080194
:107B90000ED000015FDE080E0801D16FA40ED06F79
:107BA00000011BDCAAC868F40101DD910801C9537A
:107BB0001DE1CA531BE104016651300806E167511B
:107BC0003008D8A402D0080111D0000143DE080E0D
:107BD0000801D16F9B0ED06F0001EDEC39F0A1C808
:107BE00066F4A2C867F40101DD930801C95305E1F9
:107BF000CA5303E1CB5301E134D1C95303E1300E41
:107C0000A16F09D09851800B800803E1320EA16F5B
:107C100002D0310EA16FCA5303E1300EA26F09D01A
:107C20009951800B800803E1310EA26F02D0320E11
:107C3000A26F036ACAC8D0F803C0D1F80C01E06B88
:107C40001E0EDF6F03C0E2FCCAC8E1FC00011AECA3
:107C500033F0080E08010124CC6F000E0220CD6F16
:107C6000036AC9C8D0F803C0D1F80C01E06B210E3B
:107C7000DF6F03C0E2FCC9C8E1FC00011AEC33F07D
:107C8000080E08010124CE6F000E0220CF6FCF53E3
:107C900006E1CE51090803E3CF6B0A0ECE6FCF5138
:107CA000020809E2FF0A03E1CE51200804E2030EB4
:107CB000CF6F200ECE6FCD5306E1CC51090803E300
:107CC000CD6B0A0ECC6FCD51010809E2FF0A03E12A
:107CD000CC516E0804E2020ECD6F6E0ECC6FCF5108
:107CE0000F0BD06FD16F0001E8DE01C0B2F80801C0
:107CF000CEC800F0003A0F0E001600500F0BD06FE8
:107D0000D16F0001DADE01C0B3F80801CE510F0BCC
:107D1000D06FD16F0001D1DE01C0B4F80801CD51A0
:107D20000F0BD06FD16F0001C8DE01C0BCF8080195
:107D3000CCC800F0003A0F0E001600500F0BD06FA9
:107D4000D16F0001BADE01C0BDF80801CC510F0BA4
:107D5000D06FD16F0001B1DE01C0BEF80801C95378
:107D600018E0A151300815E00101DD830801C95177
:107D70000101DE5D0DE0C9C8DEF100016BDD080E1A
:107D80000801D16FAC0ED06F0001EDEC39F00101AC
:107D90000801CA5318E0A251300815E00101DD8343
:107DA0000801CA510101DF5D0DE0CAC8DFF1000121
:107DB00051DD080E0801D16FB60ED06F0001EDEC59
:107DC00039F001010801A2510401675D05E10801D4
:107DD000A1510401665D0EE0A1C866F4A2C867F473
:107DE000000138DD080E0801D16F9B0ED06F000135
:107DF000EDEC39F00801CB5334E09A51800B800848
:107E000003E1320EAA6F02D0310EAA6F0101DD81AB
:107E10000801CB510101E05D11E0CBC8E0F10801A0
:107E2000CB51070B3009C76F000114DD080E0801A4
:107E3000D16FC00ED06F0001EDEC39F00801AA51EE
:107E40000401685D0DE0AAC868F4000103DD080EB6
:107E50000801D16FA40ED06F0001EDEC39F00401E0
:107E600008010001000C8E0E006EB9C801F0B8C800
:107E700002F0036A015209E102C001F0026A080E31
:107E8000005E015202E1006A08D0D89001BE04D021
:107E9000023601360006F9D7019E000C0801B851E0
:107EA000D8B4A5D0C46FBC51D8B4A1D0C45F05E389
:107EB0007F0EC427D8B09BD006D0810EC45FD8A057
:107EC00096D0D8B494D0C4C800F0016A026A036A9C
:107ED000C36BB9C8C2F8C28FBAC8C1F8BBC8C0F872
:107EE000190EC46FBF51C05F0DE2010EC15F0AE2FF
:107EF000C25F08E2C35F06E2C32BC22BC12BBF5196
:107F0000C02728D0BE51C15F12E2010EC25F0FE24E
:107F1000C35F0DE2C32BC22BBE51C127BF51C02787
:107F200019E3C12B17E1C22B15E1C32B13D0BD51AF
:107F30008009C25F0EE2010EC35F0BE2C32BBD518D
:107F40008009C227BE51C127E9E3C22BE7E1C32B59
:107F5000E5D70380C42F01D00BD0D890C037C137EC
:107F6000C237C337D890033602360136C537BAD781
:107F7000C5A106D0D890013202320332C53302D0F7
:107F8000000635E0C5BF1ED0D890C037C137C23714
:107F9000C337BF51C05F07E2010EC15F04E2C25F99
:107FA00002E2C35F1AE3BE51C15F05E2010EC25F88
:107FB00002E2C35F12E3BD518009C25F03E2010E1A
:107FC000C35F0BE3032A09E1022A07E1012A05E165
:107FD000002A0DE0013202320332B9C8C4F8BD51A3
:107FE000C41BC4AF02D0018E06D0019E04D0006A2B
:107FF000016A026A036A0001000C0801BC51D8B48E
:1080000071D0006EC051D8B46DD0002604E3810E4B
:10801000002668E204D07F0E005E64E363E0BDC822
:10802000C4F8C151C41BBD8FC18FBF51C303F4CF6E
:10803000C6F8BE51C203F4CF03F0F3CFC5F8C303B3
:10804000F350C627F450C523000E0322BF51C203CC
:10805000F350C627F450C523000E026A0322022201
:10806000BD51C303F350C527F4500322000E022272
:10807000BD51C203F3500326F4500222000E016AE0
:108080000122BF51C103F350C527F4500322000E53
:1080900002220122BE51C103F3500326F4500222F2
:1080A000000E0122BD51C103F3500226F4500122FB
:1080B000002A01BE05D0C537033602360136000658
:1080C000000EC5AF0AD0032A02220122015005E1A9
:1080D000025003E1035001E1002AC4BF018EC4AF86
:1080E000019E04D0006A016A026A036A0001000C62
:1080F0008E0E006E0801B851005EB9C802F0BAC811
:1081000001F0028E005209E0D890025202E10152C1
:1081100004E002320132002EF7D7B9AF05D0011EBC
:10812000021E012AD8B4022A0001000C0801CF6BFC
:10813000D06B010ED16FDA6AD96A080ED46FC70E00
:10814000D36F080EEA6ECB0EE96ED4C8E2FFD3C837
:10815000E1FFD1C8D2F8D890E550EE02F350CF231A
:10816000F450D023D22FF7D7CFC8DEFFD0C8CFF836
:10817000D06BD8B0D02BD32BD8B4D42BD12BD1519A
:108180000508DFE100014CEF41F00801CE51D219A2
:10819000800BD86FCEAF0BD0CB1FCC1FCD1FCE1F07
:1081A000CB2BD8B4CC2BD8B4CD2BD8B4CE2BD2AFCC
:1081B0000BD0CF1FD01FD11FD21FCF2BD8B4D02BA5
:1081C000D8B4D12BD8B4D22B006A016A026A036AF0
:1081D000D36BD46BD56BD66BD251D111D011CF11DB
:1081E0002CE0200ED76FD890CB37CC37CD37CE3799
:1081F000D337D437D537D637D251D65D08E1D151F0
:10820000D55D05E1D051D45D02E1CF51D35D0FE3DF
:10821000CF51D35FD051D8A0D03DD45FD151D8A099
:10822000D13DD55FD251D8A0D23DD65FD88000369F
:10823000013602360336D72FD6D7D8AF0BD0001E63
:10824000011E021E031E002AD8B4012AD8B4022A35
:10825000D8B4032A080EEA6ED30EE96E0001000CB2
:10826000010E0801BF6FC06BC16BC26BC46BC56BE5
:10827000BBBF01D01AD0010EC46FBBC8CAF8BAC8C0
:10828000C9F8B9C8C8F8B8C8C7F8FF0ECE6FCD6F27
:10829000CC6FCB6F00014AD703C0BBF802C0BAF85D
:1082A00001C0B9F800C0B8F80801BF5306E1C053D7
:1082B00004E1C15302E1C25377E0BBC8CEF8BAC8AB
:1082C000CDF8B9C8CCF8B8C8CBF8D26BD16BD06BAD
:1082D000BCC8CFF8000159DF03C0C2F802C0C1F822
:1082E00001C0C0F800C0BFF8036A0801C551BD2530
:1082F000016EBE51032201C0C7F803C0C8F8EACF1F
:10830000CAF8E9CFC9F8BBC8CEF8BAC8CDF8B9C821
:10831000CCF8B8C8CBF8D26BD16BD06BBCC8CFF857
:10832000000133DFEFCF00F0ECCF01F0ECCF02F033
:10833000ECCF03F0CAC8EAFFC9C8E9FF03C0CEF812
:1083400002C0CDF801C0CCF800C0CBF8300E080157
:108350000024006E000E0120000E0220000E0320FB
:10836000C8C8EAFFC7C8E9FF00C0EFFF036AC551EC
:10837000BD25E96EBE510320EA6EEF5039080AE2CE
:10838000036AC551BD25E96EBE510320EA6E070E92
:10839000EF24EF6EC52BC2C8BBF8C1C8BAF8C0C87D
:1083A000B9F8BFC8B8F881D7C42D0AD0036AC5513F
:1083B000BD25E96EBE510320EA6E2D0EEF6EC52B72
:1083C000C36BD890C531C35D2FE2036AC351BD258D
:1083D000E96EBE510320EA6EEFCFC6F8036AC351BF
:1083E000BD25016EBE51032203C0C8F8C351C55D4F
:1083F000FF0F036ABD25E96EBE510320EA6EEFCF81
:10840000C9F8C8C8EAFF01C0E9FFC9C8EFFFC351F6
:10841000C55DFF0F036ABD25E96EBE510320EA6EFC
:10842000C6C8EFFFC32BCDD7036AC551BD25E96E82
:10843000BE510320EA6EEF6ABDC801F0BEC802F06B
:108440000001000C08019B6B9C6B9D6B9E6B050EE5
:108450009F6F230EA06F500EA16F300EA26FA36FFF
:108460000D0EA46F050EA56F230EA66F540EA76FF9
:10847000300EA86FA96F0D0EAA6F050EAB6F230EFD
:10848000AC6F5A0EAD6F300EAE6FAF6F0D0EB06F9A
:1084900098517F0BB16FB15101084BE2B96BB1C874
:1084A000B8F80001E0DC03C09EF802C09DF801C0EE
:1084B0009CF800C09BF89EC8BBF89DC8BAF89CC841
:1084C000B9F89BC8B8F80801BF6BBE6B400EBD6F12
:1084D000830EBC6F0001E2DC00C0B8F801C0B9F83F
:1084E00002C0BAF803C0BBF803C0BFF802C0BEF8B0
:1084F00001C0BDF800C0BCF80801C36BC26B440EDC
:10850000C16F840EC06F000178DD03C09EF802C009
:108510009DF801C09CF800C09BF89EC8BBF89DC8A0
:10852000BAF89CC8B9F89BC8B8F8E2DD01C0B1F848
:10853000080199517F0BB26FB25101084BE2B96B40
:10854000B2C8B8F800018FDC03C09EF802C09DF8E5
:1085500001C09CF800C09BF89EC8BBF89DC8BAF843
:108560009CC8B9F89BC8B8F80801BF6BBE6B200E59
:10857000BD6F830EBC6F000191DC00C0B8F801C074
:10858000B9F802C0BAF803C0BBF803C0BFF802C014
:10859000BEF801C0BDF800C0BCF80801C36BC26BD7
:1085A000440EC16F840EC06F000127DD03C09EF82A
:1085B00002C09DF801C09CF800C09BF89EC8BBF8A3
:1085C0009DC8BAF89CC8B9F89BC8B8F891DD01C03D
:1085D000B2F808019A51770BB36FB351070B01083A
:1085E0004CE2B351070BB96BB86F00013CDC03C020
:1085F0009EF802C09DF801C09CF800C09BF89EC880
:10860000BBF89DC8BAF89CC8B9F89BC8B8F808016F
:10861000BF6BBE6B600EBD6F810EBC6F00013EDC98
:1086200000C0B8F801C0B9F802C0BAF803C0BBF87E
:1086300003C0BFF802C0BEF801C0BDF800C0BCF85E
:108640000801C36BC26B440EC16F840EC06F000182
:10865000D4DC03C09EF802C09DF801C09CF800C0A5
:108660009BF89EC8BBF89DC8BAF89CC8B9F89BC8CF
:10867000B8F83EDD01C0B3F80801080EEA6EB40E8A
:10868000E96ECD6BCF6B040ECE6F00013AEC2FF08C
:108690000801B15305E1350EA26F300EA36F66D00D
:1086A0009851800B800833E1320ED880B157BB6BF4
:1086B000BA6BB96BB1C8B8F80A0EBC6F080EBE6FC2
:1086C000B40EBD6F0001CCDD02C0B9F801C0B8F82E
:1086D0000801B85302E1B95313E0080ED16FB40E8C
:1086E000D06F0001D0EC29F00150010805E2B4C8B8
:1086F000A2F8B5C8A3F802D0B4C8A3F806D0080100
:10870000350EA26F300EA36F000131D00801320E7A
:10871000B127BB6BBA6BB96BB1C8B8F80A0EBC6FA6
:10872000080EBE6FB40EBD6F00019ADD02C0B9F82D
:1087300001C0B8F80801B85302E1B95313E0080EBC
:10874000D16FB40ED06F0001D0EC29F001500108B8
:1087500005E2B4C8A2F8B5C8A3F802D0B4C8A3F81B
:1087600006D00801350EA26F300EA36F0001080E6F
:108770000801D16F9F0ED06F0001EDEC39F02AECAB
:108780003CF00801B25305E1350EA86F300EA96F19
:1087900066D09951800B800832E1320EB227BB6B54
:1087A000BA6BB96BB2C8B8F80A0EBC6F080EBE6FD0
:1087B000B40EBD6F000154DD02C0B9F801C0B8F8B5
:1087C0000801B85302E1B95313E0080ED16FB40E9B
:1087D000D06F0001D0EC29F00150010805E2B4C8C7
:1087E000A8F8B5C8A9F802D0B4C8A9F806D00801FD
:1087F000350EA86F300EA96F000132D00801320E7D
:10880000D880B257BB6BBA6BB96BB2C8B8F80A0E56
:10881000BC6F080EBE6FB40EBD6F000121DD02C03B
:10882000B9F801C0B8F80801B85302E1B95313E030
:10883000080ED16FB40ED06F0001D0EC29F00150BA
:10884000010805E2B4C8A8F8B5C8A9F802D0B4C8B0
:10885000A9F806D00801350EA86F300EA96F0001E7
:10886000080E0801D16FA50ED06F0001EDEC39F0B4
:108870002AEC3CF00801B35305E1350EAE6F300E23
:10888000AF6F66D09A51800B800832E1320EB32769
:10889000BB6BBA6BB96BB3C8B8F80A0EBC6F080EE5
:1088A000BE6FB40EBD6F0001DBDC02C0B9F801C0C1
:1088B000B8F80801B85302E1B95313E0080ED16FBC
:1088C000B40ED06F0001D0EC29F00150010805E290
:1088D000B4C8AEF8B5C8AFF802D0B4C8AFF806D087
:1088E0000801350EAE6F300EAF6F000132D00801B7
:1088F000320ED880B357BB6BBA6BB96BB3C8B8F83C
:108900000A0EBC6F080EBE6FB40EBD6F0001A8DC6E
:1089100002C0B9F801C0B8F80801B85302E1B95370
:1089200013E0080ED16FB40ED06F0001D0EC29F027
:108930000150010805E2B4C8AEF8B5C8AFF802D0DE
:10894000B4C8AFF806D00801350EAE6F300EAF6F69
:108950000001080E0801D16FAB0ED06F0001EDECE5
:1089600039F02AEC3CF0000C6B50060B2AE00101B8
:10897000C2A11ED005010C6B0C510001FBEC1FF0D5
:1089800005010C2B000187EC28F0160E05010C5D8B
:10899000F3E16BCFD5F8570E0801D66F00012BEC31
:1089A00033F00A0E87EC28F00D0E87EC28F0010159
:1089B0006B6A010E0801D16F00010AEC29F0900EDC
:1089C0006B6E29EF45F04790479C479E0101D139D6
:1089D000006E0F0E00160050FF0FF20F1EE20E0F7A
:1089E00000015DEF45F00801986B996B9A6B0001EF
:1089F0003EEC3CF0010111D00801986B996B9A6B29
:108A000000016CEC3DF0010108D00801986B996BF6
:108A10009A6B000117DD010100D005010BB102D0F6
:108A20008D9601D08D8696960BB302D08D9801D08D
:108A30008D8896980BB502D08D9A01D08D8A969A22
:108A4000050E0801D46F00011FEC29F02AEC3CF060
:108A50008BD70BC50EF2036A05010B51220F016E75
:108A6000000E03220150BF0FE96E010E0320EA6ED3
:108A7000EFCFD1F10101D89005010B35036A370F13
:108A8000016E000E03220150BF0FE96E010E03209C
:108A9000EA6EECCF03F0ED52EFCFDBF1010103C042
:108AA000DCF1D26BD46BD36BD66BD56BD86BD76B39
:108AB000DA6BD96BDD6B0001000CF2CF0EF0F29E89
:108AC000E824F76AF736E50FF66E8A0EF722000EF5
:108AD000F86EFB6E0A00F550FA6E0800F5500EBEF7
:108AE000F28EF96EE689E689E689E689E689E68905
:108AF000E689E689E689E689E689F8890A8AE689C7
:108B00000601396B3A6B3B6B3C91060EEA6E2C0EFC
:108B1000E96E0801CD6BCF6B0D0ECE6F00013AEC04
:108B20002FF0010167B153D03BC6E0FC3AC6DFFC31
:108B30000C01E26B190EE16F00011AEC33F002C078
:108B40003EF601C03DF606012B51025C33E303E122
:108B50002A513D5D2FE30101C2A129D006013D6BE1
:108B60003D510001B9EC11F006013D2B000187ECED
:108B700028F0150E06013D5DF3E1100EE96E2BC6DF
:108B8000C4F82AC6C3F8000173EC3AF0180E0601C7
:108B90003D6F3D510001B9EC11F006013D2B000184
:108BA00087EC28F01F0E06013D5DF3E10101000E88
:108BB000016EA9D0190E0801D46F00011FEC29F035
:108BC00006013A2BD8B43B2B0001ABD70101C2A15F
:108BD00010D006013D6B3D510001D8EC11F00601AB
:108BE0003D2B000187EC28F00D0E06013D5DF3E101
:108BF000010167A186D0036A060139512C0F016E6D
:108C0000060E032201C03DF603C03EF600011FEC34
:108C100039F03EC6EAFF3DC6E9FF01C0EFFF0101A2
:108C2000C2A115D0036A060139512C0FE96E060E58
:108C30000320EA6EEFCF3DF63DC6D5F8370E0801AA
:108C4000D66F00012BEC33F0200E87EC28F00601E4
:108C50003CB117D0036A39512C0FE96E060E032080
:108C6000EA6EEF50FE080CE1036A39512C0FE96EF1
:108C7000060E0320EA6EEFCF2CF63C81010E396F11
:108C800035D0036A39512C0FE96E060E0320EA6EC7
:108C9000EF50EF081DE10101C2A107D00D0E000148
:108CA00087EC28F00A0E87EC28F006012F513008D7
:108CB00009E13051300806E1010E016E010123D0B7
:108CC00005D00601000E016E01011DD007D006017E
:108CD000320E0801D46F00011FEC29F00601395152
:108CE0000B0802E3392B02D0396B3C91010167B1CB
:108CF00007D0320E0801D46F00011FEC29F00101EA
:108D000078D7000E016E0001000C070E05016F6F91
:108D1000FF0E706F300E716F726F736BA50E746FF4
:108D20003C0E756FEF0E766F070E776FFF0E786F44
:108D3000300E796F7A6F7B6BB40E7C6F300E7D6F67
:108D4000EF0E7E6F060E7F6FFF0E806F300E816F0D
:108D5000826F836B630E846FEF0E856F070E866FD5
:108D6000FF0E876F300E886F896F8A6BB10E8B6F25
:108D7000300E8C6FEF0E8D6F070E8E6FFF0E8F6FA4
:108D8000300E906F916F926B900E936F300E946FC8
:108D9000EF0E956F070E966FFF0E976F300E986F60
:108DA000996F9A6BA00E9B6F310E9C6FEF0E9D6FAB
:108DB000070E9E6FFF0E9F6F300EA06FA16FA26B0C
:108DC000A00EA36F300EA46FEF0EA56F070EA66F57
:108DD000FF0EA76F300EA86FA96FAA6BA50EAB6F21
:108DE000310EAC6FEF0EAD6F070EAE6FFF0EAF6FB3
:108DF000300EB06FB16FB26BA50EB36F300EB46FA3
:108E0000EF0EB56F070EB66FFF0EB76F300EB86F6F
:108E1000B96FBA6BA70EBB6F300EBC6FEF0EBD6F94
:108E2000070EBE6FFF0EBF6F300EC06FC16FC26BFB
:108E3000A70EC36F310EC46FEF0EC56F070EC66F5E
:108E4000FF0EC76F300EC86FC96FCA6BA70ECB6F0E
:108E5000310ECC6FEF0ECD6F070ECE6FFF0ECF6FC2
:108E6000300ED06FD16FD26BA50ED36F320ED46F90
:108E7000EF0ED56F070ED66FFF0ED76F300ED86F7F
:108E8000D96FDA6BA50EDB6F320EDC6FEF0EDD6F84
:108E9000090EDE6FFF0EDF6F300EE06FE16FE26BE9
:108EA000A50EE36F3B0EE46FE56BE66BEF0EE76F2D
:108EB000080EE86FFF0EE96F300EEA6FEB6FEC6B98
:108EC000A50EED6F340EEE6F300EEF6FEF0EF06FFC
:108ED000070EF16FFF0EF26F300EF36FF46FF56B4C
:108EE000A10EF66F300EF76FEF0EF86F070EF96FE9
:108EF000FF0EFA6F300EFB6FFC6FFD6BA10EFE6F65
:108F0000310EFF6FEF0E0601006F070E016FFF0EAF
:108F1000026F300E036F046F056BA10E066F330EE8
:108F2000076FEF0E086F070E096FFF0E0A6F300E06
:108F30000B6F0C6F0D6BA10E0E6F320E0F6FEF0EDD
:108F4000106F070E116FFF0E126F300E136F146F3C
:108F5000156BA10E166F310E176FEF0E186F060E00
:108F6000196FFF0E1A6F300E1B6F1C6F1D6B570EA3
:108F70001E6FEF0E1F6F070E206FFF0E216F300E5A
:108F8000226F236F246B890E256F266BEF0E276FE0
:108F9000286B296B05016D51330A0001D8B497D0B5
:108FA000320AD8B49DD0030AD8B49BD0010AD8B4F1
:108FB00099D0070AD8B497D0010AD8B495D0030A3B
:108FC000D8B493D00E0AD8B491D0010AD8B497D0AF
:108FD000030AD8B49DD00D0AD8B4A3D00A0AD8B4D5
:108FE000A9D0030AD8B4AFD0010AD8B4B5D01F0AAB
:108FF000D8B4BBD0010AD8B4C1D0030AD8B4C7D002
:10900000010AD8B4CDD0260AD8B4D3D0010AD8B436
:10901000E1D00C0AD8B4EFD0220AD8B4EDD0030ABC
:10902000D8B4F6D00D0AD8B4F4D0010AD8B4FAD026
:10903000030AD8B411D1010AD8B414D10F0AD8B494
:1090400017D1030AD8B451D1070AD8B457D1010AAD
:10905000D8B45DD1030AD8B463D1010AD8B469D1B8
:109060003F0AD8B46FD1030AD8B46DD1070AD8B477
:1090700077D1010AD8B481D1030AD8B486D1010AC4
:10908000D8B484D10F0AD8B48ED1010AD8B494D1FF
:10909000030AD8B49FD1010AD8B4A5D1070AD8B41D
:1090A000A3D1010AD8B4A1D1030AD8B49FD1010A2F
:1090B000D8B49DD11E0AD8B4A2D1030AD8B4A8D17D
:1090C000080AD8B4A6D1010AD8B4A4D1A4D1050EF7
:1090D0000801D16F8E0ED06F0001EDEC39F09FD1F9
:1090E0009ED19DD19CD19BD19AD199D1050E0801D9
:1090F000D16F6F0ED06F0001EDEC39F090D1050EFD
:109100000801D16F770ED06F0001EDEC39F087D1F7
:10911000050E0801D16F7F0ED06F0001EDEC39F024
:109120007ED1050E0801D16F860ED06F0001EDECE7
:1091300039F075D1050E0801D16F960ED06F000180
:10914000EDEC39F06CD1050E0801D16F9E0ED06F99
:109150000001EDEC39F063D1050E0801D16FA60EC8
:10916000D06F0001EDEC39F05AD1050E0801D16F36
:10917000AE0ED06F0001EDEC39F051D1050E0801B3
:10918000D16FB60ED06F0001EDEC39F048D1050E6D
:109190000801D16FBE0ED06F0001EDEC39F03FD168
:1091A000050E0801D16FC60ED06F0001EDEC39F04D
:1091B00036D102010F510F0B30090601266F8A0EBE
:1091C000256F060E0801D16F200ED06F0001EDEC67
:1091D00039F025D102010F510F0B30090601266F1E
:1091E000890E256F060E0801D16F200ED06F000189
:1091F000EDEC39F014D113D1300E0501EF6F050EEF
:109200000801D16FE80ED06F0001EDEC39F007D105
:1092100006D1050E0801D16FD60ED06F0001EDEC1E
:1092200039F0FDD0050E0801D16FCE0ED06F0001D0
:10923000EDEC39F0640E0801D46F00011FEC29F049
:10924000300E0501EF6F050E0801D16FE80ED06FEB
:109250000001EDEC39F0E3D0020E0101DB27000E36
:10926000DC2300010101DB51D8B4DC07DB0700017E
:109270000101DC5307E1DB510F0804E3DC6B100E46
:10928000DB6F06D0DC51000803E2DC6BFF0EDB6F06
:10929000DCC129F6DBC128F6060129312B6F283104
:1092A0002A6F2B332A332B332A332B332A330F0ED7
:1092B0002B172AC6D1F800015DEC3DF001C0E5F5A1
:1092C000060128510F0B2A6F2B6BE8CFD1F8000154
:1092D0005DEC3DF001C0E6F5050E0801D16FDE0E34
:1092E000D06F0001EDEC39F09AD0050E0801D16F76
:1092F000F10ED06F0001EDEC39F091D0050E0801B0
:10930000D16FF90ED06F0001EDEC39F088D0060E68
:109310000801D16F010ED06F0001EDEC39F07FD064
:10932000060E0801D16F090ED06F0001EDEC39F087
:1093300076D0060E0801D16F110ED06F0001EDEC52
:1093400039F06DD06CD00101CA51880906012A6F2D
:109350000801986B996B9A6F00016CEC3DF05FD03F
:109360000101CA51080906012A6F0801986B996B1F
:109370009A6F00016CEC3DF052D00801986B996B2C
:109380009A6B00016CEC3DF04AD049D00101C65106
:10939000800906012A6F0801986B996F9A6B00018A
:1093A0006CEC3DF03CD00801986BC6C199F89A6B03
:1093B00000016CEC3DF033D00101C751800906017A
:1093C0002A6FE8CF98F80801996B9A6B00016CEC52
:1093D0003DF025D0C7C198F80801996B9A6B000140
:1093E0006CEC3DF01CD01BD01AD019D018D008015D
:1093F000986B996B9A6B00016CEC3DF010D0060EE7
:109400000801D16F190ED06F0001EDEC39F007D0D3
:1094100006D005D004D0000E016E0FD000D005019B
:109420006E2D09D0070E06012B6FD00E2A6F00019A
:1094300080EC45F00501010E016E0001000C0501F4
:109440000D6B1E6BFE0E1F6F206B216B010167B150
:109450003AD021C5E0FC20C5DFFC0C01E26B320EE6
:10946000E16F00011AEC33F002C023F501C022F5D0
:109470000501025006081BE2FF0A03E12251CF0852
:1094800016E20101C2A110D00501226B2251000198
:10949000E1EC0DF00501222B000187EC28F0230EF2
:1094A0000501225DF3E10101000E016E84D0320E50
:1094B0000801D46F00011FEC29F00501202BD8B45E
:1094C000212BC4D70101050EEA6E0E0EE96E0801CC
:1094D000CD6BCF6B100ECE6F00013AEC2FF0010177
:1094E000C2A110D00501226B2251000102EC0EF046
:1094F0000501222B000187EC28F0100E0501225DEA
:10950000F3E1010167A13CD005011E510F08D8B05D
:1095100002D0010135D000011FEC39F001C00DF57A
:109520000A0E0801D46F00011FEC29F00101C2A14D
:109530000DD00DC5D5F8370E0801D66F00012BEC04
:1095400033F0200E87EC28F007D00101320E08011D
:10955000D46F00011FEC29F005011F510D5D04E1DE
:109560001E6B0DC50EF50AD01E2B036A1E510E0F81
:10957000E96E050E0320EA6E0DC5EFFF0101C2D7AB
:1095800005010E51FE0813E1036A1E510E0FE96E2C
:10959000050E0320EA6EEF50EF0809E11E510508A1
:1095A00006E1010E016E010106D005D00501000E95
:1095B000016E010100D000018AEF6AF006013B6BE9
:1095C0003C6B3D6B3E6B3F913F93010167B152D0C5
:1095D0003EC6E0FC3DC6DFFC0C01E26B320EE16FE3
:1095E00000011AEC33F002C041F601C040F606015A
:1095F0002E51025C33E303E12D51405D2FE3010165
:10960000C2A129D00601406B4051000153EC11F07A
:109610000601402B000187EC28F0140E0601405D86
:10962000F3E1100EE96E2EC6C4F82DC6C3F8000192
:1096300073EC3AF0170E0601406F4051000153ECF5
:1096400011F00601402B000187EC28F01E0E0601E8
:10965000405DF3E10101000E016E2BD2320E0801D4
:10966000D46F00011FEC29F006013D2BD8B43E2B2E
:10967000ACD70101060EEA6E2F0EE96E0801CD6B24
:10968000CF6B0C0ECE6F00013AEC2FF00101C2A19E
:1096900010D00601406B4051000172EC11F0060140
:1096A000402B000187EC28F00C0E0601405DF3E131
:1096B000010167A1FED100011FEC39F001C03BF6AA
:1096C00006013FA3A1D13B3D38D10101C2A10CD07D
:1096D0003BC6D5F8370E0801D66F00012BEC33F0EE
:1096E000200E87EC28F0010106012F51880803E0C5
:1096F0002F51810810E10101C2A108D00D0E000117
:1097000087EC28F00A0E87EC28F00101010E016EAB
:10971000D0D111D106013051510804E03051520826
:10972000D8A48BD00101C2A107D00D0E000187EC97
:1097300028F00A0E87EC28F006013FA106D0010EA2
:10974000016E0101B6D177D006010101C2A110D08E
:109750000601406B4051000172EC11F00601402BF4
:10976000000187EC28F00C0E0601405DF3E10101D9
:10977000060EEA6E2F0EE96E0801CD6BCF6B0C0E54
:10978000CE6F00013AEC2FF006013F93010167B163
:1097900052D03EC6E0FC3DC6DFFC0C01E26B320E4F
:1097A000E16F00011AEC33F002C041F601C040F64F
:1097B00006012E51025C33E303E12D51405D2FE39E
:1097C0000101C2A129D00601406B4051000188EC83
:1097D00011F00601402B000187EC28F0090E06016C
:1097E000405DF3E1100EE96E2EC6C4F82DC6C3F835
:1097F000000173EC3AF00C0E0601406F405100017D
:1098000088EC11F00601402B000187EC28F0130EC4
:109810000601405DF3E10101000E016E4AD1320EF6
:109820000801D46F00011FEC29F006013D2BD8B4CC
:109830003E2BACD701017FD006013051410804E036
:1098400030514208D8A476D03F810101C2A110D086
:109850000601406B4051000172EC11F00601402BF3
:10986000000187EC28F00C0E0601405DF3E10101D8
:10987000060EEA6E2F0EE96E0801CD6BCF6B0C0E53
:10988000CE6F00013AEC2FF006013F93010167B162
:1098900052D03EC6E0FC3DC6DFFC0C01E26B320E4E
:1098A000E16F00011AEC33F002C041F601C040F64E
:1098B00006012E51025C33E303E12D51405D2FE39D
:1098C0000101C2A129D00601406B4051000188EC82
:1098D00011F00601402B000187EC28F0090E06016B
:1098E000405DF3E1100EE96E2EC6C4F82DC6C3F834
:1098F000000173EC3AF00C0E0601406F405100017C
:1099000088EC11F00601402B000187EC28F0130EC3
:109910000601405DF3E10101000E016ECAD0320E76
:109920000801D46F00011FEC29F006013D2BD8B4CB
:109930003E2BACD7010166D00601036A3C512F0FC4
:10994000E96E060E0320EA6E3BC6EFFF0101C2A1DD
:1099500017D0036A06013C512F0FE96E060E032053
:10996000EA6EEFCF40F640C6D5F8370E0801D66F45
:1099700000012BEC33F0200E87EC28F007D001011A
:10998000320E0801D46F00011FEC29F006013C2BB8
:109990003C510B0802E23F9334D02F51900831E143
:1099A0003C5102082EE13051410A00010FE0030A48
:1099B0000DE0120A0BE0010A09E0030A07E0320A8F
:1099C00005E0010A03E0030A01E001D019D0060115
:1099D0003F930101C2A10FD00601406B405100012D
:1099E000A1EC11F00601402B000187EC28F0100ECD
:1099F0000601405DF3E106013E6B3D6B000100D0C6
:109A0000060101014ED006013B51900806E03B5192
:109A1000810803E03B51880826E13C6B036A3C5116
:109A20002F0FE96E060E0320EA6E3BC6EFFF010121
:109A3000C2A115D0036A06013C512F0FE96E060E34
:109A40000320EA6EEFCF40F640C6D5F8370E080186
:109A5000D66F00012BEC33F0200E87EC28F00601C6
:109A60003C2B3F831ED00101C2A114D05B0E00012C
:109A700087EC28F03BC6D5F8370E0801D66F0001F9
:109A80002BEC33F05D0E87EC28F0200E87EC28F0ED
:109A900007D00101320E0801D46F00011FEC29F03C
:109AA0000601320E0801D46F00011FEC29F00101FC
:109AB00000D60001000C050E05016F6F810E706F5E
:109AC000090E716F726B020E736FFF0E746F050ECD
:109AD000756F810E766F090E776F040E786F4E0EDC
:109AE000796FFF0E7A6F050E7B6F810E7C6F090E0A
:109AF0007D6F040E7E6F470E7F6FFF0E806F050E29
:109B0000816F810E826F090E836F060E846F120EB5
:109B1000856FFF0E866F050E876F810E886F090EA9
:109B2000896F040E8A6F480E8B6FFF0E8C6F090EC3
:109B30008D6F810E8E6F010E8F6F040E906F4E0E23
:109B4000916F926B936B946B956BFF0E966F060EF5
:109B5000976FFF0E986F880E996F010E9A6F9B6B2F
:109B60009C6FFF0E9D6F060E9E6F810E9F6F010E04
:109B7000A06F060EA16FA26F020EA36FFF0EA46F5F
:109B8000060EA56F810EA66F010EA76F060EA86FB9
:109B9000A96F030EAA6FFF0EAB6F060EAC6F810E9E
:109BA000AD6F010EAE6F040EAF6FB06B020EB16FF2
:109BB000FF0EB26F060EB36F810EB46F010EB56F5C
:109BC000040EB66FB76B030EB86FFF0EB96F060EBB
:109BD000BA6F810EBB6F010EBC6F040EBD6F330EEA
:109BE000BE6F020EBF6FFF0EC06F060EC16F810EFB
:109BF000C26F010EC36F040EC46F330EC56F030E28
:109C0000C66FFF0EC76F060EC86F810EC96F010EBB
:109C1000CA6F040ECB6F350ECC6FCD6BFF0ECE6FBF
:109C2000060ECF6F810ED06F010ED16F040ED26F72
:109C3000350ED36F030ED46FFF0ED56F060ED66FA1
:109C4000810ED76F010ED86F040ED96F3E0EDA6FFA
:109C5000020EDB6FFF0EDC6F060EDD6F810EDE6F16
:109C6000010EDF6F040EE06F3E0EE16F030EE26F38
:109C7000FF0EE36F060EE46F810EE56F010EE66FD7
:109C8000040EE76F380EE86F020EE96FFF0EEA6F01
:109C9000060EEB6F810EEC6F010EED6F040EEE6F92
:109CA000380EEF6F030EF06FFF0EF16F060EF26FBE
:109CB000810EF36F010EF46F040EF56F080EF66F50
:109CC000210EF76FFF0EF86F060EF96F810EFA6F17
:109CD000010EFB6F040EFC6F080EFD6F310EFE6F60
:109CE000FF0EFF6F060E0601006F810E016F010E61
:109CF000026F040E036F080E046F056BFF0E066FF4
:109D0000050E076F810E086F010E096F060E0A6FB0
:109D1000040E0B6FFF0E0C6F050E0D6F810E0E6F94
:109D2000010E0F6F060E106F050E116FFF0E126FF2
:109D3000070E136F810E146F010E156F040E166F50
:109D40003F0E176F010E186F196BFF0E1A6F050E7D
:109D50001B6F810E1C6F010E1D6F040E1E6F480ECF
:109D60001F6FFF0E206F050E216F890E226F010EEF
:109D7000236F246F030E256FFF0E266F050E276FCE
:109D8000810E286F090E296F070E2A6F220E2B6F86
:109D9000FF0E2C6F05016D51010A0001D8B4A3D04C
:109DA000030AD8B4A1D0010AD8B4A7D0070AD8B4FE
:109DB000A5D0010AD8B4A3D0030AD8B4A1D00E0A02
:109DC000D8B49FD0010AD8B4A5D0030AD8B4ABD078
:109DD0000D0AD8B4B1D00C0AD8B4B7D0070AD8B499
:109DE000BDD00C0AD8B4C3D00D0AD8B4C9D0030A68
:109DF000D8B4CFD0010AD8B4D5D01F0AD8B4DBD09C
:109E0000010AD8B4E1D0020AD8B4E7D0070AD8B41E
:109E1000F8D0010AD8B4FED0030AD8B404D1010A9C
:109E2000D8B407D10F0AD8B40AD1030AD8B437D1AD
:109E3000070AD8B43DD1010AD8B443D1030AD8B433
:109E400058D1010AD8B46DD13F0AD8B472D1190AD9
:109E5000D8B470D10C0AD8B476D1010AD8B484D160
:109E6000030AD8B492D1010AD8B4A0D10E0AD8B44A
:109E7000AED1020AD8B4ACD1010AD8B4ADD1180A17
:109E8000D8B4AED1070AD8B4B8D1010AD8B4C2D177
:109E9000030AD8B4C7D1010AD8B4CDD10F0AD8B4B7
:109EA000D7D1010AD8B4DDD1030AD8B4E8D1010A68
:109EB000D8B4EED1070AD8B4FFD1010AD8B40BD276
:109EC000030AD8B417D2010AD8B41ED21F0AD8B4D4
:109ED00023D2010AD8B429D2030AD8B42FD20E0A49
:109EE000D8B435D23DD240D2050E0801D16F6F0EE5
:109EF000D06F0001EDEC39F037D236D235D234D202
:109F000033D2050E0801D16F750ED06F0001EDEC54
:109F100039F02AD2050E0801D16F7B0ED06F0001F7
:109F2000EDEC39F021D2050E0801D16F810ED06F12
:109F30000001EDEC39F018D2050E0801D16F870E43
:109F4000D06F0001EDEC39F00FD2050E0801D16F92
:109F50009E0ED06F0001EDEC39F006D2050E08011F
:109F6000D16FA50ED06F0001EDEC39F0FDD1050EDB
:109F70000801D16F970ED06F0001EDEC39F0F4D1EC
:109F8000050E0801D16FAC0ED06F0001EDEC39F079
:109F9000EBD1050E0801D16FB30ED06F0001EDECCF
:109FA00039F0E2D1050E0801D16FBA0ED06F000171
:109FB000EDEC39F0D9D1050E0801D16FC10ED06F8B
:109FC0000001EDEC39F0D0D1050E0801D16FC80EBB
:109FD000D06F0001EDEC39F0C7D10101D139006E2D
:109FE0000F0E001600500B0803E1050E0501D46F9B
:109FF000050E0801D16FCF0ED06F0001EDEC39F0E6
:10A00000B3D1050E0801D16FD60ED06F0001EDEC73
:10A0100039F0AAD1050E0801D16FDD0ED06F000115
:10A02000EDEC39F0A1D1020E0101DB27000EDC239B
:10A0300000010101DB51D8B4DC07DB07000101019D
:10A04000DC5307E1DB51010804E3DC6B010EDB6F3D
:10A0500008D0DC5303E1DB510D0803E2DC6B0E0E8C
:10A06000DB6FDC31036EDB31026E0332023203320E
:10A070000232033202320F0E031602C094F50501BC
:10A080000101DB510F0BE8CF95F50501050E080125
:10A09000D16F8D0ED06F0001EDEC39F065D1050E5A
:10A0A0000801D16FE40ED06F0001EDEC39F05CD106
:10A0B000050E0801D16FEB0ED06F0001EDEC39F009
:10A0C00053D10101D139006E0F0E00160050060861
:10A0D00004E1020E0501F76F03D0200E0501F76FB2
:10A0E000050E0801D16FF20ED06F0001EDEC39F0D2
:10A0F0003BD10101D139006E0F0E00160050060849
:10A1000004E1030E0501FE6F03D0300E0501FE6F62
:10A11000050E0801D16FF90ED06F0001EDEC39F09A
:10A1200023D1060E0801D16FD06B0001EDEC39F0A0
:10A130001BD11AD1060E0801D16F210ED06F00017C
:10A14000EDEC39F011D1010E02010F5D0F0B06018C
:10A15000196F020E186F060E0801D16F130ED06F23
:10A160000001EDEC39F000D1010E02010F5D0F0B83
:10A170000601196F010E186F060E0801D16F130E3C
:10A18000D06F0001EDEC39F0EFD0010E02010F5D50
:10A190000F0B0601196F040E186F060E0801D16F20
:10A1A000130ED06F0001EDEC39F0DED0010E02018C
:10A1B0000F5D0F0B0601196F030E186F060E0801D5
:10A1C000D16F130ED06F0001EDEC39F0CDD0CCD0B3
:10A1D000010E016ED7D0C8D0010E016ED3D0C4D00D
:10A1E0000101CA51880906012D6F0801986B996B0E
:10A1F0009A6F00013EEC3CF0B7D00101CA5108094A
:10A2000006012D6F0801986B996B9A6F00013EEC67
:10A210003CF0AAD00801986B996B9A6B00013EEC58
:10A220003CF0A2D00801986B996BCAC19AF8000162
:10A230003EEC3CF099D00101C651800906012D6F1A
:10A240000801986B996F9A6B00013EEC3CF08CD042
:10A250000801986BC6C199F89A6B00013EEC3CF07E
:10A2600083D00101C751800906012D6FE8CF98F80E
:10A270000801996B9A6B00013EEC3CF075D0C7C1A8
:10A2800098F80801996B9A6B00013EEC3CF06CD099
:10A290000101C751800906012D6F0101C6518009D6
:10A2A00006012E6F2DC698F8E8CF99F808019A6B31
:10A2B00000013EEC3CF058D00101C6518009060176
:10A2C0002D6FC7C198F8E8CF99F808019A6B000183
:10A2D0003EEC3CF049D00101C751800906012D6FC9
:10A2E000E8CF98F8C6C199F808019A6B00013EECD6
:10A2F0003CF03AD0C7C198F8C6C199F808019A6BEA
:10A3000000013EEC3CF030D00801986B996B9A6BE1
:10A3100000013EEC3CF028D0060E0801D16F1B0E68
:10A32000D06F0001EDEC39F01FD0060E0801D16F9F
:10A33000070ED06F0001EDEC39F016D0060E0801C3
:10A34000D16F0D0ED06F0001EDEC39F00DD0060E7F
:10A350000801D16F270ED06F0001EDEC39F004D069
:10A36000000E016E0FD000D005016E2D09D0070E32
:10A3700006012E6FD00E2D6F0001DEEC4AF00501B4
:10A38000010E016E0001000C0501E76BE86BE96B43
:10A39000020EEA6F030EEB6FEC91D92D04D0230E61
:10A3A000EA6F0D0EEB6F050EEA6EDA0EE96E08012C
:10A3B000CD6BCF6B0D0ECE6F00013AEC2FF001018B
:10A3C00067B153D0E9C5E0FCE8C5DFFC0C01E26BE6
:10A3D000190EE16F00011AEC33F002C0EEF501C076
:10A3E000EDF50501D851025C33E303E1D751ED5D92
:10A3F0002FE30101C2A129D00501ED6BED51000150
:10A40000FDEC12F00501ED2B000187EC28F0190E90
:10A410000501ED5DF3E1100EE96ED8C5C4F8D7C5AE
:10A42000C3F8000173EC3AF01C0E0501ED6FED511D
:10A430000001FDEC12F00501ED2B000187EC28F086
:10A44000230E0501ED5DF3E10101000E016ECFD099
:10A45000190E0801D46F00011FEC29F00501E82B4B
:10A46000D8B4E92B0001ABD70101C2A110D005017E
:10A47000ED6BED5100011EEC13F00501ED2B000119
:10A4800087EC28F0110E0501ED5DF3E1010167A1F4
:10A49000ACD0036A0501E751DA0F016E050E032205
:10A4A00001C0EDF503C0EEF500011FEC39F0EEC57B
:10A4B000EAFFEDC5E9FF01C0EFFF0101C2A131D004
:10A4C000036A0501E751DA0FE96E050E0320EA6E13
:10A4D000EF501F0812E2036AE751DA0FE96E050E2A
:10A4E0000320EA6EEFCFEDF5ED51000187EC28F087
:10A4F000200E87EC28F015D00501036AE751DA0F2A
:10A50000E96E050E0320EA6EEFCFEDF5EDC5D5F847
:10A51000370E0801D66F00012BEC33F0200E87ECCC
:10A5200028F00501D95340E1ECB117D0036AE75197
:10A53000DA0FE96E050E0320EA6EEF5002080CE117
:10A54000036AE751DA0FE96E050E0320EA6EEFCFDA
:10A55000DAF5EC81010EE76F26D0036AE751DA0FD6
:10A56000E96E050E0320EA6EEF5003081CE10101BD
:10A57000C2A107D00D0E000187EC28F00A0E87EC6F
:10A5800028F00501DB51450809E0DB51650806E0CC
:10A59000010E016E01012BD005D00501FF0E016EE9
:10A5A000010125D005010FD0036AE751DA0FE96EEA
:10A5B000050E0320EA6EEF500D0805E1010E016E55
:10A5C000010115D00501E7510B0802E3E72B02D08A
:10A5D000E76BEC91010167B107D0320E0801D46F2F
:10A5E00000011FEC29F0010152D7000E016E00019D
:10A5F000000C05017491040E756F230E766F4F0EDB
:10A60000776F310E786F0D0E796F0C0E7A6F230E07
:10A610007B6F550E7C6F380E7D6F300E7E6F7F6FB7
:10A62000806F380E816F300E826F836F846F080EDB
:10A63000856F0D0E866F080E876F230E886F410E93
:10A64000896F580E8A6F5A0E8B6F380E8C6F300ED2
:10A650008D6F8E6F0D0E8F6F050E906F230E916FA5
:10A66000520E926F936B946B0D0E956F050E966F55
:10A67000020E976F510E986F520E996F530E9A6F8C
:10A68000030E9B6F070E9C6F020E9D6F4F0E9E6F09
:10A69000520E9F6F530EA06F3A0EA16F310EA26F34
:10A6A000030EA36F050EA46F020EA56F510EA66FC9
:10A6B000520EA76F560EA86F030EA96F090EAA6F50
:10A6C000020EAB6F4F0EAC6F520EAD6F560EAE6FEB
:10A6D0003A0EAF6F300EB06FB16FB26F030EB36F43
:10A6E000050EB46F020EB56F510EB66F410EB76F07
:10A6F000460EB86F030EB96F070EBA6F020EBB6F2E
:10A700004F0EBC6F410EBD6F460EBE6F3A0EBF6F4F
:10A71000310EC06F030EC16F050EC26F230EC36FE3
:10A72000460EC46FC56BC66B0D0EC76F040EC86FA7
:10A73000230EC96F470ECA6F460ECB6F0D0ECC6F3E
:10A74000080ECD6F230ECE6F410ECF6F580ED06F17
:10A75000460ED16FD26BD36BD46B0D0ED56F6D518E
:10A76000010A0001D8B4A0D0030AD8B4A1D0010ACC
:10A77000D8B4A2D0070AD8B4A3D0010AD8B4A1D0C3
:10A78000030AD8B4A7D00E0AD8B4ADD0010AD8B401
:10A79000B3D0030AD8B4B1D0350AD8B4AFD07F0A49
:10A7A000D8B4ADD0470AD8B4ABD0070AD8B4B1D02A
:10A7B0000D0AD8B4AFD0030AD8B4B8D0010AD8B4BF
:10A7C000C1D01F0AD8B4BED0010AD8B4BCD0020A86
:10A7D000D8B4B9D0070AD8B4B7D0010AD8B4C0D019
:10A7E000030AD8B4C9D0010AD8B40FD10F0AD8B41B
:10A7F00016D1030AD8B450D1070AD8B459D1010AE6
:10A80000D8B462D1030AD8B470D1010AD8B47ED1C9
:10A810003F0AD8B48CD1190AD8B4C6D10C0AD8B41E
:10A82000C4D1010AD8B400D20C0AD8B4FDD1020AAE
:10A83000D8B439D2010AD8B437D2180AD8B435D22C
:10A84000070AD8B433D2010AD8B431D2030AD8B433
:10A850002FD2010AD8B42DD20F0AD8B42BD2010AB4
:10A86000D8B429D2030AD8B427D2010AD8B425D241
:10A87000070AD8B423D2010AD8B421D2030AD8B423
:10A880001FD2010AD8B41DD21F0AD8B41BD20E0A97
:10A89000D8B419D20F0AD8B424D2030AD8B42FD20C
:10A8A0000F0AD8B42DD22DD2010E016E41D22DD275
:10A8B000010E016E3DD229D2010E016E39D225D290
:10A8C00024D2050E0801D16F960ED06F0001EDEC79
:10A8D00039F01BD2050E0801D16FB40ED06F000104
:10A8E000EDEC39F012D2050E0801D16FA40ED06F35
:10A8F0000001EDEC39F009D208D207D206D205D218
:10A90000050E0801D16FC80ED06F0001EDEC39F0D3
:10A91000FCD1FBD1310E0501786F050E0801D16F16
:10A92000750ED06F0001EDEC39F0EFD1300E05015E
:10A93000786F050E0801D16F750ED06F0001EDEC38
:10A9400039F0E3D1E2D1E1D1300E0501A26F050E5D
:10A950000801D16F9C0ED06F0001EDEC39F0D5D11C
:10A96000310E0501A26F050E0801D16F9C0ED06F4C
:10A970000001EDEC39F0C9D10101DC51030808E315
:10A9800003E1DB51FE0804E3080EDB27000EDC23A5
:10A990000501D66B0101DC510F0B0501D76FD66F96
:10A9A000D76BE8CFD1F800015DEC3DF001C0B0F508
:10A9B0000101DB51F00B0501D66FD76BD733D633CE
:10A9C000D733D633D733D633D733D6330F0ED71743
:10A9D000D6C5D1F800015DEC3DF001C0B1F5010133
:10A9E000DB510F0B0501D66FD76BE8CFD1F8000113
:10A9F0005DEC3DF001C0B2F5050E0801D16FAA0E65
:10AA0000D06F0001EDEC39F080D10101DB5302E1A0
:10AA1000DC5304E0080EDB5F000EDC5B0001050187
:10AA2000D66B0101DC510F0B0501D76FD66FD76BC9
:10AA3000E8CFD1F800015DEC3DF001C0B0F50101B7
:10AA4000DB51F00B0501D66FD76BD733D633D73335
:10AA5000D633D733D633D733D6330F0ED717D6C521
:10AA6000D1F800015DEC3DF001C0B1F50101DB5111
:10AA70000F0B0501D66FD76BE8CFD1F800015DEC65
:10AA80003DF001C0B2F5050E0801D16FAA0ED06FDE
:10AA90000001EDEC39F039D1310E0501C06F050E22
:10AAA0000801D16FBA0ED06F0001EDEC39F02DD155
:10AAB000300E0501C06F050E0801D16FBA0ED06FC0
:10AAC0000001EDEC39F021D1380E0501C56F300ED3
:10AAD000C66F050E0801D16FC20ED06F0001EDECFC
:10AAE00039F005016E6B000110D1320E0501C56F02
:10AAF000300EC66F050E0801D16FC20ED06F000177
:10AB0000EDEC39F005016E6B0001FFD0350E05014B
:10AB1000C56F300EC66F050E0801D16FC20ED06F23
:10AB20000001EDEC39F005016E6B0001EED005017E
:10AB3000D66B0101DA510F0B0501D76FD66FD76BBA
:10AB4000E8CFD1F800015DEC3DF001C0D2F5010184
:10AB5000D951F00B0501D66FD76BD733D633D73326
:10AB6000D633D733D633D733D6330F0ED717D6C510
:10AB7000D1F800015DEC3DF001C0D3F50101D951E0
:10AB80000F0B0501D66FD76BE8CFD1F800015DEC54
:10AB90003DF001C0D4F5050E0801D16FCD0ED06F88
:10ABA0000001EDEC39F0B1D0B0D0520E0501926F3A
:10ABB000050EEA6E6F0EE96E0801CD6BCF6B050EC8
:10ABC000CE6F00013AEC2FF00801BB6BBA6BB96B8A
:10ABD0000FC2B8F80A0EBC6F050EBE6F6F0EBD6FC8
:10ABE000000130EC41F0015002101DE0050E08019B
:10ABF000D16F6F0ED06F0001D0EC29F00150010829
:10AC000005E26FC593F570C594F505D0300E0501CA
:10AC1000936F6FC594F5050E0801D16F900ED06F3C
:10AC20000001EDEC39F071D04D0E0501926F050E6B
:10AC3000EA6E6F0EE96E0801CD6BCF6B050ECE6F1D
:10AC400000013AEC2FF00801BB6BBA6BB96B0FC275
:10AC5000B8F80A0EBC6F050EBE6F6F0EBD6F000117
:10AC600030EC41F0015002101DE0050E0801D16FDB
:10AC70006F0ED06F0001D0EC29F00150010805E201
:10AC80006FC593F570C594F505D0300E0501936F2F
:10AC90006FC594F5050E0801D16F900ED06F0001BD
:10ACA000EDEC39F032D031D030D02FD02ED02DD0A5
:10ACB0002CD02BD02AD029D028D027D026D025D0D0
:10ACC00024D023D022D00501748100012AEC3CF06D
:10ACD000050E0801D16F870ED06F0001EDEC39F041
:10ACE00014D00501748100012AEC3CF0050E080126
:10ACF000D16F7A0ED06F0001EDEC39F006D005D09F
:10AD000004D0000E016E14D000D005016E2D0ED0BF
:10AD1000000E74B1010ED66F070ED86FD00ED76F2C
:10AD2000D6C5D9F50001C4EC51F00501010E016E44
:10AD30000001000C0501276B286B296B2A9122C5A5
:10AD4000EAFF21C5E9FF0801CD6BCF6B23C5CEF823
:10AD500000013AEC2FF0010167B153D029C5E0FCA6
:10AD600028C5DFFC0C01E26B190EE16F00011AEC43
:10AD700033F002C02CF501C02BF505012551025C12
:10AD800033E303E124512B5D2FE30101C2A129D05C
:10AD900005012B6B2B51000136EC13F005012B2B19
:10ADA000000187EC28F01D0E05012B5DF3E1100E6C
:10ADB000E96E25C5C4F824C5C3F8000173EC3AF068
:10ADC000200E05012B6F2B51000136EC13F005010D
:10ADD0002B2B000187EC28F0270E05012B5DF3E1FA
:10ADE0000101000E016EE4D0190E0801D46F0001BC
:10ADF0001FEC29F00501282BD8B4292B0001ABD773
:10AE00000101C2A110D005012B6B2B51000159EC9F
:10AE100013F005012B2B000187EC28F0150E05011E
:10AE20002B5DF3E1010167A1C1D0036A0501275140
:10AE30002125016E2251032201C02BF503C02CF500
:10AE400000011FEC39F02CC5EAFF2BC5E9FF01C05A
:10AE5000EFFF0101C2A131D0036A0501275121256D
:10AE6000E96E22510320EA6EEF501F0812E2036AD6
:10AE700027512125E96E22510320EA6EEFCF2BF5F1
:10AE80002B51000187EC28F0200E87EC28F015D01C
:10AE90000501036A27512125E96E22510320EA6E3C
:10AEA000EFCF2BF52BC5D5F8370E0801D66F000173
:10AEB0002BEC33F0200E87EC28F00501265354E1EB
:10AEC0002AB11FD0036A27512125E96E22510320A0
:10AED000EA6EEF50020814E122C503F0036A27511D
:10AEE0002125E96E22510320EA6EEFCF2DF522C510
:10AEF000EAFF21C5E9FF2DC5EFFF2A81010E276F6B
:10AF000032D0036A27512125E96E22510320EA6ECF
:10AF1000EF50030828E10101C2A107D00D0E000186
:10AF200087EC28F00A0E87EC28F0010E0501212598
:10AF3000E96E000E2221EA6EEF5045080FE0010E87
:10AF40002125E96E000E2221EA6EEF50650806E029
:10AF5000010E016E01012CD005D00501FF0E016E1E
:10AF6000010126D005010FD0036A27512125E96E82
:10AF700022510320EA6EEF500D0805E1010E016E2B
:10AF8000010116D00501010E235D275D02E2272B8A
:10AF900002D0276B2A91010167B107D0320E080158
:10AFA000D46F00011FEC29F001013DD7000E016EA6
:10AFB0000001000C0801A66BA76BA86BA96BAA6B1C
:10AFC000A55303E0A551060828E2AB6BAB51000185
:10AFD0007BEC08F00801AB2B000187EC28F0190E80
:10AFE0000801AB5DF3E1A5C8ABF81F0EAC6F000123
:10AFF0006BEC39F01B0E0801AB6FAB5100017BEC21
:10B0000008F00801AB2B000187EC28F0210E0801A5
:10B01000AB5DF3E1000E016ECDD0A5C84DF2A96B7A
:10B02000010EA86FA953D8A4B9D0A8510C08D8A074
:10B03000B5D0A76B900EA66F010EA55D036AAB6F2E
:10B0400003C0ACF8A7C8E0FCA6C8DFFC03C0E2FC64
:10B05000E8CFE1FC00011AEC33F002C0A7F801C010
:10B06000A6F8200E0801A627000EA723010EA85D52
:10B07000AB6F000EA959AC6FE8CFE0FCABC8DFFCAA
:10B080000C01E26B0C0EE16F00011AEC33F0015081
:10B090000801A6270250A7230101C2A141D008013F
:10B0A000A82D3DD0A9533BE1AB6BAB5100019BEC0C
:10B0B00008F00801AB2B000187EC28F0050E080111
:10B0C000AB5DF3E1A5C8ABF81F0EAC6F00016BECF4
:10B0D00039F0070E0801AB6FAB5100019BEC08F093
:10B0E0000801AB2B000187EC28F0170E0801AB5DBF
:10B0F000F3E1A7C8D5F8370ED66F00012BEC33F07B
:10B10000A6C8D5F8370E0801D66F00012BEC33F036
:10B110000A0E87EC28F00D0E87EC28F008010101DB
:10B12000F2CFABF8F29EA7C8AAFFA6C8A9FFA69CBB
:10B13000A69EA680A8500801ABBFF28EAA6FAA51A6
:10B14000F00B09E04D0EA825E96E020EA921EA6E6A
:10B15000FF0EEF6E07D04D0EA825E96E020EA92155
:10B16000EA6EEF6A0101C2A114D04D0E0801A825B4
:10B17000E96E020EA921EA6EEFCFABF8ABC8D5F8A5
:10B18000570ED66F00012BEC33F0200E87EC28F021
:10B1900001010801A82BD8B4A92B44D70101C2A1F1
:10B1A00008D00A0E000187EC28F00D0E87EC28F07D
:10B1B000010108010001000C0101D13905016C6F8A
:10B1C0000F0E6C17010E6C5DF20F1DE20E0F0001E9
:10B1D00005EF59F06AC56DF56BC56EF55BEC4DF08A
:10B1E000050111D06AC56DF56BC56EF585EC46F0AD
:10B1F000050109D06AC56DF56BC56EF5F9EC52F025
:10B20000050101D005010001000CF2CF0EF0F29E05
:10B21000E824F76AF736350FF66EB20EF722000E05
:10B22000F86EFB6E0A00F550FA6E0800F5500EBE7F
:10B23000F28EF96ED4B1D4B1D4B1D4B1D4B1D4B109
:10B24000D4B1D4B1D4B1D4B1D4B1E4B1F4B1D4B1A6
:10B250000F0E0501226F810E236F010E246F060E63
:10B26000256F020E266F276B286B296B2A6B2B6BC1
:10B270002C6B2D6B2E6B2F6B306BFF0E316F326F83
:10B28000090E336F810E346F010E356F040E366F69
:10B29000470E376F386B396B3A6B3B6BFF0E3C6F69
:10B2A000090E3D6F810E3E6F010E3F6F040E406F21
:10B2B000480E416F426B436B446B456BFF0E466F0C
:10B2C000090E476F810E486F010E496F040E4A6FD9
:10B2D0004E0E4B6F4C6B4D6B4E6B4F6BFF0E506FAA
:10B2E000070E516F0101D139006E0F0E001600508C
:10B2F0000A08D8B4CCD0C7C127F5C6C128F5D139C2
:10B30000006E0F0E0016005008080EE0D139006ED6
:10B310000F0E00160050070807E0D139006E0F0E1F
:10B3200000160050090811E10501222B036A515152
:10B33000220FE96E050E0320EA6E0101D2510F0BB8
:10B34000EF6E0501512B286B0101036A0501515174
:10B35000220FE96E050E0320EA6E0101D4390501C2
:10B36000546F0F0E541754510F0BEF6E010E5125F1
:10B37000036A220FE96E050E0320EA6ED4C154F56C
:10B3800054510F0BEF6E020E5125036A220FE96E26
:10B39000050E0320EA6E0101D4310501556F01014C
:10B3A000D3310501546F553354335533543355332A
:10B3B00054330F0E551754510F0BEF6E030E5125DA
:10B3C000036A220FE96E050E0320EA6E0101D351D4
:10B3D0000F0BEF6E040E05015125036A220FE96E73
:10B3E000050E0320EA6E0101D6390501546F0F0ED8
:10B3F000541754510F0BEF6E050E5125036A220F9F
:10B40000E96E050E0320EA6ED6C154F554510F0BB8
:10B41000EF6E060E5125036A220FE96E050E03201A
:10B42000EA6E0101D6310501556F0101D5310501E3
:10B43000546F5533543355335433553354330F0EFF
:10B44000551754510F0BEF6E070E5125036A220F4B
:10B45000E96E050E0320EA6E0101D5510F0BEF6E68
:10B46000050E0801D16F220ED06F0001EDEC39F00E
:10B470004E0E06012E6F200E2D6F0001DEEC4AF0FD
:10B48000012C01D003D0000E016E4AD10101D13947
:10B49000006E0F0E00160050050805E1010E016E4A
:10B4A00000013ED10101D8390501526F0F0E52172C
:10B4B00052510F0B386FD8C152F552510F0B396FE3
:10B4C0000101D8310501536F0101D7310501526FD8
:10B4D0005333523353335233533352330F0E5317C4
:10B4E00052510F0B3A6F0101D7510F0BE8CF3BF5CB
:10B4F0000501050E0801D16F330ED06F0001EDEC90
:10B5000039F0070E06012E6FD00E2D6F0001DEEC14
:10B510004AF0012C01D003D0000E016E01D10101CF
:10B52000D1A709D01B0E05016A6F010E6B6F0001D8
:10B5300043DE59D001011C0E05016A6F010E6B6FCD
:10B5400000013ADE0101D139006E0F0E00160050E5
:10B550000B080DE1020130B908D0370E05016A6F02
:10B56000010E6B6F000128DE02013ED00101DA39C5
:10B570000501526F0F0E521752510F0B426FDAC175
:10B5800052F552510F0B436F0101DA310501536F30
:10B590000101D9310501526F5333523353335233C2
:10B5A000533352330F0E531752510F0B446F010197
:10B5B000D9510F0BE8CF45F50501050E0801D16FF4
:10B5C0003D0ED06F0001EDEC39F0030E06012E6F39
:10B5D000E80E2D6F0001DEEC4AF0012C01D003D003
:10B5E000000E016E9DD002010101D1A541D0140EC3
:10B5F00005016A6F010E6B6F0001DEDD0101DC6B7E
:10B60000070EDB6FD89002010E35036A370F016E0B
:10B61000000E03220150BF0FE96E010E0320EA6EF7
:10B62000DCC1ECFFED52DBC1EFFF05014C6B4D6B54
:10B630004E6B0101DB510F0BE8CF4FF50501050EF5
:10B640000801D16F470ED06F0001EDEC39F0030E09
:10B6500006012E6FE80E2D6F0001DEEC4AF0150E8C
:10B6600005016A6F010E6B6F0001A6DD45D0010177
:10B67000140E05016A6F010E6B6F00019DDD010163
:10B68000DC390501526F0F0E521752510F0B4C6FE0
:10B69000DCC152F552510F0B4D6F0101DC31050138
:10B6A000536F0101DB310501526F53335233533372
:10B6B0005233533352330F0E531752510F0B4E6FF9
:10B6C0000101DB510F0BE8CF4FF50501050E080115
:10B6D000D16F470ED06F0001EDEC39F0030E06017B
:10B6E0002E6FE80E2D6F0001DEEC4AF0012C01D028
:10B6F00003D0000E016E14D00101D1A108D00F0EAD
:10B7000005016A6F010E6B6F000156DD07D0100E48
:10B7100005016A6F010E6B6F00014EDD010E016EB7
:10B7200000EF62F00501796B7A6B7B6B7C91050E03
:10B73000EA6E6C0EE96E0801CD6BCF6B0D0ECE6F0D
:10B7400000013AEC2FF0010167B153D07BC5E0FC5A
:10B750007AC5DFFC0C01E26B190EE16F00011AECF7
:10B7600033F002C07EF501C07DF505016B51025C2E
:10B7700033E303E16A517D5D2FE30101C2A129D0CA
:10B7800005017D6B7D510001EEEC11F005017D2B73
:10B79000000187EC28F0180E05017D5DF3E1100E25
:10B7A000E96E6BC5C4F86AC5C3F8000173EC3AF0E2
:10B7B0001B0E05017D6F7D510001EEEC11F00501BE
:10B7C0007D2B000187EC28F0220E05017D5DF3E161
:10B7D0000101FF0E016EECD0190E0801D46F0001BB
:10B7E0001FEC29F005017A2BD8B47B2B0001ABD7D5
:10B7F0000101C2A110D005017D6B7D5100010FEC4C
:10B8000012F005017D2B000187EC28F0100E0501D8
:10B810007D5DF3E1010167A1C9D0036A050179519A
:10B820006C0F016E050E032201C07DF503C07EF58D
:10B8300000011FEC39F07EC5EAFF7DC5E9FF01C0BC
:10B84000EFFF0101C2A115D0036A050179516C0F08
:10B85000E96E050E0320EA6EEFCF7DF57DC5D5F8C4
:10B86000370E0801D66F00012BEC33F0200E87EC69
:10B8700028F005017CB117D0036A79516C0FE96E8D
:10B88000050E0320EA6EEF50FE080CE1036A7951C1
:10B890006C0FE96E050E0320EA6EEFCF6CF57C812C
:10B8A000010E796F78D0036A79516C0FE96E050E3D
:10B8B0000320EA6EEF50EF0860E10101C2A108D059
:10B8C0000D0E000187EC28F00A0E87EC28F001012C
:10B8D000C2A143D005016F510F0B006E00387D6F80
:10B8E000F00E7D1770510F0B7D137E6B7E510001A2
:10B8F00027EC12F005017E2B000187EC28F00D0EDD
:10B9000005017E5DF3E16FC5D5F8570E0801D66FCE
:10B9100000012BEC33F02C0E87EC28F070C5D5F825
:10B92000570E0801D66F00012BEC33F0200E87EC88
:10B9300028F0280E87EC28F07DC5D5F8570E0801B1
:10B94000D66F00012BEC33F0290E87EC28F00D0E9A
:10B9500087EC28F00A0E87EC28F005016F510F0BD9
:10B96000006E00387D6FF00E7D1770510F0B7D114A
:10B97000016E01011DD007D00501320E0801D46F00
:10B9800000011FEC29F0050179510B0802E3792B26
:10B9900002D0796B7C91010167B107D0320E0801AA
:10B9A000D46F00011FEC29F0010135D7EE0E016EB6
:10B9B0000001000C0E0E0501226FFF0E236F300EEA
:10B9C000246F256F266B620E276F286B296B2A6BFD
:10B9D0002B6B2C6B2D6B2E6B2F6BEF0E306F0A0EBB
:10B9E000316FFF0E326F300E336F346F356BB30E25
:10B9F000366F376B386B396B3A6BEF0E3B6F0A0E55
:10BA00003C6FFF0E3D6F300E3E6F3F6F406BB00ED0
:10BA1000416F426B436B446B456BEF0E466F090EF3
:10BA2000476FFF0E486F300E496F4A6F4B6B500ED9
:10BA30004C6F4D6B4E6B4F6BEF0E506F090E516F8D
:10BA4000FF0E526F300E536F546F556B510E566F81
:10BA5000576B586B596BEF0E5A6F080E5B6FFF0EEA
:10BA60005C6F300E5D6F5E6F5F6BB40E606F310E9A
:10BA7000616F626BEF0E636F646B656B666B676B18
:10BA8000686B696B036AC7C16AF503C06BF50C018B
:10BA9000E06B210EDF6F03C0E2FCC7C1E1FC0001D7
:10BAA0001AEC33F0080E05010124666F000E022027
:10BAB000676F675306E16651070803E3676B080E7B
:10BAC000666F6751020809E2FF0A03E16651200828
:10BAD00004E2030E676F200E666F67510F0B6A6FEB
:10BAE000E8CFD1F800015DEC3DF001C04DF5050156
:10BAF00066C500F0003A0F0E001600500F0B6A6F7B
:10BB0000E8CFD1F800015DEC3DF001C04EF5050134
:10BB100066510F0B6A6FE8CFD1F800015DEC3DF084
:10BB200001C04FF5050E0801D16F470ED06F00011F
:10BB3000EDEC39F0030E05016B6FE80E6A6F000142
:10BB4000F1DD01C069F50501695330E06951100864
:10BB500003E06951500824E1020E6A6FFA0E0801F1
:10BB6000D46F00011FEC29F005016A2FF7D7050EED
:10BB70000801D16F470ED06F0001EDEC39F0030ED4
:10BB800006012B6FE80E2A6F000180EC45F0012CB6
:10BB900001D004D0000E016ED6EF61F006D0050191
:10BBA000000E016E0001D6EF61F00501036AC6C107
:10BBB0006AF503C06BF50C01E06B1E0EDF6F03C06E
:10BBC000E2FCC6C1E1FC00011AEC33F0080E0501ED
:10BBD0000124646F000E0220656F655306E1645115
:10BBE000070803E3656B080E646F6551010809E2FD
:10BBF000FF0A03E164516E0804E2020E656F6E0EE7
:10BC0000646F65510F0B6A6FE8CFD1F800015DECEE
:10BC10003DF001C057F5050164C500F0003A0F0E74
:10BC2000001600500F0B6A6FE8CFD1F800015DECF1
:10BC30003DF001C058F5050164510F0B6A6FE8CF64
:10BC4000D1F800015DEC3DF001C059F5050E080189
:10BC5000D16F510ED06F0001EDEC39F0030E0501EC
:10BC60006B6FE80E6A6F00015DDD01C069F50501CB
:10BC700069532DE06951100803E06951500823E130
:10BC8000020E6A6FFA0E0801D46F00011FEC29F052
:10BC900005016A2FF7D7050E0801D16F510ED06F3D
:10BCA0000001EDEC39F0030E06012B6FE80E2A6F50
:10BCB000000180EC45F0012C01D003D0000E016E94
:10BCC00075D305D00501000E016E00016FD301018F
:10BCD000D43905016A6F6B6B0F0E6A176A510F0B2F
:10BCE000006E036A6A6FE8CFD1F800015DEC3DF0A9
:10BCF00001C028F5D4C16AF505016B6B6A510F0BC1
:10BD0000006E036A6A6FE8CFD1F800015DEC3DF088
:10BD100001C029F50101D43105016B6F0101D33157
:10BD200005016A6F6B336A336B336A336B336A3383
:10BD30000F0E6B176A510F0B006E036A6A6FE8CF24
:10BD4000D1F800015DEC3DF001C02AF50101D351AD
:10BD50000F0B006E036AE8CF6AF5E8CFD1F8000157
:10BD60005DEC3DF001C02BF50101D63905016A6F8C
:10BD70006B6B0F0E6A176A510F0B006E036A6A6FC6
:10BD8000E8CFD1F800015DEC3DF001C02CF5D6C143
:10BD90006AF505016B6B6A510F0B006E036A6A6FDF
:10BDA000E8CFD1F800015DEC3DF001C02DF50101B7
:10BDB000D63105016B6F0101D53105016A6F6B3317
:10BDC0006A336B336A336B336A330F0E6B176A5106
:10BDD0000F0B006E036A6A6FE8CFD1F800015DECCB
:10BDE0003DF001C02EF50101D5510F0B006E036A25
:10BDF000E8CF6AF5E8CFD1F800015DEC3DF001C075
:10BE00002FF5050E0801D16F220ED06F0001EDEC69
:10BE100039F0170E05016B6F700E6A6F000182DC3E
:10BE200001C069F5050169532EE06951100803E06E
:10BE30006951500823E1080E6A6FFA0E0801D46FA9
:10BE400000011FEC29F005016A2FF7D7050E080144
:10BE5000D16F220ED06F0001EDEC39F0070E060114
:10BE60002B6FD00E2A6F000180EC45F0012C01D021
:10BE700003D0000E016E9AD205D00501000E016EAE
:10BE8000000194D20501685301E1686B685107080D
:10BE900002E2070E686F370E626F050E0801D16F60
:10BEA0005B0ED06F0001EDEC39F0030E05016B6FF6
:10BEB000E80E6A6F000136DC01C069F505016953BF
:10BEC0002DE06951100803E06951500823E1020E8A
:10BED0006A6FFA0E0801D46F00011FEC29F005010A
:10BEE0006A2FF7D7050E0801D16F5B0ED06F0001E6
:10BEF000EDEC39F0030E06012B6FE80E2A6F0001FE
:10BF000080EC45F0012C01D003D0000E016E4ED222
:10BF100005D00501000E016E000148D20101D8399B
:10BF200005016A6F6B6B0F0E6A176A510F0B006E7B
:10BF3000036A6A6FE8CFD1F800015DEC3DF001C003
:10BF400037F5D8C16AF505016B6B6A510F0B006EAE
:10BF5000036A6A6FE8CFD1F800015DEC3DF001C0E3
:10BF600038F50101D83105016B6F0101D7310501A9
:10BF70006A6F6B336A336B336A336B336A330F0E1A
:10BF80006B176A510F0B006E036A6A6FE8CFD1F826
:10BF900000015DEC3DF001C039F50101D7510F0BF7
:10BFA000006E036AE8CF6AF5E8CFD1F800015DECD6
:10BFB0003DF001C03AF5050E0801D16F310ED06F8A
:10BFC0000001EDEC39F0030E05016B6FE80E6A6FAE
:10BFD000000192EC5BF001C069F50501695328E0AE
:10BFE0006951100803E06951500822E1080E6A6F98
:10BFF000FA0E0801D46F00011FEC29F005016A2F29
:10C00000F7D7050E0801D16F310ED06F0001EDECAE
:10C0100039F0070E06012B6FD00E2A6F000180EC5D
:10C0200045F0012C01D003D0000E016EBFD10501F7
:10C030000101D1A742D01B0E05016A6F6B6B000195
:10C04000DCEC58F0030E05016B6FE80E6A6F00011F
:10C0500092EC5BF001C069F5050169532CE0695170
:10C06000100803E06951500821E1040E6A6FFA0ECE
:10C070000801D46F00011FEC29F005016A2FF7D7E2
:10C080001B0E6A6F6B6B0001DCEC58F0030E0601AF
:10C090002B6FE80E2A6F000180EC45F0012C01D0D7
:10C0A00003D0000E016E82D105D00501000E016E95
:10C0B00000017CD10501FCD001011C0E05016A6F55
:10C0C0006B6B0001DCEC58F0030E05016B6FE80EA2
:10C0D0006A6F000192EC5BF001C069F505016953DC
:10C0E0002BE06951100803E06951500821E1040E6A
:10C0F0006A6FFA0E0801D46F00011FEC29F00501E8
:10C100006A2FF7D71C0E6A6F6B6B0001DCEC58F0DE
:10C11000030E06012B6FE80E2A6F000180EC45F03C
:10C12000012C01D003D0000E016E40D105D00501D5
:10C13000000E016E00013AD10101DA3905016A6F82
:10C140006B6B0F0E6A176A510F0B006E036A6A6FF2
:10C15000E8CFD1F800015DEC3DF001C042F5DAC155
:10C160006AF505016B6B6A510F0B006E036A6A6F0B
:10C17000E8CFD1F800015DEC3DF001C043F50101CD
:10C18000DA3105016B6F0101D93105016A6F6B333B
:10C190006A336B336A336B336A330F0E6B176A5132
:10C1A0000F0B006E036A6A6FE8CFD1F800015DECF7
:10C1B0003DF001C044F50101D9510F0B006E036A37
:10C1C000E8CF6AF5E8CFD1F800015DEC3DF001C0A1
:10C1D00045F5050E0801D16F3C0ED06F0001EDEC66
:10C1E00039F0070E05016B6FD00E6A6F000192ECFB
:10C1F0005BF001C069F5050169535AE06951100807
:10C2000003E0695150084FE1080E6A6FFA0E080109
:10C21000D46F00011FEC29F005016A2FF7D7050E36
:10C220000801D16F3C0ED06F0001EDEC39F0070E24
:10C2300005016B6FD00E6A6F000192EC5BF001C0DC
:10C2400069F5050169532EE06951100803E0695151
:10C25000500823E1080E6A6FFA0E0801D46F00013E
:10C260001FEC29F005016A2FF7D7050E0801D16FE1
:10C270003C0ED06F0001EDEC39F0070E06012B6F7C
:10C28000D00E2A6F000180EC45F0012C01D003D0C4
:10C29000000E016E8BD005D00501000E016E00016D
:10C2A00085D0050105D0000E016E00017FD005018B
:10C2B0000101D1A309D0110E05016A6F010E6B6F48
:10C2C0000001DCEC58F008D0130E05016A6F010E76
:10C2D0006B6F0001DCEC58F0640E0801D46F0001B4
:10C2E0001FEC29F00101D1B10AD0100E05016A6FCF
:10C2F000010E6B6F0001DCEC58F009D001010F0E4C
:10C3000005016A6F010E6B6F0001DCEC58F0640EE2
:10C310000801D46F00011FEC29F00101D1A530D034
:10C32000DC6B480EDB6FD89002010E35036A370FC5
:10C33000016E000E03220150BF0FE96E010E0320B3
:10C34000EA6EDCC1ECFFED52DBC1EFFF140E05011C
:10C350006D6F010E6E6F000185EC46F0180E050141
:10C360006D6F010E6E6F000185EC46F0150E050134
:10C370006D6F010E6E6F000185EC46F011D001016A
:10C38000140E05016D6F010E6E6F000185EC46F015
:10C39000180E05016D6F010E6E6F000185EC46F001
:10C3A000640E0801D46F00011FEC29F005EF62F064
:10C3B000010E016E09EF62F00101D139006E0F0E1E
:10C3C00000160050020A000119E0010A17E0060AEF
:10C3D00015E00D0A13E0010A11E00E0A0FE0030A4E
:10C3E0000DE00F0A0BE00A0A09E0070A07E00C0A51
:10C3F00005E0060A08E0010A0BE00ED028EF59F02C
:10C4000001500ED00DD0DAEF5CF0015009D008D009
:10C41000CFD7015005D004D0000E016E01D000D05E
:10C42000000C0DC5A5F8DAEC57F00201593D7CD09F
:10C430000DC522F50C0E0501236F00014EEC33F003
:10C44000012C71D0050EEA6E0E0EE96EF2CF22F5C8
:10C45000F29E000E70EC1FF00A000900F550EE6E1F
:10C460000009FBE1050122BFF28E050E0801A66F4F
:10C470000E0EA56F000188EC2FF00101D139006E7E
:10C480000F0E001600500D0849E1D1A70AD01B0E6F
:10C4900005016D6F010E6E6F0001F9EC52F009D0CD
:10C4A00001011C0E05016D6F010E6E6F0001F9ECAC
:10C4B00052F00101D1A50AD0150E05016D6F010ED4
:10C4C0006E6F0001F9EC52F009D00101140E050164
:10C4D0006D6F010E6E6F0001F9EC52F00C0E02014F
:10C4E0000F6F350E05016D6F6E6B0001F9EC52F0A8
:10C4F000070E0501D86FD00ED76F010ED96F00015E
:10C50000C4EC51F03A0E0501D86F980ED76F010EAA
:10C51000D96F0001C4EC51F003D0010100014CDFE0
:10C52000010E016E2BD00201050EEA6E0E0EE96EB1
:10C53000F2CF22F5F29E000E000188EC1FF00A00F7
:10C540000900F550EE6E0009FBE1050122BFF28EF5
:10C55000050E0801A66F0E0EA56F000188EC2FF0E6
:10C56000080E0501226FFA0E0801D16F00010AECD6
:10C5700029F00501222FF7D7000E016E0001000CF3
:10C5800005013B51390805E2370E3B5D016E05D0D0
:10C5900004D0300E3B5D016E00D00001000C05019F
:10C5A000336B346B356B020E366F900E376F21C5CF
:10C5B000E9FF22C5EAFFEC6AED52EF6A050EEA6E6A
:10C5C000230EE96E0801CD6BCF6B100ECE6F00010C
:10C5D0003AEC2FF00101D139006E0F0E0016005019
:10C5E0000C0805E1050E0501366FFE0E376F020ED1
:10C5F0000501386FC80E0801D46F00011FEC29F047
:10C600000501382FF7D7010167A13BD00501335150
:10C610000F08D8B002D0010134D000011FEC39F06E
:10C6200001C034F50A0E0801D46F00011FEC29F097
:10C630000101C2A10DD034C5D5F8570E0801D66F3F
:10C6400000012BEC33F0200E87EC28F007D001011D
:10C650000A0E0801D46F00011FEC29F005013751C3
:10C66000345D04E1336B34C523F50AD0332B036A00
:10C670003351230FE96E050E0320EA6E34C5EFFF38
:10C68000C2D7030E05013625335D03E2000E016EAD
:10C690006FD00101D139006E0F0E001600500C084A
:10C6A00029E136C535F5030E05013625355D01E076
:10C6B00022E2036A3551230F016E050E032201C0E9
:10C6C00038F503C039F5036A3551230FE96E050EBD
:10C6D0000320EA6EEFCF3AF53AC53BF5000150DF93
:10C6E00039C5EAFF38C5E9FF01C0EFFF0501352B69
:10C6F0000101D9D70501356B3551030837E321C551
:10C70000E9FF22C5EAFFEF34026EEC34036E023615
:10C7100003360236033602360336F00E0216025096
:10C72000ED52EF6E03C0ECFF22C503F022C5EAFF15
:10C7300021C5E9FFECCF3BF5ED52EFCF3AF535518E
:10C740003625036A230FE96E050E0320EA6EEF50CB
:10C750000F0B3A113BC503F022C5EAFF21C5E9FFE3
:10C760003BC5ECFFED52EF6E352BC6D7010E016EC7
:10C770000001000C0501336B346B020E356F900E17
:10C78000366F21C5E9FF22C5EAFFEF6A050EEA6EA2
:10C79000230EE96E0801CD6BCF6B100ECE6F00013A
:10C7A0003AEC2FF00101D139006E0F0E0016005047
:10C7B0000C0805E1050E0501356FFE0E366F020E01
:10C7C0000501376FC80E0801D46F00011FEC29F076
:10C7D0000501372FF7D7010167A13BD00501335180
:10C7E0000F08D8B002D0010134D000011FEC39F09D
:10C7F00001C034F50A0E0801D46F00011FEC29F0C6
:10C800000101C2A10DD034C5D5F8570E0801D66F6D
:10C8100000012BEC33F0200E87EC28F007D001014B
:10C820000A0E0801D46F00011FEC29F005013651F2
:10C83000345D04E1336B34C523F50AD0332B036A2E
:10C840003351230FE96E050E0320EA6E34C5EFFF66
:10C85000C2D7020E05013525335D03E2000E016EDD
:10C860007CD00101D139006E0F0E001600500C086B
:10C870003EE1036A05013551230F016E050E0322C7
:10C8800001C037F503C038F5036A3551230FE96E4F
:10C89000050E0320EA6EEFCF39F539C53BF50001EF
:10C8A0006FDE38C5EAFF37C5E9FF01C0EFFF010EB3
:10C8B00005013525036A230F016E050E032201C011
:10C8C00037F503C038F5010E3525036A230FE96EED
:10C8D000050E0320EA6EEFCF39F539C53BF50001AF
:10C8E0004FDE38C5EAFF37C5E9FF01C0EFFF22C5BB
:10C8F00003F00501036A3551230FE96E050E03208D
:10C90000EA6EEFCF39F522C5EAFF21C5E9FF39C547
:10C91000EFFF21C5E9FF22C5EAFFEF38006EF00EF8
:10C92000001600C0EFFF22C503F022C5EAFF21C5B3
:10C93000E9FFEFCF39F5010E3525036A230FE96EC4
:10C94000050E0320EA6EEF500F0B391122C5EAFFE6
:10C9500021C5E9FFEF6E010E016E0001000C05011B
:10C960000D6B0E6B0F6B00012AEC3CF00101D1390D
:10C97000006E0F0E001600500C081DE0D139006E3D
:10C980000F0E001600500D0816E0080E05016D6F21
:10C990006E6B00015BEC4DF0050E0501226F0E0E73
:10C9A000216F0001FCDD012C04D00FC5DCF10EC5A8
:10C9B000DBF15DD00101D139006E0F0E0016005081
:10C9C0000C0818E1080E05016D6F6E6B000185EC17
:10C9D00046F0050E0501226F0D0E216F0001CADE23
:10C9E000012C06D005010D510101DC6BDB6F00014C
:10C9F0003ED00101D139006E0F0E001600500D0817
:10CA000037E1080E05016D6F6E6B0001F9EC52F015
:10CA1000050E0501226F100E216F0F0E236F070EFA
:10CA2000256FD00E246F266B00019AEC56F0012C76
:10CA30001ED016C53BF5A4DD01C01FF517C53BF59B
:10CA40009FDD01380501216FF00E211718C53BF558
:10CA5000000196DD050121510110206F1FC50FF562
:10CA600020C50EF50FC5DCF10EC5DBF1000101019B
:10CA70000001000C05013E6B3F6B406B516B900E4B
:10CA8000526F0D0E6D6F010E6E6F00015BEC4DF07D
:10CA9000050EEA6E410EE96E0801CD6BCF6B100EEC
:10CAA000CE6F00013AEC2FF03C0E05016D6F6E6BFE
:10CAB00000015BEC4DF00101C2A110D00501536BE8
:10CAC00053510001ECEC10F00501532B000187ECF1
:10CAD00028F0110E0501535DF3E1010167B141D06A
:10CAE0003FC5E0FC3EC5DFFC0C01E26B320EE16F9E
:10CAF00000011AEC33F002C054F501C053F50501F2
:10CB0000545303E15351C70820E20101C2A10FD0E1
:10CB10000501536B5351000104EC11F00501532B37
:10CB2000000187EC28F00B0E0501535DF3E10501D0
:10CB30003D5308E10E0E6D6F010E6E6F00015BEC50
:10CB40004DF00501000E016E67D0320E0801D46F62
:10CB500000011FEC29F005013E2BD8B43F2B010149
:10CB6000BDD767A134D0050151510308D8B002D018
:10CB700001012DD000011FEC39F001C040F50A0E73
:10CB80000801D46F00011FEC29F005015251405DEE
:10CB900004E1516B40C541F50AD0512B036A515154
:10CBA000410FE96E050E0320EA6E40C5EFFF01015B
:10CBB000C2A10CD040C5D5F8570E0801D66F0001B0
:10CBC0002BEC33F0200E87EC28F00101CAD7C2A16C
:10CBD00008D00A0E000187EC28F00D0E87EC28F033
:10CBE00001010501515103080BE1443D09D04251B7
:10CBF000500806E14351020803E3010E016E0CD018
:10CC00003D5308E10E0E6D6F010E6E6F00015BEC7F
:10CC10004DF00501000E016E0001000C0501146BC2
:10CC2000156B166B276B900E286F050EEA6E290E9A
:10CC3000E96E0801CD6BCF6B140ECE6F00013AEC9C
:10CC40002FF0050EEA6E170EE96E0801CD6BCF6B63
:10CC5000100ECE6F00013AEC2FF0020E05016D6F41
:10CC60006E6B00015BEC4DF00101C2A110D005011B
:10CC70003D6B3D5100011AEC0EF005013D2B00010A
:10CC800087EC28F00E0E05013D5DF3E1010167B16F
:10CC900036D015C5E0FC14C5DFFC0C01E26B320E8A
:10CCA000E16F00011AEC33F002C03EF501C03DF522
:10CCB00005013E5303E13D51C70815E20101C2A140
:10CCC00010D005013D6B3D51000131EC0EF0050126
:10CCD0003D2B000187EC28F00A0E05013D5DF3E1D4
:10CCE000010172EF6AF0320E0801D46F00011FECEF
:10CCF00029F00501142BD8B4152B0101C8D767A161
:10CD000034D0050127510F08D8B002D001012DD031
:10CD100000011FEC39F001C016F50A0E0801D46FAE
:10CD200000011FEC29F005012851165D04E1276B75
:10CD300016C517F50AD0272B036A2751170FE96E7E
:10CD4000050E0320EA6E16C5EFFF0101C2A10CD04B
:10CD500016C5D5F8570E0801D66F00012BEC33F03D
:10CD6000200E87EC28F00101CAD7C2A107D00A0E15
:10CD7000000187EC28F00D0E87EC28F00501275103
:10CD80000408D8B035D319C50FF51AC50EF51BC563
:10CD900011F51CC510F51DC513F51EC512F510C5FE
:10CDA00000F011C503F0040E115D06E1020E005CF7
:10CDB0000001D8B464D00501080E035C05E10052FF
:10CDC0000001D8B4C4D00501040E035C06E10D0EC9
:10CDD000005C0001D8B4F9D00501040E035C06E143
:10CDE0000E0E005C0001D8B425D10501050E035CD0
:10CDF00006E1030E005C0001D8B452D10501050E16
:10CE0000035C06E1010E005C0001D8B449D10501C4
:10CE1000040E035C06E10F0E005C0001D8B4AAD139
:10CE20000501050E035C06E1050E005C0001D8B4A7
:10CE3000D6D10501050E035C06E1040E005C00017D
:10CE4000D8B403D20501040E035C06E12C0E005C8D
:10CE50000001D8B464D20501200E035C06E1010E86
:10CE6000005C0001D8B45BD20501040E035C06E14E
:10CE70002D0E005C0001D8B452D2050186D201010A
:10CE8000D16B010E05013D6F0001F4DD012C2BD0AB
:10CE9000600E0101D113C2A110D005013D6B3D51BF
:10CEA000000146EC0EF005013D2B000187EC28F057
:10CEB000140E05013D5DF3E10101050EEA6E290E38
:10CEC000E96EF2CF3DF5F29E000E000160EC0EF02F
:10CED0000A000900F550EE6E0009FBE105013DBFB7
:10CEE000F28E29D000010101D189C2A110D0050123
:10CEF0003D6B3D51000178EC0EF005013D2B00012A
:10CF000087EC28F0100E05013D5DF3E10101050EEF
:10CF1000EA6E290EE96EF2CF3DF5F29E000E000199
:10CF200090EC0EF00A000900F550EE6E0009FBE1EE
:10CF300005013DBFF28E0D513009396F050E080114
:10CF4000A66F290EA56F000188EC2FF04FD20101CA
:10CF5000D16B500ED113C2A110D005013D6B3D51D4
:10CF60000001A8EC0EF005013D2B000187EC28F034
:10CF7000140E05013D5DF3E10101050EEA6E290E77
:10CF8000E96EF2CF3DF5F29E000E0001C2EC0EF00C
:10CF90000A000900F550EE6E0009FBE105013DBFF6
:10CFA000F28E0D513009396F050E0801A66F290E5A
:10CFB000A56F000188EC2FF0390E05016A6F010E94
:10CFC0006B6F0001DCEC58F011D20101D16BD18BF9
:10CFD000C2A110D005013D6B3D510001DAEC0EF00D
:10CFE00005013D2B000187EC28F0110E05013D5D88
:10CFF000F3E10101050EEA6E290EE96EF2CF3DF56F
:10D00000F29E000E0001F2EC0EF00A000900F5504D
:10D01000EE6E0009FBE105013DBFF28E0D513009B6
:10D02000396F050E0801A66F290EA56F000188EC67
:10D030002FF0DCD10101D16B300ED113C2A110D081
:10D0400005013D6B3D5100010AEC0FF005013D2B40
:10D05000000187EC28F0100E05013D5DF3E10101B0
:10D06000050EEA6E290EE96EF2CF3DF5F29E000E36
:10D07000000122EC0FF00A000900F550EE6E0009E5
:10D08000FBE105013DBFF28E0D513009396F050EF0
:10D090000801A66F290EA56F000188EC2FF0A6D11C
:10D0A0000501102D32D0115105082FE10E2D2DD084
:10D0B0000F532BE10101D16B900ED113C2A110D0FF
:10D0C00005013D6B3D5100013AEC0FF005013D2B90
:10D0D000000187EC28F0110E05013D5DF3E101012F
:10D0E000050EEA6E290EE96EF2CF3DF5F29E000EB6
:10D0F000000152EC0FF00A000900F550EE6E000935
:10D10000FBE105013DBFF28E29D00101D16BD18930
:10D11000C2A110D005013D6B3D5100016AEC0FF03A
:10D1200005013D2B000187EC28F00F0E05013D5D48
:10D13000F3E10101050EEA6E290EE96EF2CF3DF52D
:10D14000F29E000E000181EC0FF00A000900F5507C
:10D15000EE6E0009FBE105013DBFF28E0D51300975
:10D16000396F050E0801A66F290EA56F000188EC26
:10D170002FF03CD10101D16BD18FC2A110D005019C
:10D180003D6B3D51000199EC0FF005013D2B000175
:10D1900087EC28F0100E05013D5DF3E10101050E5D
:10D1A000EA6E290EE96EF2CF3DF5F29E000E000107
:10D1B000B1EC0FF00A000900F550EE6E0009FBE13A
:10D1C00005013DBFF28E0D513009396F050E080182
:10D1D000A66F290EA56F000188EC2FF007D1010181
:10D1E000D16B700ED113C2A110D005013D6B3D5122
:10D1F0000001C9EC0FF005013D2B000187EC28F080
:10D20000110E05013D5DF3E10101050EEA6E290EE7
:10D21000E96EF2CF3DF5F29E000E0001E1EC0FF059
:10D220000A000900F550EE6E0009FBE105013DBF63
:10D23000F28E0D513009396F050E0801A66F290EC7
:10D24000A56F000188EC2FF0D1D0050112510E0816
:10D2500031E113510E082EE10101D16BB00ED11353
:10D26000C2A110D005013D6B3D510001F9EC0FF05A
:10D2700005013D2B000187EC28F0100E05013D5DF6
:10D28000F3E10101050EEA6E290EE96EF2CF3DF5DC
:10D29000F29E000E000111EC10F00A000900F5509A
:10D2A000EE6E0009FBE105013DBFF28E0D51300924
:10D2B000386F2CD00101D16BD18DC2A110D00501E6
:10D2C0003D6B3D51000129EC10F005013D2B0001A3
:10D2D00087EC28F0100E05013D5DF3E10101050E1C
:10D2E000EA6E290EE96EF2CF3DF5F29E000E0001C6
:10D2F00041EC10F00A000900F550EE6E0009FBE168
:10D3000005013DBFF28E0D513009396F050E080140
:10D31000A66F290EA56F000188EC2FF067D00101E0
:10D32000D16BA00ED113C2A110D005013D6B3D51B0
:10D33000000159EC10F005013D2B000187EC28F0AD
:10D34000160E05013D5DF3E10101050EEA6E290EA1
:10D35000E96EF2CF3DF5F29E000E000174EC10F084
:10D360000A000900F550EE6E0009FBE105013DBF22
:10D37000F28E0D513009396F050E0801A66F290E86
:10D38000A56F000188EC2FF031D00101C2A110D0AF
:10D3900005013D6B3D5100018CEC10F005013D2B6A
:10D3A000000187EC28F0100E05013D5DF3E101015D
:10D3B000D16B050EEA6E290EE96EF2CF3DF5F29EB5
:10D3C000000E0001A4EC10F00A000900F550EE6E0A
:10D3D0000009FBE105013DBFF28E050E0801A66FB5
:10D3E000290EA56F000188EC2FF000D07AD005013E
:10D3F0002751030846E11A3D44D01851600803E064
:10D40000185161083EE13D6B00013AEC65F0012CDA
:10D4100038D00101D16B600ED113C2A110D005012B
:10D420003D6B3D510001BBEC10F005013D2B0001AF
:10D4300087EC28F0130E05013D5DF3E10101050EB7
:10D44000EA6E290EE96EF2CF3DF5F29E000E000164
:10D45000D4EC10F00A000900F550EE6E0009FBE173
:10D4600005013DBFF28E0D513009396F050E0801DF
:10D47000A66F290EA56F000188EC2FF0010132D0B4
:10D4800000010101C2A110D005013D6B3D51000119
:10D490008CEC10F005013D2B000187EC28F0100EFC
:10D4A00005013D5DF3E10101D16B050EEA6E290E28
:10D4B000E96EF2CF3DF5F29E000E0001A4EC10F0F3
:10D4C0000A000900F550EE6E0009FBE105013DBFC1
:10D4D000F28E050E0801A66F290EA56F000188ECDB
:10D4E0002FF001010001E6EF6BF0040EEA6EEF0E83
:10D4F000E96E0801CD6BCF6B140ECE6F00013AECD4
:10D500002FF0330E05016D6F6E6B000185EC46F058
:10D510001FEF4AF00152D8A487D105016D6B6E6BE5
:10D5200000015BEC4DF0070E06012E6FD00E2D6F43
:10D530000001DEEC4AF00152D8A444D105016D6B24
:10D540006E6B00015BEC4DF0070E06012E6FD00EE6
:10D550002D6F0001DEEC4AF00152D8A433D1010155
:10D56000C1BB2DD0040EEA6EEF0EE96EF2CF0DF5C1
:10D57000F29E000E000167EC0DF00A000900F55064
:10D58000EE6E0009FBE105010DBFF28E0401EE51C4
:10D590003009FF6F040E0801A66FEF0EA56F0001A2
:10D5A00088EC2FF0040E05010D6FFA0E0801D46F00
:10D5B00000011FEC29F005010D2FF7D7F5D10D0E55
:10D5C00005016D6F6E6B0001F9EC52F0320E08012F
:10D5D000D46F00011FEC29F0050E0501226F030E28
:10D5E000216F0A0E236F3A0E256F980E246F010EDD
:10D5F000266F00019AEC56F0012C01D02ED0040EBB
:10D60000EA6EEF0EE96EF2CF0DF5F29E000E67ECBA
:10D610000DF00A000900F550EE6E0009FBE105016E
:10D620000DBFF28E0401EE513009FF6F040E0801A8
:10D63000A66FEF0EA56F000188EC2FF0040E050118
:10D640000D6FFA0E0801D46F00011FEC29F00501DF
:10D650000D2FF7D7A9D1B5D000010101D16BD00EA4
:10D66000D113040EEA6EEF0EE96EF2CF0DF5F29EC5
:10D67000000E00017FEC0DF00A000900F550EE6E7F
:10D680000009FBE105010DBFF28E0401EE513009E6
:10D69000FF6F040E0801A66FEF0EA56F000188EC66
:10D6A0002FF00101C2A10FD005010D6B0D5100013A
:10D6B00097EC0DF005010D2B000187EC28F0140EFE
:10D6C00005010D5DF3E1040E05010D6FFA0E080171
:10D6D000D46F00011FEC29F005010D2FF7D7130EB1
:10D6E000D86F880ED76FD96B0001C4EC51F02AECCB
:10D6F0003CF00101C1A307D0EEC40DF5000111EC0F
:10D7000062F038D00101310E05016D6F6E6B0001C2
:10D71000F9EC52F01F0E0501D86F400ED76F010EC5
:10D72000D96F0001C4EC51F0200E05010D6FFA0E07
:10D730000801D46F00011FEC29F005010D2FF7D768
:10D7400000012AEC3CF03E0E05016D6F6E6B00018E
:10D75000F9EC52F01F0E0501D86F400ED76F010E85
:10D76000D96F0001C4EC51F00101D183D185D1877B
:10D77000D1910001036A0401EE51220F016E000EE7
:10D7800003220150BF0FE96E010E0320EA6ED1C1E2
:10D79000EFFF0001AFEC64F0D8900401EE35036AAE
:10D7A000370F016E000E03220150BF0FE96E010E0C
:10D7B0000320EA6EDCC1ECFFED52DBC1EFFF050197
:10D7C000F3D00001EEC40DF50EEF66F00101D15368
:10D7D00002E10501E9D00D0E05016D6F6E6B0001D0
:10D7E0005BEC4DF04E0E06012E6F200E2D6F0001EA
:10D7F000DEEC4AF00101C1A307D0EEC40DF5000133
:10D8000011EC62F010D00101310E05016D6F6E6BED
:10D8100000015BEC4DF04E0E06012E6F200E2D6FB9
:10D820000001DEEC4AF072D00101D16BC00ED113C1
:10D83000040EEA6EEF0EE96EF2CF0DF5F29E000EC9
:10D840000001B1EC0DF00A000900F550EE6E000980
:10D85000FBE105010DBFF28E0401EE513009FF6FAF
:10D86000040E0801A66FEF0EA56F000188EC2FF0E3
:10D870000101C2A10FD005010D6B0D510001C9ECD2
:10D880000DF005010D2B000187EC28F0100E0501AD
:10D890000D5DF3E100012AEC3CF00D0E05016D6F0A
:10D8A0006E6B000185EC46F01F0E06012B6F400EDB
:10D8B0002A6F000180EC45F02AEC3CF01A0E0501BD
:10D8C0006A6F6B6B0001DCEC58F0030E06012B6FE6
:10D8D000E80E2A6F000180EC45F00101C1A307D0DA
:10D8E000EEC40DF5000111EC62F010D00101310E13
:10D8F00005016D6F6E6B000185EC46F0170E060199
:10D900002B6F700E2A6F000180EC45F00101D1836E
:10D91000110E05016A6F010E6B6F0001DCEC58F00F
:10D920000101D1871B0E05016A6F010E6B6F0001AB
:10D93000DCEC58F00101D185150E05016A6F010E6E
:10D940006B6F0001DCEC58F00101D191100E050164
:10D950006A6F010E6B6F0001DCEC58F0036A020184
:10D960000E51220F016E000E03220150BF0FE96E0F
:10D97000010E0320EA6ED1C1EFFF0001AFEC64F0AD
:10D98000D89002010E35036A370F016E000E032294
:10D990000150BF0FE96E010E0320EA6EDCC1ECFFFF
:10D9A000ED52DBC1EFFF0501000135EF6DF0010E17
:10D9B000EA6EE10EE96E0801CD6BCF6B070ECE6FFC
:10D9C00000013AEC2FF03CEC39F00101C2A10FD07C
:10D9D0000401EE6BEE51000132EC0DF00401EE2B70
:10D9E000000187EC28F0200E0401EE5DF3E1010E4A
:10D9F0000401ED6FED5106083BE30101C2A122D005
:10DA00000401EE6BEE51000152EC0DF00401EE2B1F
:10DA1000000187EC28F0050E0401EE5DF3E1EDC492
:10DA2000ABF81F0E0801AC6F00016BEC39F03A0E39
:10DA300087EC28F0200E87EC28F0200E87EC28F0E9
:10DA400007D00101320E0801D46F00011FEC29F04C
:10DA5000EDC40BF5E3EC44F00A0E0801D46F0001AD
:10DA60001FEC29F0EDC4EEF440D50401ED2BC2D734
:10DA70000001000C040EEA6EF80EE96E0801CD6B91
:10DA8000CF6B130ECE6F00013AEC2FF0050EEA6E4D
:10DA90000B0EE96E0801CD6BCF6B130ECE6F00013C
:10DAA0003AEC2FF00C01E06BF6C4DFFCE26B120ED7
:10DAB000E16F00011AEC33F002C003F001505A0F7D
:10DAC000016E020E032201C01EF503C01FF5040EF5
:10DAD0000801CE6FF80ECD6F03C0D0F801C0CFF8AB
:10DAE000120ED16F000149EC2FF00C0E0401F86FFB
:10DAF000036A0301C251C30FE96E030E0320EA6EED
:10DB0000EF2C03D03E0E0401F96F040E0801CE6F16
:10DB1000F80ECD6F00012EEC2AF0050E0801D46F2F
:10DB200000011FEC29F00C01E06BF7C4DFFCE26B95
:10DB3000120EE16F00011AEC33F002C003F0015045
:10DB40005A0F016E020E032201C01EF503C01FF51D
:10DB5000050E0801CE6F0B0ECD6F03C0D0F801C0CB
:10DB6000CFF8120ED16F000149EC2FF00A0E05011B
:10DB70000B6F036A0301C251C30FE96E030E03204A
:10DB8000EA6EEF50020803E13E0E05010C6F050E30
:10DB90000801CE6F0B0ECD6F00012EEC2AF0000CA9
:10DBA0000401ED6BED6BED51020821E3036AED51C9
:10DBB000C30FE96E030E0320EA6EEF6A036AED51AC
:10DBC000C70F016E030E032203C0EFF4036AED5189
:10DBD000CF0FE96E030E0320EA6EEFCFF0F4EFC42F
:10DBE000EAFF01C0E9FFF0C4EFFFED2BDCD7030132
:10DBF000C26B01016793679567970401636B63C408
:10DC000065F465C464F4036A0301C251C70FE96E89
:10DC1000030E0320EA6EEFCFEEF4036AC251C70F82
:10DC2000E96E030E0320EA6E010EEF240401EF6F8C
:10DC3000EEC4F6F4F76F00011DDF000C0401D56B94
:10DC4000D66BD76BD86BFA0E0801D16F00010AECC6
:10DC500029F0FF0E0401A66FA56FA76FAA6BA96F2D
:10DC6000A86F5B90589E456A446A476A466A4C6A48
:10DC70005B925B945B965C6A5D6A5E6A5F6AD86B76
:10DC8000D8510C080AE3036AD8514D0FE96E020E11
:10DC90000320EA6EEF6AD82BF3D7010EEA6EBF0EAF
:10DCA000E96E0801CD6BCF6B590ECE6F00013AECD7
:10DCB0002FF00401D86BD8510108D8A086D0D851D4
:10DCC000040DF350EE6BED6F690EED25E96E040E59
:10DCD000EE21EA6EFF0EEC6EED52EF6ED851040DA0
:10DCE000F350EE6BED6F020EED25016E000EEE218E
:10DCF000036E0150690FE96E040E0320EA6EEF6AAD
:10DD0000D851040DF350EE6BED6F750EED25E96EF5
:10DD1000040EEE21EA6EFF0EEC6EED52EF6ED8515E
:10DD2000040DF350EE6BED6F020EED25016E000E4B
:10DD3000EE21036E0150750FE96E040E0320EA6EAA
:10DD4000EF6AD851040DF350EE6BED6F810EED25A7
:10DD5000E96E040EEE21EA6EFF0EEC6EED52EF6EF0
:10DD6000D851040DF350EE6BED6F020EED25016EF0
:10DD7000000EEE21036E0150810FE96E040E0320A8
:10DD8000EA6EEF6AD851040DF350EE6BED6F8D0E15
:10DD9000ED25E96E040EEE21EA6EFF0EEC6EED52FB
:10DDA000EF6ED851040DF350EE6BED6F020EED25C2
:10DDB000016E000EEE21036E01508D0FE96E040E10
:10DDC0000320EA6EEF6AD82B76D7040EEA6EC10EF6
:10DDD000E96EF2CFEDF4F29E000E00016CEC22F041
:10DDE0000A000900F550EE6E0009FBE10401EDBFE9
:10DDF000F28E040E0801A66FC10EA56F000188EC1B
:10DE00002FF06FEF35F0040E0401ED6FFA0E0801EC
:10DE1000D16F00010AEC29F00401ED2FF7D79D80A6
:10DE2000F28A070EB46E9750976E0D0E006E002E9C
:10DE3000FED7B450A19CB56AFA0E0801D16F00015B
:10DE40000AEC29F011C26AF410C269F411C26EF42E
:10DE500010C26DF4196AF2BE198EF29E400E0C01CA
:10DE6000E66FE76B000163EC24F019BEF28E02C08E
:10DE7000D6F401C0D5F4196AF2BE198EF29E440E92
:10DE80000C01E66FE76B000163EC24F019BEF28E23
:10DE900002C0D6F401C0D5F4196AF2BE198EF29E02
:10DEA000420E0C01E66FE76B000163EC24F019BE33
:10DEB000F28E02C0D6F401C0D5F4196AF2BE198EF2
:10DEC000F29E460E0C01E66FE76B000163EC24F056
:10DED00019BEF28E02C0D6F401C0D5F4010EEA6E6E
:10DEE000680EE96E0801CD6BCF6B400ECE6F00015E
:10DEF0003AEC2FF0646B64C062F001016791040E8C
:10DF00000801A66FC10EA56F000188EC2FF0656BAC
:10DF10000D0E666FEA6A680EE96E0801CD6BCF6B75
:10DF2000FF0ECE6F00013AEC2FF0636B63C061F01F
:10DF30005B9EA38A9D8AC00EF2120101BFA17BD114
:10DF4000040EEA6EC10EE96EF2CFEDF4F29E000E01
:10DF5000000184EC22F00A000900F550EE6E000981
:10DF6000FBE10401EDBFF28E040E0801A66FC10EA5
:10DF7000A56F000188EC2FF0BDEC36F00401ED6BCD
:10DF8000ED51000110EC19F00401ED2B000187ECBC
:10DF900028F0040E0401ED5DF3E1040EEE6FD90EDE
:10DFA000ED6F140EEF6F0001F8EF37F0012C29D060
:10DFB000040EEA6EC10EE96EF2CFEDF4F29E000E91
:10DFC0009BEC22F00A000900F550EE6E0009FBE11F
:10DFD0000401EDBFF28E040E0801A66FC10EA56FFD
:10DFE000000188EC2FF0080E0401ED6FFA0E080115
:10DFF000D16F00010AEC29F00401ED2FF7D7F2D020
:10E000000001F2CFEDF4F29EAA6A110EA96EA69C51
:10E01000A69EA680A8500401EDBFF28ED76FD7B19F
:10E02000B9D0D781AA6A110EA96ED7C4A8FFA69C41
:10E03000A69EA684F2CF00F0F29E0F01550EA76EA9
:10E04000AA0EA76EA682A6B2FED7A6940050F21220
:10E05000040EEA6EC10EE96EF2CFEDF4F29E000EF0
:10E060000001B2EC22F00A000900F550EE6E000942
:10E07000FBE10401EDBFF28E040E0801A66FC10E94
:10E08000A56F000188EC2FF0280E0401ED6FFA0E49
:10E090000801D16F00010AEC29F00401ED2FF7D738
:10E0A000040EEA6EC10EE96EF2CFEDF4F29E000EA0
:10E0B0000001CAEC22F00A000900F550EE6E0009DA
:10E0C000FBE10401EDBFF28E040E0801A66FC10E44
:10E0D000A56F000188EC2FF0280E0401ED6FFA0EF9
:10E0E0000801D16F00010AEC29F00401ED2FF7D7E8
:10E0F000040EEA6EC10EE96EF2CFEDF4F29E000E50
:10E100000001E2EC22F00A000900F550EE6E000971
:10E11000FBE10401EDBFF28E040E0801A66FC10EF3
:10E12000A56F000188EC2FF0280E0401ED6FFA0EA8
:10E130000801D16F00010AEC29F00401ED2FF7D797
:10E14000040EEA6EC10EE96EF2CFEDF4F29E000EFF
:10E150000001FAEC22F00A000900F550EE6E000909
:10E16000FBE10401EDBFF28E040E0801A66FC10EA3
:10E17000A56F000188EC2FF0040E0401ED6FFA0E7C
:10E180000801D16F00010AEC29F00401ED2FF7D747
:10E19000FF0028D0040EEA6EC10EE96EF2CFEDF456
:10E1A000F29E000E000111EC23F00A000900F55068
:10E1B000EE6E0009FBE10401EDBFF28E040E0801D2
:10E1C000A66FC10EA56F000188EC2FF0080E0401A8
:10E1D000ED6FFA0E0801D16F00010AEC29F004017D
:10E1E000ED2FF7D7F2CFEDF4F29EAA6A110EA96EC9
:10E1F000A69CA69EA680A850EDBFF28ED76FD7A191
:10E2000018D0D791AA6A110EA96ED7C4A8FFA69CF0
:10E21000A69EA684F2CF00F0F29E0F01550EA76EC7
:10E22000AA0EA76EA682A6B2FED7A6940050F2123E
:10E23000040155D10101BFA353D1040EEA6EC10EF2
:10E24000E96EF2CFEDF4F29E000E000129EC23F00E
:10E250000A000900F550EE6E0009FBE10401EDBF74
:10E26000F28E040E0801A66FC10EA56F000188ECA6
:10E270002FF0BDEC36F0670E87EC28F0040E050198
:10E28000256FD90E246F140E266F0001CAEC36F0EC
:10E29000012C34D00401D95145082EE1DA514F0840
:10E2A0002BE1DB514E0828E1040EEA6EC10EE96E47
:10E2B000F2CFEDF4F29E000E000141EC23F00A00D3
:10E2C0000900F550EE6E0009FBE10401EDBFF28E8E
:10E2D000040E0801A66FC10EA56F000188EC2FF097
:10E2E000080E0401ED6FFA0E0801D16F00010AEC6F
:10E2F00029F00401ED2FF7D7F2D00001F2CFEDF4B1
:10E30000F29EAA6A110EA96EA69CA69EA680A8508F
:10E310000401EDBFF28ED76FD7B1B9D0D781AA6A09
:10E32000110EA96ED7C4A8FFA69CA69EA684F2CF04
:10E3300000F0F29E0F01550EA76EAA0EA76EA682E0
:10E34000A6B2FED7A6940050F212040EEA6EC10ED9
:10E35000E96EF2CFEDF4F29E000E000159EC23F0CD
:10E360000A000900F550EE6E0009FBE10401EDBF63
:10E37000F28E040E0801A66FC10EA56F000188EC95
:10E380002FF0280E0401ED6FFA0E0801D16F000185
:10E390000AEC29F00401ED2FF7D7040EEA6EC10E46
:10E3A000E96EF2CFEDF4F29E000E000171EC23F065
:10E3B0000A000900F550EE6E0009FBE10401EDBF13
:10E3C000F28E040E0801A66FC10EA56F000188EC45
:10E3D0002FF0280E0401ED6FFA0E0801D16F000135
:10E3E0000AEC29F00401ED2FF7D7040EEA6EC10EF6
:10E3F000E96EF2CFEDF4F29E000E000189EC23F0FD
:10E400000A000900F550EE6E0009FBE10401EDBFC2
:10E41000F28E040E0801A66FC10EA56F000188ECF4
:10E420002FF0280E0401ED6FFA0E0801D16F0001E4
:10E430000AEC29F00401ED2FF7D7040EEA6EC10EA5
:10E44000E96EF2CFEDF4F29E000E0001A1EC23F094
:10E450000A000900F550EE6E0009FBE10401EDBF72
:10E46000F28E040E0801A66FC10EA56F000188ECA4
:10E470002FF0040E0401ED6FFA0E0801D16F0001B8
:10E480000AEC29F00401ED2FF7D7FF0028D0040E85
:10E49000EA6EC10EE96EF2CFEDF4F29E000E0001BD
:10E4A000B9EC23F00A000900F550EE6E0009FBE11B
:10E4B0000401EDBFF28E040E0801A66FC10EA56F18
:10E4C000000188EC2FF0080E0401ED6FFA0E080130
:10E4D000D16F00010AEC29F00401ED2FF7D70101FB
:10E4E000BFB102D0BFA329D0F2CFEDF4F29EAA6A49
:10E4F000110EA96EA69CA69EA680A8500401EDBF91
:10E50000F28ED76FD7A118D0D791AA6A110EA96E33
:10E51000D7C4A8FFA69CA69EA684F2CF00F0F29EC8
:10E520000F01550EA76EAA0EA76EA682A6B2FED741
:10E53000A6940050F21204010101040EEA6EC10E0D
:10E54000E96EF2CFEDF4F29E000E0001C3EC20F074
:10E550000A000900F550EE6E0009FBE10401EDBF71
:10E56000F28E040E0801A66FC10EA56F000188ECA3
:10E570002FF0D7EC6CF0D0EC6DF0640E0801D16F89
:10E5800000010AEC29F00401A791196AF2BE198E64
:10E59000F29E480E0C01EF6F010EF06FA7C4F1FC64
:10E5A0000001F0EC25F019BEF28E0A0E0801D16FC1
:10E5B00000010AEC29F0448AC4C112F2498A01011F
:10E5C000C2A506D0C289010802E1498401D049826E
:10E5D00002010E6B0F6B036A0101C451220F016E21
:10E5E000000E03220150BF0FE96E010E0320EA6EF8
:10E5F000EF50F00B08E0C4C114F24A80C1B303D05D
:10E60000C5C115F24A82050E0801D16F00010AEC5E
:10E6100029F00101C3B701D09D9A0001BDEC36F08D
:10E62000B7EFFFF002010F530BE0080197517F0B8A
:10E6300006E195517F0B03E196517F0B01E0468C7B
:10E640000101D139006E0F0E00160050FF0FF30FBD
:10E6500023E20D0F00014EEF73F095C898F896C8AD
:10E6600099F897C89AF83EEC3CF0010115D095C88E
:10E6700098F896C899F897C89AF86CEC3DF00101A3
:10E680000BD095C898F896C899F897C89AF822ECD4
:10E6900042F0010101D001010001000CF2CF0EF0A7
:10E6A000F29EE824F76AF736C70FF66EE60EF722F9
:10E6B000000EF86EFB6E0A00F550FA6E0800F55079
:10E6C0000EBEF28EF96E5AE65AE65AE65AE65AE657
:10E6D0005AE65AE65AE65AE65AE65AE66EE682E6FE
:10E6E0000401C16BC26BC36B140EC46F180EC56FEF
:10E6F000070EC66FC76B050EC86F060EC96F120EE8
:10E70000CA6F0101D139006E0F0E00160050020AC7
:10E7100000011BE0070A22E0010A29E00E0A30E0AE
:10E72000020A2EE0010A2CE00E0A2AE00C0A28E078
:10E73000070A2FE0010A36E0030A3CE00F0A43E033
:10E74000070A41E0050A49E052D0120E0401C56FE4
:10E750000D0EC46F070EC66FC76B4BD00C0E0401B5
:10E76000C56F0A0EC46F070EC66FC76B42D0100E7E
:10E770000401C56F0C0EC46F070EC66FC76B39D08E
:10E78000180E0401C56F140EC46F070EC66FC76B59
:10E7900030D0180E0401C56F080EC46F070EC66F87
:10E7A000C76B27D0180E0401C56F140EC46F070E77
:10E7B000C66F1FD0140E0401C56F0C0EC46F070E78
:10E7C000C66FC76B16D0180E0401C56F140EC46F48
:10E7D000070EC66F020EC76F0CD0100E0401C56F76
:10E7E0000A0EC46F070EC66FC76B03D00001E8D1D5
:10E7F0000401C5510101CD5D02E2CDC1C5F40401A2
:10E80000C4510101CE5D02E2CEC1C4F4196AF2BE68
:10E81000198EF29E7F0E0C01E66FC5C4E7FC000165
:10E82000CAEC24F019BEF28E01C0C8F4196AF2BE17
:10E83000198EF29E7F0E0C01E66FC4C4E7FC000146
:10E84000CAEC24F019BEF28E01C0C9F4196AF2BEF6
:10E85000198EF29E7F0E0C01E66FC6C4E7FC000124
:10E86000CAEC24F019BEF28E01C0CAF40101D139FC
:10E87000006E0F0E001600500A08D8B4F2D0D890DF
:10E88000CF31FF0A800FBE533AE1BD5D38E2800E02
:10E89000D880BD550401CB6FD8900101CF31040160
:10E8A000CB5DCC6F196AF2BE198EF29EE8CFE6FC02
:10E8B000C8C4E7FC0001CAEC24F019BEF28E01C006
:10E8C000C2F40401C251C55D03E2C5C4C2F404D060
:10E8D000C25302E1010EC26FC8C100F002010E5125
:10E8E000016E04E0D8900032012EFCD700A003D0C6
:10E8F0000401C29F02D00401C28F3ED00101D89012
:10E90000CF317F0FBE5303E1BD5D37E036E3800EAC
:10E91000BD5D0401CB6FD8900101CF310401CB5D07
:10E92000CC6F196AF2BE198EF29EE8CFE6FCC8C41D
:10E93000E7FC0001CAEC24F019BEF28E01C0C2F45B
:10E940000401C251C55D03E2C5C4C2F404D0C25380
:10E9500002E1010EC26FC8C100F002010E51016E4A
:10E9600004E0D8900032012EFCD700A003D00401AF
:10E97000C28F02D00401C29F01017F0ED880CF5503
:10E98000BC5336E1BB5D34E2800ED880BB55D880E5
:10E99000CF550401CC6F196AF2BE198EF29EE8CFF2
:10E9A000E6FCC9C4E7FC0001CAEC24F019BEF28EF3
:10E9B00001C0C1F40401C151C45D03E2C4C4C1F487
:10E9C00004D0C15302E1010EC16FC9C100F00201C0
:10E9D0000E51016E04E0D8900032012EFCD700A049
:10E9E00003D00401C18F02D00401C19F39D00101BD
:10E9F0007F0ECF25BC5303E1BB5D33E032E3800ED5
:10EA0000BB5DD880CF550401CC6F196AF2BE198E58
:10EA1000F29EE8CFE6FCC9C4E7FC0001CAEC24F092
:10EA200019BEF28E01C0C1F40401C151C45D03E2FC
:10EA3000C4C4C1F404D0C15302E1010EC16FC9C105
:10EA400000F002010E51016E04E0D8900032012E58
:10EA5000FCD700A003D00401C19F02D00401C18FE4
:10EA60000101D890CF31FF0A800FBA5343E1B95D5D
:10EA700041E2800ED880B9550401CB6FD8900101D6
:10EA8000CF310401CB5DCC6F196AF2BE198EF29EB4
:10EA9000E8CFE6FCCAC4E7FC0001CAEC24F019BECA
:10EAA000F28E01C0C3F40401C351C65D03E2C6C4C3
:10EAB000C3F405D0C351C75D02E3C7C4C3F4010169
:10EAC000D139006E0F0E001600500D0804E004014D
:10EAD000C38706D001010401C35302E1010EC36FD5
:10EAE0000101C3A303D00401C38F02D00401C39F5B
:10EAF00047D00101D890CF317F0FBA5303E1B95D00
:10EB000040E03FE3800EB95D0401CB6FD890010176
:10EB1000CF310401CB5DCC6F196AF2BE198EF29E23
:10EB2000E8CFE6FCCAC4E7FC0001CAEC24F019BE39
:10EB3000F28E01C0C3F40401C351C65D03E2C6C432
:10EB4000C3F405D0C351C75D02E3C7C4C3F40101D8
:10EB5000D139006E0F0E001600500D0804E00401BC
:10EB6000C38706D001010401C35302E1010EC36F44
:10EB70000101C3A303D00401C39F02D00401C38FCA
:10EB80000101A9510401C35D0DE10101AA51040174
:10EB9000C25D08E10101AB510401C15D03E1000167
:10EBA0000FD00401C3C4A9F1C2C4AAF1C1C4ABF11E
:10EBB000C2C495F8C1C496F8C3C497F8000132DD09
:10EBC000BFEFFFF00401C36BC491C493196AF2BE96
:10EBD000198EF29E460E0C01E66FE76B000163ECA6
:10EBE00024F019BEF28E02C0C2F401C0C1F4FF0EBF
:10EBF0000401C11BC21BC2C492F4C1C491F4A7A1F9
:10EC000007D0C1518008D8A4B4D0C253D8A4B1D081
:10EC1000C1C400F0C251036E05E100520001D8B436
:10EC200078D00401035006E1010E005C0001D8B465
:10EC300078D00401200E035C05E100520001D8B435
:10EC400075D00401035006E1020E005C0001D8B447
:10EC500072D00401020E035C05E100520001D8B439
:10EC60006AD00401040E035C05E100520001D8B42F
:10EC700062D00401080E035C05E100520001D8B423
:10EC80005AD00401400E035C04E10052000153E03D
:10EC90000401800E035C04E1005200014CE0040119
:10ECA000035005E1400E005C000149E004010350FF
:10ECB00005E1200E005C000142E00401035005E183
:10ECC000800E005C000141E00401035005E1040EE8
:10ECD000005C00013AE00401035005E1080E005C0D
:10ECE000000133E00401035005E1100E005C000157
:10ECF0002CE00401010E035C04E10052000125E058
:10ED00000401100E035C04E1005200011EE0040146
:10ED10001ED05BB402D05BA601D0468A5B945B96A2
:10ED200027D00401C4815B84000122D00401C48186
:10ED30005B8600011DD00401C481000119D0606B05
:10ED40005B980401C491000113D00401C48158B43C
:10ED500006D045BA04D058BE02D05BA007D05B9065
:10ED6000589E459A58A402D044805886000100D08D
:10ED70000401C4A105D0C3C493F4938F5B9A4CD013
:10ED80008EC492F48DC491F40101C2A146D0040155
:10ED9000C15302E1C25340E0C4B33ED0C151FF0AA7
:10EDA000C56FC251FF0AC66FC76BC75100013CEC6B
:10EDB0001FF00401C72B000187EC28F0100E04019E
:10EDC000C75DF3E1C6C4D5F8370E0801D66F000160
:10EDD0002BEC33F0C5C4D5F8370E0801D66F00010F
:10EDE0002BEC33F0200E87EC28F0C2C4D5F8370E98
:10EDF0000801D66F00012BEC33F0C1C4D5F8370EF3
:10EE00000801D66F00012BEC33F00A0E87EC28F0D6
:10EE10000D0E87EC28F0040101010001E4EFB2F0CF
:10EE20000401F56B010EF56FF55106081CE3F5C4FE
:10EE30000BF50001E3EC44F00401F42D09D00E0EB3
:10EE400005016A6F010E6B6F0001DCEC58F008D011
:10EE50000D0E05016A6F010E6B6F0001DCEC58F0BE
:10EE60000401F52BE1D700014CEF78F00401F46BBD
:10EE7000F46BF451020821E3036AF451C30FE96E05
:10EE8000030E0320EA6EEF6A036AF451C70F016EA6
:10EE9000030E032203C0F6F4036AF451CF0FE96EA8
:10EEA000030E0320EA6EEFCFF7F4F6C4EAFF01C0C9
:10EEB000E9FFF7C4EFFFF42BDCD7F56B00011CEC86
:10EEC0002CF00301C26B01016793679567970401FA
:10EED000636B63C465F465C464F4036A0301C251DF
:10EEE000C70FE96E030E0320EA6EEFCFF5F4F5C409
:10EEF000F6F4130E0401F76F00013AEC6DF04DEFDC
:10EF000078F00401DE6BDF6BDD2D21D0A7A11ED0D0
:10EF1000040EEA6EE00EE96EF2CFF4F4F29E000EFB
:10EF20000001D1EC23F00A000900F550EE6E000953
:10EF3000FBE10401F4BFF28E040E0801A66FE00E9F
:10EF4000A56F000188EC2FF0FF000401ABD0DD536A
:10EF5000D8A4A8D0A7B1A6D00301C26B036AC2513E
:10EF6000C30FE96E030E0320EA6E010EEF6E040E6E
:10EF7000EA6EE00EE96EF2CFF4F4F29E000E0001AC
:10EF800018EC20F00A000900F550EE6E0009FBE1D4
:10EF90000401F4BFF28E040E0801CE6FE00ECD6FB7
:10EFA00000012EEC2AF0040EEA6EE00EE96EF2CFBC
:10EFB000F4F4F29E000EE9EC23F00A000900F5508B
:10EFC000EE6E0009FBE10401F4BFF28E040E0801AD
:10EFD000CE6FE00ECD6F00012EEC2AF0FF0E040183
:10EFE000A66FA56FA76FA96FA86F196AF2BE198ED9
:10EFF000F29E480E0C01EF6F010EF06FA7C4F1FCFA
:10F000000001F0EC25F019BEF28E196AF2BE198EDD
:10F01000F29E4C0E0C01E86FE96BA6C4EBFCA5C494
:10F02000EAFC00011CEC26F019BEF28E196AF2BE51
:10F03000198EF29E4A0E0C01E86FE96BA9C4EBFC35
:10F04000A8C4EAFC00011CEC26F019BEF28E0101F6
:10F05000C2A705D0800E0401DE17DF6B05D07F0E3E
:10F060000401DE13FF0EDF13196AF2BE198EF29E41
:10F07000400E0C01E86FE96BDFC4EBFCDEC4EAFC78
:10F0800000011CEC26F019BEF28EBE6A9D90010EA6
:10F090000401F46F0001C4D6E9D60101BF5301E0B9
:10F0A0009D9A04010001000C0401DD6BDE6B020E71
:10F0B0000301C75DF00FD8B037D1100F000197EFF3
:10F0C00079F0040163530CE1448CCFC3C7F3036AA6
:10F0D0000301C251C30FE96E030E0320EA6EEF6A0B
:10F0E000030122D10401632D04D00101C18B03D09F
:10F0F00004010101C19B448E030116D10401635137
:10F100000101C45D03E063C4C4F1448E03010CD16A
:10F11000040163510101C55D03E063C4C5F1448E80
:10F12000030102D1040163510101C75D03E063C41F
:10F13000C7F1448E0301F8D00401635305E10101D6
:10F14000C395448E06D00401632D03D00101C3850D
:10F15000448E0301E9D0040163510101C65D03E05F
:10F1600063C4C6F1448E0301DFD00401635305E19B
:10F170000101C391448E06D00401632D03D0010127
:10F18000C381448E0301D0D0040163510101CC5DE1
:10F1900004E063C4CCF1448E07D0CC51030DF3CF0F
:10F1A000DFF40401DFC4BEFF0301BED004016351DC
:10F1B0000101CB5D03E063C4CBF1448E0301B4D005
:10F1C0000401635305E10101C393448E06D0040199
:10F1D000632D03D00101C383448E0301A5D0010137
:10F1E000BF6BC06B0401632D04D00101BF812CD023
:10F1F00004016351020804E10101BF8325D0040129
:10F200006351030805E10101BF85C0831DD00401DE
:10F210006351040805E10101BF85C08515D00401D3
:10F220006351050805E10101BF85C0810DD00401CE
:10F230006351060804E10101BF8706D00401635150
:10F24000070803E10101BF890401635304E00101E0
:10F25000C293C2910401448E030166D0196AF2BEC2
:10F26000198EF29E400E0C01E66FE76B000163EC15
:10F2700024F019BEF28E02C0DEF401C0DDF40401F8
:10F28000635307E1800EDD17DE6B0101C29709D0E1
:10F290000401632D07D07F0EDD13FF0EDE13010185
:10F2A000C2870401196AF2BE198EF29E400E0C014B
:10F2B000E86FE96BDEC4EBFCDDC4EAFC00011CEC8A
:10F2C00026F019BEF28E448E03012ED00401635144
:10F2D0000101CD5D03E063C4CDF1448E030124D070
:10F2E000040163510101CE5D03E063C4CEF1448E9D
:10F2F00003011AD004016351010A000105E0030A69
:10F3000007E0020A09E008D00101C38BC39D08D0C1
:10F310000101C38DC39B04D00101C39BC39D00D0D9
:10F32000448E030101D00301030145EF7BF0F2CFCE
:10F330000EF0F29EE824F76AF736590FF66EF30ED8
:10F34000F722000EF86EFB6E0A00F550FA6E080008
:10F35000F5500EBEF28EF96EC2F0E4F0FCF010F142
:10F36000CCF2E0F224F138F156F16AF1C0F188F103
:10F37000F4F2DEF1ACF15CF2010E0301C85DF90FAD
:10F3800052E2070F000116EF7AF00401635305E122
:10F390000101C387458E06D00401632D04D001010D
:10F3A000C397458E0401448E03013DD0040163538D
:10F3B00004E10101C38905D00401632D03D00101DB
:10F3C000C3990401448E03012ED00401635301E16B
:10F3D0004582030128D00401635301E14584030100
:10F3E00022D00401632D03D00101C28302D00101A8
:10F3F000C293448E030117D00401632D03D0010191
:10F40000C18302D00101C193448E03010CD00401D9
:10F41000632D03D00101C18902D00101C199448E3D
:10F42000030101D00301030145EF7BF0F2CF0EF0A1
:10F43000F29EE824F76AF736570FF66EF40EF722BD
:10F44000000EF86EFB6E0A00F550FA6E0800F550DB
:10F450000EBEF28EF96E8AF3ACF3CAF3D6F3E2F382
:10F46000F8F30EF40401DD6B036A0301C251C70F08
:10F47000E96E030E0320EA6E010EEF5CF90FD8B0BF
:10F4800079D0070F0001BDEF7AF00401DD2B0001F8
:10F490000401DD2B00010401DD2B00010401DD2B43
:10F4A00000010401DD2B00010401DD2B000104013A
:10F4B00063532FE10301C251020815E10401DD533A
:10F4C00004E10101C86B0ED00401010E006EDD5194
:10F4D000016E04E0D8900036012EFCD70050FF0AE0
:10F4E0000101C81714D00401DD5304E10101C96B07
:10F4F0000ED00401010E006EDD51016E04E0D890C3
:10F500000036012EFCD70050FF0A0101C9172ED08A
:10F5100004010301C251020815E10401DD5305E1B4
:10F52000FF0E0101C86F0DD00401010E006EDD5108
:10F53000016E04E0D8900036012EFCD70050010186
:10F54000C81314D00401DD5305E1FF0E0101C96F9A
:10F550000DD00401010E006EDD51016E04E0D89063
:10F560000036012EFCD700500101C913448E03015F
:10F5700001D00301030145EF7BF0F2CF0EF0F29EC4
:10F58000E824F76AF736A50FF66EF50EF722000E9F
:10F59000F86EFB6E0A00F550FA6E0800F5500EBECC
:10F5A000F28EF96EAEF4A8F4A2F49CF496F490F402
:10F5B0008AF4036A0301C251C30FE96E030E0320EC
:10F5C000EA6EEF5002081EE1036AC251C70FE96EEE
:10F5D000030E0320EA6E010EEF5C0401DE6F036A86
:10F5E0000301C251C70FE96E030E0320EA6EEFCF8D
:10F5F000DFF4DEC4F6F4DFC4F7F400013AEC6DF09A
:10F600001BD00301036AC251C70FE96E030E03202A
:10F61000EA6EEFCFDEF4036AC251C70FE96E030E44
:10F620000320EA6E010EEF240401DF6FDEC4F6F45E
:10F63000F76F00013AEC6DF0000C010167936795DC
:10F6400067970401636B63C465F465C464F4FF0EDB
:10F65000636F0301C2530BE1C7510D0808E10101BB
:10F66000CC51030DF3CFDEF40401DEC4BEFF000174
:10F67000A0DF000C0301C251FC0F07E2040F0001E0
:10F6800049EF7BF011D578D6EDD60001D6DF99EFA2
:10F690007FF0F2CF0EF0F29EE824F76AF736BD0F46
:10F6A000F66EF60EF722000EF86EFB6E0A00F550AD
:10F6B000FA6E0800F5500EBEF28EF96E84F686F6EC
:10F6C00088F688F6010167B33CD00301C25324E1F8
:10F6D000036AC251C30FE96E030E0320EA6EEF6A9C
:10F6E000036AC251C70F016E030E0322040103C057
:10F6F000DEF4036A0301C251CF0FE96E030E03204B
:10F70000EA6EEFCFDFF40401DEC4EAFF01C0E9FFD7
:10F71000DFC4EFFF13D00301036AC251C30FE96EC8
:10F72000030E0320EA6E020EEF6E036AC251C70F8A
:10F73000E96E030E0320EA6E010EEF6E000139DF61
:10F7400002D000017ADF000C0301C751120A000148
:10F750002FE0100A49E0010A60E00A0AD8B490D00C
:10F76000020AD8B4A9D0070AD8B4C2D0030AD8B4C0
:10F77000F3D0010AD8B4CAD11F0AD8B417D2170AD5
:10F78000D8B448D2010AD8B445D2030AD8B458D262
:10F79000010AD8B460D20D0AD8B468D2020AD8B42B
:10F7A00070D2070AD8B478D21D0AD8B47FD289D2D1
:10F7B000010E0401F56F00011CEC2CF0036A03013B
:10F7C000C251C70FE96E030E0320EA6E010EEF6E01
:10F7D000036AC251C30FE96E030E0320EA6E020EE4
:10F7E000EF6E00016FDF74D2030EEA6ED30EE96E86
:10F7F000F2CFDDF4F29E000E11EC0BF00A000900CE
:10F80000F550EE6E0009FBE10401DDBFF28E646B82
:10F81000636B63C465F400015BD2030EEA6ED30E22
:10F82000E96EF2CFDDF4F29E000E26EC0BF00A003A
:10F830000900F550EE6E0009FBE10401DDBFF28E18
:10F84000030EEA6EE50EE96EF2CFDDF4F29E000ED5
:10F8500000013BEC0BF00A000900F550EE6E0009C8
:10F86000FBE10401DDBFF28E010E646F656B636B1B
:10F870000101C1AB03D00401632B0101000128D2B7
:10F88000020E0401F56F00011CEC2CF0036A030169
:10F89000C251C70FE96E030E0320EA6E010EEF6E30
:10F8A000036AC251C30FE96E030E0320EA6E020E13
:10F8B000EF6E000107DF0CD2030E0401F56F0001AB
:10F8C0001CEC2CF0036A0301C251C70FE96E030E52
:10F8D0000320EA6E010EEF6E036AC251C30FE96E98
:10F8E000030E0320EA6E020EEF6E0001EBDEF0D194
:10F8F000030EEA6ED30EE96EF2CFDDF4F29E000E37
:10F9000050EC0BF00A000900F550EE6E0009FBE127
:10F910000401DDBFF28E030EEA6EE50EE96EF2CF52
:10F92000DDF4F29E000E000166EC0BF00A00090007
:10F93000F550EE6E0009FBE10401DDBFF28E636B52
:10F940000101C3A303D00401632B0101010E0401D3
:10F95000646F656B0001BCD1030EEA6ED30EE96ED5
:10F96000F2CFDDF4F29E000E7CEC0BF00A000900F1
:10F97000F550EE6E0009FBE10401DDBFF28E030ECF
:10F98000EA6EE50EE96EF2CFDDF4F29E000E0001A4
:10F9900093EC0BF00A000900F550EE6E0009FBE154
:10F9A0000401DDBFF28E030EEA6EF70EE96EF2CFB0
:10F9B000DDF4F29E000E0001AAEC0BF00A00090033
:10F9C000F550EE6E0009FBE10401DDBFF28E040E7E
:10F9D000EA6E090EE96EF2CFDDF4F29E000E000130
:10F9E000C1EC0BF00A000900F550EE6E0009FBE1D6
:10F9F0000401DDBFF28E040EEA6E1B0EE96EF2CF3B
:10FA0000DDF4F29E000E0001D8EC0BF00A000900B4
:10FA1000F550EE6E0009FBE10401DDBFF28E040E2D
:10FA2000EA6E2D0EE96EF2CFDDF4F29E000E0001BB
:10FA3000EFEC0BF00A000900F550EE6E0009FBE157
:10FA40000401DDBFF28E040EEA6E3F0EE96EF2CFC6
:10FA5000DDF4F29E000E000106EC0CF00A00090035
:10FA6000F550EE6E0009FBE10401DDBFF28E040EDD
:10FA7000EA6E510EE96EF2CFDDF4F29E000E000147
:10FA80001DEC0CF00A000900F550EE6E0009FBE1D8
:10FA90000401DDBFF28E0101BFA105D0010E0401FA
:10FAA000636F2ED00101BFA305D0020E0401636F66
:10FAB00027D00101BFA515D0C0A305D0030E0401B6
:10FAC000636F0DD00101C0A505D0040E0401636F62
:10FAD00006D00101C0A104D0050E0401636F01012D
:10FAE0000FD0BFA705D0060E0401636F09D0010136
:10FAF000BFA904D0070E0401636F02D00401636B39
:10FB0000060E0401646F656B0001E2D0030EEA6E1D
:10FB1000D30EE96EF2CFDDF4F29E000E34EC0CF061
:10FB20000A000900F550EE6E0009FBE10401DDBF9B
:10FB3000F28E030EEA6EE50EE96EF2CFDDF4F29E70
:10FB4000000E00014AEC0CF00A000900F550EE6EC0
:10FB50000009FBE10401DDBFF28E030EEA6EF70E31
:10FB6000E96EF2CFDDF4F29E000E000162EC0CF0C3
:10FB70000A000900F550EE6E0009FBE10401DDBF4B
:10FB8000F28E0101C3AB05D0010E0401636F09D0F1
:10FB90000101C3AD04D0020E0401636F02D0040161
:10FBA000636B020E646F656B000192D0030EEA6E08
:10FBB000D30EE96EF2CFDDF4F29E000E7AEC0CF07B
:10FBC0000A000900F550EE6E0009FBE10401DDBFFB
:10FBD000F28E030EEA6EE50EE96EF2CFDDF4F29ED0
:10FBE000000E000191EC0CF00A000900F550EE6ED9
:10FBF0000009FBE10401DDBFF28E636B0101C2A7C6
:10FC000003D00401632B0101010E0401646F656BD5
:10FC100000015ED001016785180E0401646F010EBA
:10FC2000656F0301C751060A000103E0010A04E001
:10FC300006D0CDC163F403D0CEC163F400D048D068
:10FC400001016785060E0401646FC4C163F4010EEF
:10FC5000656F00013DD0010167850C0E0401646FE2
:10FC6000C5C163F4010E656F000132D001016785E3
:10FC7000180E0401646F010E656FC7C163F40001C3
:10FC800027D001016785140E0401646F010E656FB2
:10FC9000C6C163F400011CD001016785320E040166
:10FCA000646F656BCCC163F4000112D001016785FC
:10FCB0006787280E0401646F656BCBC163F4000194
:10FCC00007D001016793679567976797000100D098
:10FCD000AFEF7FF00301C851030A000112E0070AE9
:10FCE00010E0010A26E0040A57E0030A55E0040A7E
:10FCF000D8B4A3D0010AD8B4D3D00F0AD8B403D152
:10FD000009D1030EEA6ED30EE96EF2CFDDF4F29E56
:10FD1000000E11EC0BF00A000900F550EE6E000920
:10FD2000FBE10401DDBFF28E646B636B63C465F4B9
:10FD3000F7D0030EEA6ED30EE96EF2CFDDF4F29E39
:10FD4000000E26EC0BF00A000900F550EE6E0009DB
:10FD5000FBE10401DDBFF28E030EEA6EE50EE96EF3
:10FD6000F2CFDDF4F29E000E00013BEC0BF00A0036
:10FD70000900F550EE6E0009FBE10401DDBFF28ED3
:10FD8000010E646F656B636B0101C2A303D00401B4
:10FD9000632B01010401C4D0030EEA6ED30EE96E99
:10FDA000F2CFDDF4F29E000EA8EC0CF00A00090080
:10FDB000F550EE6E0009FBE10401DDBFF28E030E8B
:10FDC000EA6EE50EE96EF2CFDDF4F29E000E000160
:10FDD000BDEC0CF00A000900F550EE6E0009FBE1E5
:10FDE0000401DDBFF28E036A0301C251C70FE96E41
:10FDF000030E0320EA6EEF50010A000103E0030A3C
:10FE00000AE012D00401636B0101C3B703D00401FF
:10FE1000632B01010DD00401636B0101C3B903D051
:10FE20000401632B010104D00401636B010100D0C4
:10FE3000010E0401646F656B73D0030EEA6ED30E7E
:10FE4000E96EF2CFDDF4F29E000ED2EC0CF00A0067
:10FE50000900F550EE6E0009FBE10401DDBFF28EF2
:10FE6000030EEA6EE50EE96EF2CFDDF4F29E000EAF
:10FE70000001EAEC0CF00A000900F550EE6E0009F2
:10FE8000FBE10401DDBFF28E010E646F656B636BF5
:10FE90000101C1A303D00401632B0101040140D07F
:10FEA000030EEA6ED30EE96EF2CFDDF4F29E000E81
:10FEB00002EC0DF00A000900F550EE6E0009FBE1BE
:10FEC0000401DDBFF28E030EEA6EE50EE96EF2CF9D
:10FED000DDF4F29E000E00011AEC0DF00A0009009C
:10FEE000F550EE6E0009FBE10401DDBFF28E010E5C
:10FEF000646F656B636B0101C1A903D00401632BBF
:10FF0000010104010DD00401F56B00011CEC2CF083
:10FF10001DEC7BF00101679367956797040100D0A2
:10FF20000001AFEF7FF0010167A305D000013AEFB8
:10FF30007BF01CD0010167830301C251000107E07F
:10FF4000010A07E0030A06E0010A04E004D0A4EF76
:10FF50007BF0C0D655D001016793000100D00101AC
:10FF600067A305D063C4E0F40001C4DA0101040111
:10FF7000FFEF8DF004016551635D03E1010E64251F
:10FF8000636F63070301C2530AE1C7510D0807E11C
:10FF900004016351030DF3CFE0F4E0C4BEFF63C47A
:10FFA000E0F40001A7DA56EF83F004016451635DC9
:10FFB00003E1010E655D636F632B0301C2530AE128
:10FFC000C7510D0807E104016351030DF3CFE0F4BD
:10FFD000E0C4BEFF63C4E0F400018CDA81EF84F07A
:10FFE000036A6151680FE96E000E0320EA6EEFCFDD
:0EFFF000C2F40401C2C401F000019CEFFAF05B
:020000040001F9
:100000000401DD6B030EEA6ED30EE96EF2CFDEF46F
:10001000F29E000E000150EC0BF00A000900F550B2
:10002000EE6E0009D8A40EEF80F00401DEBFF28E60
:10003000030EEA6EE50EE96EF2CFDEF4F29E000EDC
:10004000000166EC0BF00A000900F550EE6E0009A5
:10005000D8A424EF80F00401DEBFF28E010E646F9D
:10006000656B036A0301C251C70FE96E030E0320DB
:10007000EA6EEF50070A0001D8B45DEF80F0010A84
:10008000D8B460EF80F0030AD8B463EF80F0010ABF
:10009000D8B466EF80F0070AD8B469EF80F0010A9F
:1000A000D8B46CEF80F0030AD8B46FEF80F0090A7F
:1000B000D8B4A7EF80F0AEEF80F00401DD2B000193
:1000C0000401DD2B00010401DD2B00010401DD2B07
:1000D00000010401DD2B00010401DD2B00010401FE
:1000E000DD53D8A475EF80F0DD2B0301C251020867
:1000F000D8A48EEF80F0C8C100F00401DD51016E7C
:10010000D8B488EF80F0D8900032012E83EF80F0D1
:10011000636B00B0632BA3EF80F00301C2510308AF
:10012000D8A4A3EF80F0C9C100F00401DD51016E35
:10013000D8B4A0EF80F0D8900032012E9BEF80F071
:10014000636B00B0632B01016783B4EF80F004019F
:10015000F56B00011CEC2CF01DEC7BF001016793AA
:1001600067956797B4EF80F00001AFEF7FF005016E
:100170000751F00B006E003A0F0E00160050000100
:10018000D8B4D9EF80F0010AD8B413EF81F0030A94
:10019000D8B46BEF81F0010AD8B4A6EF81F0070A5A
:1001A000D8B4F8EF81F0010AD8B42DEF82F062EFF5
:1001B00082F0050107510F0B0908D8A0F6EF80F077
:1001C000010E085D036A0925E96E0A510320EA6EF3
:1001D000300EEF6E036A08510925E96E0A510320BB
:1001E000EA6E07513009EF6E11EF81F007510F0BE6
:1001F0000F08D8A011EF81F0010E085D036A0925F0
:10020000E96E0A510320EA6E310EEF6E036A08515F
:100210000925E96E0A510320EA6E0A0E075D3009CE
:10022000EF6E78EF82F0050107510F0B0308D8A09D
:1002300031EF81F0010E085D036A0925E96E0A516C
:100240000320EA6E310EEF6E036A08510925E96E4C
:100250000A510320EA6E0A0E075D3009EF6E69EF5E
:1002600081F007510F0B0D08D8A04EEF81F0010E61
:10027000085D036A0925E96E0A510320EA6E320E11
:10028000EF6E036A08510925E96E0A510320EA6EF0
:10029000140E075D3009EF6E69EF81F007510F0B07
:1002A0000F08D8A069EF81F0010E085D036A0925E7
:1002B000E96E0A510320EA6E330EEF6E036A0851AD
:1002C0000925E96E0A510320EA6E1E0E075D30090A
:1002D000EF6E78EF82F0050107510F0B0708D8A0E9
:1002E00089EF81F0010E085D036A0925E96E0A5164
:1002F0000320EA6E330EEF6E036A08510925E96E9A
:100300000A510320EA6E1E0E075D3009EF6EA4EF5E
:1003100081F007510F0B0F08D8A0A4EF81F0010E58
:10032000085D036A0925E96E0A510320EA6E340E5E
:10033000EF6E036A08510925E96E0A510320EA6E3F
:10034000280E075D3009EF6E78EF82F00501075146
:100350000F0B0108D8A0C4EF81F0010E085D036AFD
:100360000925E96E0A510320EA6E340EEF6E036A26
:1003700008510925E96E0A510320EA6E280E075D2F
:100380003009EF6EF6EF81F007510F0B0B08D8A084
:10039000E1EF81F0010E085D036A0925E96E0A515B
:1003A0000320EA6E350EEF6E036A08510925E96EE7
:1003B0000A510320EA6E320E075D3009EF6EF6EF48
:1003C00081F0010E085D036A0925E96E0A510320D8
:1003D000EA6E360EEF6E036A08510925E96E0A517E
:1003E0000320EA6E3C0E075D3009EF6E78EF82F075
:1003F000050107510F0B0508D8A016EF82F0010E7A
:10040000085D036A0925E96E0A510320EA6E360E7B
:10041000EF6E036A08510925E96E0A510320EA6E5E
:100420003C0E075D3009EF6E2BEF82F0010E085D88
:10043000036A0925E96E0A510320EA6E370EEF6E52
:10044000036A08510925E96E0A510320EA6E460E37
:10045000075D3009EF6E78EF82F0050107510F0B51
:100460000908D8A04BEF82F0010E085D036A092548
:10047000E96E0A510320EA6E380EEF6E036A0851E6
:100480000925E96E0A510320EA6E500E075D300916
:10049000EF6E60EF82F0010E085D036A0925E96ED8
:1004A0000A510320EA6E390EEF6E036A08510925DE
:1004B000E96E0A510320EA6E5A0E075D3009EF6EAD
:1004C00078EF82F0010E0501085D036A0925E96EE7
:1004D0000A510320EA6E450EEF6E036A08510925A2
:1004E000E96E0A510320EA6E450EEF6E78EF82F056
:1004F0000001000C040EEA6EE10EE96E0801CD6BFE
:10050000CF6B130ECE6F00013AEC2FF0040EEA6EA3
:10051000F40EE96E0801CD6BCF6B130ECE6F0001A8
:100520003AEC2FF0036A0301C251C70FE96E030EC4
:100530000320EA6E0C01E06BEFCFDFFCE26B120EE2
:10054000E16F00011AEC33F002C003F001505A0FC2
:10055000016E020E032201C007F503C008F5040E68
:100560000801CE6FE10ECD6F03C0D0F801C0CFF807
:10057000120ED16F000149EC2FF00C0E0401E16F57
:10058000040E0801CE6FE10ECD6F00012EEC2AF0B3
:10059000050E0801D46F00011FEC29F0010167B5B9
:1005A000F0EF82F00401E051120DF350036AD30F13
:1005B000016E030E032201C007F503C008F5040E07
:1005C0000801CE6FF40ECD6F03C0D0F801C0CFF894
:1005D000120ED16F000149EC2FF036EF83F00101CC
:1005E00067B710EF83F0040EEA6EF40EE96E200E8A
:1005F0000801CD6FCF6B090ECE6F00013AEC2FF0E2
:10060000E0C407F5090E0501086F040E0A6FF40E29
:10061000096F0001ACDD0401FE6B36EF83F00101D0
:10062000040EEA6EF40EE96E200E0801CD6FCF6B5A
:10063000090ECE6F00013AEC2FF0E0C407F5090E69
:100640000501086F040E0A6FF40E096F00018FDDBB
:10065000730E0401FF6F650E0501006F630E016FDD
:10066000026BFDC4FEF42E0E0401FD6F0A0E0401A0
:10067000F46F3E0EF56F040E0801CE6FF40ECD6FD1
:1006800000012EEC2AF0000C040EEA6EDD0EE96E7D
:100690000801CD6BCF6B030ECE6F00013AEC2FF04B
:1006A000010167A359EF83F0000164D46CEF84F07B
:1006B0000101036A0301C251C30FE96E030E032057
:1006C000EA6EEF500001D8B470EF83F0010AD8B49D
:1006D000A0EF83F0030AD8B4C0EF83F06CEF84F08E
:1006E000036A0301C251C70FE96E030E0320EA6ECD
:1006F000020EEF6E036AC251C30FE96E030E0320B0
:10070000EA6E010EEF6E036AC251C70FE96E030E67
:100710000320EA6EEFCFE0F4036AC251C70FE96E1F
:10072000030E0320EA6E010EEF240401E16FE0C422
:10073000F6F4E1C4F7F400013AEC6DF06CEF84F0EC
:10074000036A0301C251C70FE96E030E0320EA6E6C
:10075000EF2A036AC251C30FE96E030E0320EA6E4B
:10076000020EEF6E030E0401DD6FDE6B040E080156
:10077000CE6FDD0ECD6F00012EEC2AF06CEF84F011
:10078000036A0301C251C70FE96E030E0320EA6E2C
:10079000EF2A036AC251C70FE96E030E0320EA6E07
:1007A000EFCFE0F4036AC251CB0FE96E030E0320D2
:1007B000EA6EEF500401E05DD8B44DEF84F0D8A0AC
:1007C0004DEF84F00301C253D8A40BEF84F0036A09
:1007D000C251C30FE96E030E0320EA6EEF6A036A8B
:1007E000C251C70F0401E06F030E0320E16F036ADB
:1007F0000301C251CF0FE96E030E0320EA6EEFCF63
:10080000E2F40401E1C4EAFFE0C4E9FFE2C4EFFF5F
:100810002EEF84F00301036AC251C30FE96E030E89
:100820000320EA6E020EEF6E036AC251C70F040185
:10083000E06F030E0320E16F036A0301C251CF0F83
:10084000E96E030E0320EA6E010EEF240401E26F4D
:10085000E1C4EAFFE0C4E9FFE2C4EFFF036A030179
:10086000C251CF0FE96E030E0320EA6EEFCFE0F422
:10087000036AC251CF0FE96E030E0320EA6E010E28
:10088000EF240401E16FE0C4F6F4E1C4F7F40001E1
:100890003AEC6DF06AEF84F00401036A0301C2517F
:1008A000C70FE96E030E0320EA6E010EEF5C040130
:1008B000E06F036A0301C251C70FE96E030E032004
:1008C000EA6EEFCFE1F4E0C4F6F4E1C4F7F400011E
:1008D0003AEC6DF06CEF84F0BBEF88F0040EEA6E3A
:1008E000DD0EE96E0801CD6BCF6B030ECE6F0001FC
:1008F0003AEC2FF0010167A384EF84F00001D5EFFB
:100900007FF00AEF86F00101036A0301C251C30FB1
:10091000E96E030E0320EA6EEF500208D8A430EF10
:1009200085F0036AC251C70FE96E030E0320EA6E19
:10093000EF52D8B430EF85F0036AC251C70FE96EA9
:10094000030E0320EA6EEF06C253D8B4F5EF84F02D
:10095000036AC251C70FE96E030E0320EA6EEF521D
:10096000D8A4F5EF84F0036AC251C30FE96E030EF9
:100970000320EA6E020EEF6E036AC251CB0FE96EDE
:10098000030E0320EA6E010EEF5C0401E06F036AC0
:100990000301C251CB0FE96E030E0320EA6EEFCFC5
:1009A000E1F4E0C4F6F4E1C4F7F400013AEC6DF0D0
:1009B000036A0301C251C70F0401E06F030E032055
:1009C000E16F036A0301C251CB0FE96E030E0320EE
:1009D000EA6EEFCFE2F40401E1C4EAFFE0C4E9FF0C
:1009E000E2C4EFFF2DEF85F00301036AC251C70F88
:1009F000E96E030E0320EA6EEF52D8A417EF85F0DC
:100A0000036AC251C70FE96E030E0320EA6EEF2A94
:100A1000036AC251C30FE96E030E0320EA6EEF6A48
:100A2000010E0401DD6FDE6B24EF85F00301036A24
:100A3000C251C30FE96E030E0320EA6E010EEF6E82
:100A4000020E0401DD6FDE6B040E0801CE6FDD0EB9
:100A5000CD6F00012EEC2AF004010AEF86F00301AD
:100A6000036AC251C70FE96E030E0320EA6EEFCF8F
:100A7000E0F4036AC251CF0FE96E030E0320EA6E61
:100A8000EF500401E05DD8B4CAEF85F0D8A0CAEFFA
:100A900085F0036A0301C251C70FE96E030E0320FC
:100AA000EA6EEF06036AC251C70FE96E030E032018
:100AB000EA6EEF500108D8A0ACEF85F0036AC2518E
:100AC000C70FE96E030E0320EA6EEF06C253D8A4E7
:100AD0007CEF85F0036AC251C30FE96E030E032059
:100AE000EA6EEF6A036AC251C70FE96E030E032074
:100AF000EA6EEF6A8EEF85F0036AC251C70FE96EA6
:100B0000030E0320EA6E010EEF6E036AC251C30F9B
:100B1000E96E030E0320EA6E020EEF6E036AC25105
:100B2000CF0FE96E030E0320EA6EEFCFE0F4036A05
:100B3000C251CF0FE96E030E0320EA6E010EEF24BF
:100B40000401E16FE0C4F6F4E1C4F7F400013AEC0B
:100B50006DF0C7EF85F00301036AC251C70FE96E5C
:100B6000030E0320EA6EEFCFE0F4036AC251C70F11
:100B7000E96E030E0320EA6E010EEF240401E16F1B
:100B8000E0C4F6F4E1C4F7F400013AEC6DF00AEFCA
:100B900086F00401036A0301C251C30FE96E030E1C
:100BA0000320EA6E020EEF6E036AC251CB0FE96EAC
:100BB000030E0320EA6E010EEF5C0401E06F036A8E
:100BC0000301C251CB0FE96E030E0320EA6EEFCF93
:100BD000E1F4E0C4F6F4E1C4F7F400013AEC6DF09E
:100BE000036A0301C251C70F0401E06F030E032023
:100BF000E16F036A0301C251CB0FE96E030E0320BC
:100C0000EA6EEFCFE2F40401E1C4EAFFE0C4E9FFD9
:100C1000E2C4EFFF0401FFEF8DF00401D76BD86B46
:100C2000D96BDA6BDB6BDC91040EEA6EC30EE96EF6
:100C30000801CD6BCF6B140ECE6F00013AEC2FF094
:100C40000101C2A173EF86F00401C1C4E9FFC2C46F
:100C5000EAFFECCFDEF4ED52EFCFDDF4C1C4E9FFE3
:100C6000C2C4EAFFECCFE0F4ED52EFCFDFF4FF0EA9
:100C7000DF1BE01BE16BE151000164EC1CF004019F
:100C8000E12B000187EC28F00C0E0401E15DD8A4F3
:100C90003BEF86F0DEC4D5F8370E0801D66F0001B1
:100CA0002BEC33F0DDC4D5F8370E0801D66F000108
:100CB0002BEC33F0200E87EC28F0E0C4D5F8370E8B
:100CC0000801D66F00012BEC33F0DFC4D5F8370EE6
:100CD0000801D66F00012BEC33F00A0E87EC28F0E8
:100CE0000D0E87EC28F00401C1C4E9FFC2C4EAFF7D
:100CF000ECCF03F0ED52EFCFD7F403C0D8F4C1C46A
:100D0000E9FFC2C4EAFFEFCF00F0E92AEF50E9069D
:100D1000036E0350D8A494EF86F0020E005C00012D
:100D2000D8B43BEF87F004010350D8A49FEF86F0BE
:100D3000040E005C0001D8B40BEF88F004010350EE
:100D4000D8A4AAEF86F0200E005C0001D8B40EEF04
:100D500088F004010350D8A4B5EF86F0400E005C83
:100D60000001D8B411EF88F004010350D8A4C0EFFB
:100D700086F0800E005C0001D8B414EF88F0040106
:100D8000010E035CD8A4CBEF86F000520001D8B46A
:100D9000B7EF88F004010350D8A4D6EF86F0080E10
:100DA000005C0001D8B4B9EF88F004010350D8A466
:100DB000E1EF86F0100E005C0001D8B4BEEF88F0C1
:100DC0000401100E035CD8A4ECEF86F00052000181
:100DD000D8B4C0EF88F00401020E035CD8A4F7EF8A
:100DE00086F000520001D8B4C5EF88F00401040E6B
:100DF000035CD8A402EF87F000520001D8B492EF50
:100E000089F00401080E035CD8A40DEF87F00052AE
:100E10000001D8B45EEF8AF004010350D8A418EFA3
:100E200087F0010E005C0001D8B4FFEF8AF00401E6
:100E3000200E035CD8A423EF87F000520001D8B441
:100E4000C8EF8BF00401400E035CD8A42EEF87F0AE
:100E500000520001D8B493EF8CF00401800E035CC3
:100E6000D8A439EF87F000520001D8B42FEF8DF0ED
:100E70000401FFEF8DF00101D151F00BD8B408EF60
:100E800088F0D151F00BD008D8B4EAEF87F058B011
:100E90004DEF87F058A45BEF87F0588AA09258ACCA
:100EA0005BEF87F0010E0801D16F00010AEC29F019
:100EB00001014FEF87F00401A7B994EF87F0A789EC
:100EC000040EEA6EC30EE96EF2CFDDF4F29E000E60
:100ED00000017EEC1CF00A000900F550EE6E0009DE
:100EE000D8A46CEF87F00401DDBFF28E0101D1912F
:100EF000C2A391EF87F0BF53D8A491EF87F004010C
:100F0000DD6BDD51000196EC1CF00401DD2B0001CE
:100F100087EC28F00A0E0401DD5DD8A481EF87F08C
:100F20000101C6EF87F00401A799040EEA6EC30E13
:100F3000E96EF2CFDDF4F29E000E0001ABEC1CF086
:100F40000A000900F550EE6E0009D8A4A1EF87F061
:100F50000401DDBFF28E0101D181C2A3C6EF87F08B
:100F6000BF53D8A4C6EF87F00401DD6BDD5100014B
:100F7000C3EC1CF00401DD2B000187EC28F0090E06
:100F80000401DD5DD8A4B6EF87F00101196AF2BE55
:100F9000198EF29E480E0C01EF6F010EF06FA7C480
:100FA000F1FC0001F0EC25F019BEF28E040E0801F0
:100FB000A66FC30EA56F000188EC2FF0468058B0D5
:100FC000E5EF87F058A4E7EF87F0589AA08208EF82
:100FD00088F00101040EEA6EC30EE96EF2CFDDF473
:100FE000F29E000E0001D7EC1CF00A000900F5503B
:100FF000EE6E0009D8A4F6EF87F00401DDBFF28E93
:10100000040E0801A66FC30EA56F000188EC2FF037
:101010000401FFEF8DF00401FFEF8DF00401FFEFFD
:101020008DF00401FFEF8DF00401A7B192EF88F07D
:10103000020EC125E96E000EC221EA6EEFCFDDF48B
:10104000000EDDBD010E000AD8A46CEF88F0196A0D
:10105000F2BE198EF29E460E0C01E66FE76B0001A0
:1010600063EC24F019BEF28E02C0DAF401C0D9F4A8
:10107000010E0401DB6FDB516308D8A06CEF88F030
:10108000D951FF0ADD6FDA51FF0ADE6FDD518008AA
:10109000D8A44FEF88F0DE53D8B451EF88F0FFEFBB
:1010A0008DF00A0E0801D16F00010AEC29F0196ACF
:1010B000F2BE198EF29E460E0C01E66FE76B000140
:1010C00063EC24F019BEF28E02C0DAF401C0D9F448
:1010D0000401DB2B3BEF88F00101C2A386EF88F00F
:1010E000BF53D8A486EF88F00401DD6BDD51000109
:1010F000EFEC1CF00401DD2B000187EC28F00C0E56
:101100000401DD5DD8A476EF88F001010401DD6BF8
:10111000000181EC77F08E9097900401FFEF8DF045
:10112000B5EF88F00101C2A3ACEF88F0BF53D8A49B
:10113000ACEF88F00401DD6BDD51000105EC1DF022
:101140000401DD2B000187EC28F00B0E0401DD5DAE
:10115000D8A49CEF88F00101010E0401DD6F0001AD
:1011600081EC77F00401FFEF8DF0FFEF8DF093EF4E
:101170007FF044EF83F00401FFEF8DF06EEF84F019
:1011800062EC7BF00401FFEF8DF00101D151F00B17
:10119000D8B48FEF89F058B0D1EF88F058A4DFEFC2
:1011A00088F0588AA09258ACDFEF88F0010E080151
:1011B000D16F00010AEC29F00101D3EF88F004019E
:1011C000A7B7FFEF88F0140E05016A6F010E6B6F71
:1011D0000001DCEC58F00101D195036A02010E51C7
:1011E000220F016E000E03220150BF0F016E010E8F
:1011F000032201C0E9FF03C0EAFFEF940401A787BF
:10120000196AF2BE198EF29E480E0C01EF6F010EA4
:10121000F06FA7C4F1FC0001F0EC25F019BEF28ECE
:10122000040EEA6EC30EE96EF2CFDDF4F29E000EFC
:101230001AEC1DF00A000900F550EE6E0009D8A462
:101240001BEF89F00401DDBFF28E040E0801A66FCA
:10125000C30EA56F000188EC2FF00101C2A347EF78
:1012600089F0BF53D8A447EF89F00401DD6BDD514D
:10127000000132EC1DF00401DD2B000187EC28F0A9
:101280000C0E0401DD5DD8A437EF89F001010401E3
:10129000DC910001AFEC64F0160E05016A6F010EDF
:1012A0006B6F0001DCEC58F00401DCB187EF89F0D2
:1012B000196AF2BE198EF29E460E0C01E66FE76BBC
:1012C000000163EC24F019BEF28E02C0DAF401C012
:1012D000D9F40401D951FF0ADD6FDA51FF0ADE6F3C
:1012E000DD53D8A479EF89F0DE510208D8B47CEF41
:1012F00089F0DC8185EF89F0160E05016A6F010E19
:101300006B6F0001DCEC58F0040155EF89F058B028
:101310008DEF89F058A48FEF89F0589AA0820401CC
:10132000FFEF8DF00101D151F00BD8B45BEF8AF0E3
:1013300058B09EEF89F058A4ACEF89F0588AA0927B
:1013400058ACACEF89F0010E0801D16F00010AEC36
:1013500029F00101A0EF89F00401A7B7CCEF89F0D3
:10136000140E05016A6F010E6B6F0001DCEC58F082
:101370000101D195036A02010E51220F016E000E88
:1013800003220150BF0F016E010E032201C0E9FFCD
:1013900003C0EAFFEF940401A787196AF2BE198E11
:1013A000F29E480E0C01EF6F010EF06FA7C4F1FC26
:1013B0000001F0EC25F019BEF28E040EEA6EC30EA9
:1013C000E96EF2CFDDF4F29E000E48EC1DF00A004B
:1013D0000900F550EE6E0009D8A4E8EF89F0040189
:1013E000DDBFF28E040E0801A66FC30EA56F0001CB
:1013F00088EC2FF00101C2A314EF8AF0BF53D8A4E8
:1014000014EF8AF00401DD6BDD51000160EC1DF08A
:101410000401DD2B000187EC28F00E0E0401DD5DD8
:10142000D8A404EF8AF001010001AFEC64F0170EBC
:1014300005016A6F010E6B6F0001DCEC58F00401CE
:10144000DC91DCB153EF8AF0196AF2BE198EF29E7C
:10145000460E0C01E66FE76B000163EC24F019BE49
:10146000F28E02C0DAF401C0D9F40401D951FF0AA6
:10147000DD6FDA51FF0ADE6FDD53D8A445EF8AF045
:10148000DE510408D8B448EF8AF0DC8151EF8AF0CD
:10149000170E05016A6F010E6B6F0001DCEC58F04E
:1014A000040121EF8AF058B059EF8AF058A45BEF9D
:1014B0008AF0589AA0820401FFEF8DF00101D1510A
:1014C000F00BD8B4FCEF8AF058B06AEF8AF058A459
:1014D00078EF8AF0588AA09258AC78EF8AF0010E23
:1014E0000801D16F00010AEC29F001016CEF8AF0CC
:1014F0000401A7A7ADEF8AF0A797040EEA6EC30E0A
:10150000E96EF2CFDDF4F29E000E000177EC1DF0E3
:101510000A000900F550EE6E0009D8A489EF8AF0A0
:101520000401DDBFF28E0101D185C2A3AAEF8AF0CA
:101530000401DD6BDD5100018FEC1DF00401DD2B9A
:10154000000187EC28F00E0E0401DD5DD8A49AEFAF
:101550008AF00101DBEF8AF00401A787040EEA6E2E
:10156000C30EE96EF2CFDDF4F29E000E0001A6EC90
:101570001DF00A000900F550EE6E0009D8A4BAEF7C
:101580008AF00401DDBFF28E0101D195C2A3DBEF29
:101590008AF00401DD6BDD510001BEEC1DF0040199
:1015A000DD2B000187EC28F0100E0401DD5DD8A4CE
:1015B000CBEF8AF00101040E0801A66FC30EA56FE0
:1015C000000188EC2FF0196AF2BE198EF29E480EC7
:1015D0000C01EF6F010EF06FA7C4F1FC0001F0ECFD
:1015E00025F019BEF28E468058B0FAEF8AF058A462
:1015F000FCEF8AF0589AA0820401FFEF8DF0010100
:10160000D151F00BD8B4C5EF8BF058B00BEF8BF085
:1016100058A419EF8BF0588AA09258AC19EF8BF0B0
:10162000010E0801D16F00010AEC29F001010DEF54
:101630008BF00401A7BD39EF8BF01C0E05016A6F1A
:10164000010E6B6F0001DCEC58F00101D197036AC9
:1016500002010E51220F016E000E03220150BF0F36
:10166000016E010E032201C0E9FF03C0EAFFEF96FD
:101670000401A78D196AF2BE198EF29E480E0C0164
:10168000EF6F010EF06FA7C4F1FC0001F0EC25F044
:1016900019BEF28E040EEA6EC30EE96EF2CFDDF4CF
:1016A000F29E000ED6EC1DF00A000900F550EE6E19
:1016B0000009D8A455EF8BF00401DDBFF28E040EB3
:1016C0000801A66FC30EA56F000188EC2FF0010181
:1016D000C2A381EF8BF0BF53D8A481EF8BF004013C
:1016E000DD6BDD510001EEEC1DF00401DD2B00018E
:1016F00087EC28F00D0E0401DD5DD8A471EF8BF0AE
:1017000001011E0E05016A6F010E6B6F0001DCEC1A
:1017100058F00401DC91DCB1B5EF8BF0420E006EA5
:10172000002EFED70000196AF2BE198EF29E460EF8
:101730000C01E66FE76B000163EC24F019BEF28E3A
:1017400002C0DAF401C0D9F40401D951FF0ADD6FF7
:10175000DA51FF0ADE6FDD2DB2EF8BF0DE53D8B425
:10176000B3EF8BF0DC818BEF8BF01F0E05016A6FFE
:10177000010E6B6F0001DCEC58F058B0C3EF8BF03A
:1017800058A4C5EF8BF0589AA0820401FFEF8DF0AA
:101790000101D151F00BD8B490EF8CF058B0D4EFD8
:1017A0008BF058A4E2EF8BF0588AA09258ACE2EF8D
:1017B0008BF0010E0801D16F00010AEC29F0010144
:1017C000D6EF8BF00401A7BD02EF8CF01C0E0501D3
:1017D0006A6F010E6B6F0001DCEC58F00101D197CC
:1017E000036A02010E51220F016E000E0322015006
:1017F000BF0F016E010E032201C0E9FF03C0EAFF23
:10180000EF960401A78D196AF2BE198EF29E480E5A
:101810000C01EF6F010EF06FA7C4F1FC0001F0ECBA
:1018200025F019BEF28E040EEA6EC30EE96EF2CFF9
:10183000DDF4F29E000E04EC1EF00A000900F550E3
:10184000EE6E0009D8A41EEF8CF00401DDBFF28E0D
:10185000040E0801A66FC30EA56F000188EC2FF0DF
:101860000101C2A34AEF8CF0BF53D8A44AEF8CF019
:101870000401DD6BDD5100011CEC1EF00401DD2BC9
:10188000000187EC28F00C0E0401DD5DD8A43AEFCE
:101890008CF001011D0E05016A6F010E6B6F0001D6
:1018A000DCEC58F00401DC91DCB180EF8CF0420EEE
:1018B000006E002EFED70000196AF2BE198EF29E4D
:1018C000460E0C01E66FE76B000163EC24F019BED5
:1018D000F28E02C0DAF401C0D9F40401D951FF0A32
:1018E000DD6FDA51FF0ADE6FDD53D8A47DEF8CF097
:1018F000DE512008D8B47EEF8CF0DC8154EF8CF000
:101900001F0E05016A6F010E6B6F0001DCEC58F0D1
:1019100058B08EEF8CF058A490EF8CF0589AA082BB
:101920000401FFEF8DF00101D151F00BD8B42CEF81
:101930008DF058B09FEF8CF058A4ADEF8CF0588A22
:10194000A09258ACADEF8CF0010E0801D16F0001F0
:101950000AEC29F00101A1EF8CF00401A7ADCDEF55
:101960008CF0A79D040EEA6EC30EE96EF2CFDDF493
:10197000F29E000E000132EC1EF00A000900F55044
:10198000EE6E0009D8A4BEEF8CF00401DDBFF28E2C
:101990000101D187F5EF8CF00401A78D196AF2BE21
:1019A000198EF29E480E0C01EF6F010EF06FA7C466
:1019B000F1FC0001F0EC25F019BEF28E040EEA6E87
:1019C000C30EE96EF2CFDDF4F29E000E4AEC1EF07B
:1019D0000A000900F550EE6E0009D8A4E9EF8CF07A
:1019E0000401DDBFF28E0101D197196AF2BE198E92
:1019F000F29E480E0C01EF6F010EF06FA7C4F1FCD0
:101A00000001F0EC25F019BEF28E040E0801A66F5D
:101A1000C30EA56F000188EC2FF046800101C2A320
:101A200024EF8DF00401DD6BDD51000162EC1EF04E
:101A30000401DD2B000187EC28F00D0E0401DD5DB3
:101A4000D8A414EF8DF0010158B02AEF8DF058A4FE
:101A50002CEF8DF0589AA0820401FFEF8DF0010168
:101A6000D151F00BD8B4FCEF8DF0D151F00BD00870
:101A7000D8B4DEEF8DF058B041EF8DF058A44FEFA1
:101A80008DF0588AA09258AC4FEF8DF0010E0801EE
:101A9000D16F00010AEC29F0010143EF8DF0040140
:101AA000A7BB88EF8DF0A78B040EEA6EC30EE96E1C
:101AB000F2CFDDF4F29E000E000178EC1EF00A0079
:101AC0000900F550EE6E0009D8A460EF8DF0040116
:101AD000DDBFF28E0101D193C2A385EF8DF0BF531C
:101AE000D8A485EF8DF00401DD6BDD51000190EC91
:101AF0001EF00401DD2B000187EC28F00A0E040122
:101B0000DD5DD8A475EF8DF00101BAEF8DF0040111
:101B1000A79B040EEA6EC30EE96EF2CFDDF4F29ECF
:101B2000000E0001A5EC1EF00A000900F550EE6E53
:101B30000009D8A495EF8DF00401DDBFF28E0101FC
:101B4000D183C2A3BAEF8DF0BF53D8A4BAEF8DF002
:101B50000401DD6BDD510001BDEC1EF00401DD2B45
:101B6000000187EC28F0090E0401DD5DD8A4AAEF7E
:101B70008DF00101040E0801A66FC30EA56F0001D0
:101B800088EC2FF0196AF2BE198EF29E480E0C01F5
:101B9000EF6F010EF06FA7C4F1FC0001F0EC25F02F
:101BA00019BEF28E468058B0D9EF8DF058A4DBEF05
:101BB0008DF0589AA082FCEF8DF00101040EEA6EC0
:101BC000C30EE96EF2CFDDF4F29E000E0001D1ECFF
:101BD0001EF00A000900F550EE6E0009D8A4EAEFE5
:101BE0008DF00401DDBFF28E040E0801A66FC30E56
:101BF000A56F000188EC2FF00401FFEF8DF00001CC
:101C0000000C0401C96BC82D2AEF8EF0C96BC651B8
:101C1000F00B006E036A0350D8A416EF8EF0800E0E
:101C2000005C0001D8B423EF8EF004010350D8A467
:101C300021EF8EF0400E005C0001D8B426EF8EF04C
:101C4000040128EF8EF00401C92B00010401C92B07
:101C500068EF8EF0020EC96FC6C400F0C751036E64
:101C6000D8A43AEF8EF0800E005C0001D8B45DEF8E
:101C70008EF004010350D8A445EF8EF0400E005CB6
:101C80000001D8B460EF8EF00401800E035CD8A48C
:101C900050EF8EF000520001D8B463EF8EF00401D3
:101CA000400E035CD8A45BEF8EF000520001D8B464
:101CB00066EF8EF0040168EF8EF00401C92B00017D
:101CC0000401C92B00010401C92B00010401C92B27
:101CD000C9C401F00001000C0401C36BC491C4939A
:101CE000196AF2BE198EF29E440E0C01E66FE76B84
:101CF000000163EC24F019BEF28E02C0C2F401C0F0
:101D0000C1F4FF0E0401C11BC21BC2C47AF4C1C4DA
:101D100079F4A7A192EF8EF076C47AF475C479F4C1
:101D20006AEF90F0C1C400F0C251036ED8A49FEFD7
:101D30008EF000520001D8B451EF8FF00401800EF4
:101D4000035CD8A4AAEF8EF000520001D8B461EF72
:101D50008FF00401400E035CD8A4B5EF8EF0005262
:101D60000001D8B461EF8FF004010350D8A4C0EF94
:101D70008EF0400E005C0001D8B461EF8FF00401DA
:101D80000350D8A4CBEF8EF0800E005C0001D8B4D5
:101D900061EF8FF004010350D8A4D6EF8EF0010E4E
:101DA000005C0001D8B4FFEF8FF004010350D8A409
:101DB000E1EF8EF0020E005C0001D8B4FFEF8FF06F
:101DC00004010350D8A4ECEF8EF0040E005C000177
:101DD000D8B4FFEF8FF004010350D8A4F7EF8EF0D2
:101DE000080E005C0001D8B4FFEF8FF0040103502F
:101DF000D8A402EF8FF0100E005C0001D8B4FFEF02
:101E00008FF004010350D8A40DEF8FF0200E005C7A
:101E10000001D8B4FFEF8FF00401010E035CD8A4D9
:101E200018EF8FF000520001D8B4FFEF8FF00401DB
:101E3000020E035CD8A423EF8FF000520001D8B447
:101E4000FFEF8FF00401040E035CD8A42EEF8FF097
:101E500000520001D8B4FFEF8FF00401080E035CBC
:101E6000D8A439EF8FF000520001D8B4FFEF8FF003
:101E70000401100E035CD8A444EF8FF0005200015F
:101E8000D8B4FFEF8FF00401200E035CD8A44FEF0D
:101E90008FF000520001D8B4FFEF8FF0040101EF82
:101EA00090F058B45DEF8FF058AE5DEF8FF05E505C
:101EB0000308D8B05DEF8FF0458A5B90589E0CEF19
:101EC00090F00401C48158BEF3EF8FF05BB0F3EFE4
:101ED0008FF058B4F3EF8FF0C2C4C7F4C1C4C6F496
:101EE000C86B00018EDE036A0150220F016E000EE6
:101EF00003220150BF0FE96E010E0320EA6EEF3896
:101F0000006E0F0E00160050D8B492EF8FF0588E6E
:101F10005E6A030E0401C36FF28AD76AD66AF1EFD4
:101F20008FF000010101C2A1F0EF8FF0C2C4C7F42D
:101F3000C1C4C6F40401C86B000163DE01C0C5F46E
:101F4000C2C4C7F4C1C4C6F40401C86B000159DEA1
:101F5000036A0150220F016E000E03220150BF0FD1
:101F6000E96E010E0320EA6EEFCFC6F40401C76BE1
:101F7000C7510001E9EC1EF00401C72B000187ECFA
:101F800028F0050E0401C75DD8A4B8EF8FF0C5C4D2
:101F9000D5F8370E0801D66F00012BEC33F0080E90
:101FA0000401C76FC7510001E9EC1EF00401C72B03
:101FB000000187EC28F0110E0401C75DD8A4D2EF10
:101FC0008FF0C6C4D5F8370E0801D66F00012BEC90
:101FD00033F00A0E87EC28F00D0E87EC28F0010193
:101FE0000401FBEF8FF05B90589E459A58A4FBEFDD
:101FF0008FF044805886C38B00010CEF90F00401F1
:10200000C4815B90589E459A58A409EF90F0448093
:10201000588600010CEF90F00401C4A116EF90F077
:10202000C3C47BF47B8F5B9A6AEF90F076C47AF43A
:1020300075C479F40101C2A16BEF90F00401C153A2
:10204000D8A427EF90F0C253D8B46AEF90F0C4B38D
:102050006AEF90F0C151FF0AC56FC251FF0AC66F07
:10206000C76BC751000104EC1FF00401C72B00012E
:1020700087EC28F0100E0401C75DD8A431EF90F072
:10208000C6C4D5F8370E0801D66F00012BEC33F02B
:10209000C5C4D5F8370E0801D66F00012BEC33F01C
:1020A000200E87EC28F0C2C4D5F8370E0801D66F91
:1020B00000012BEC33F0C1C4D5F8370E0801D66F00
:1020C00000012BEC33F00A0E87EC28F00D0E87ECA4
:1020D00028F004010101000102EFB3F005010C6BCF
:1020E0000D6B0E6B23915BAE82EF90F00001BDECA7
:1020F00036F0320E0801D16F00010AEC29F005011B
:1021000073EF90F023B1FFEF90F0630E000187ECC6
:1021100028F06E0E87EC28F00BC5ABF81F0E0801F7
:10212000AC6F00016BEC39F0320E0801D16F000189
:102130000AEC29F005010E6B0D6B00016553D8A464
:10214000C0EF90F005010D2BD8B40E2B0E510008F6
:10215000D8B0B8EF90F0FF0AD8A4B4EF90F00D51CA
:10216000F408D8B0B8EF90F0000E016E01EF91F0D6
:10217000020E0801D16F00010AEC29F09EEF90F0E9
:102180006553D8B4EEEF90F0050E0501256F0F0EE4
:10219000246F140E266F0001CAEC36F0012CECEF10
:1021A00090F005010F516308D8A4EBEF90F01051A7
:1021B0006808D8A4EBEF90F011516E08D8A4EBEFAB
:1021C00090F00B513009125DD8A4EBEF90F0010EA6
:1021D000016E01EF91F00001C0EF90F005010C2BB2
:1021E0000C510208D8B0F6EF90F02381640E08017C
:1021F000D16F00010AEC29F0050182EF90F0000E8A
:10220000016E0001000C05010C6B0D6B0E6B239130
:102210005BAE17EF91F00001BDEC36F0320E080115
:10222000D16F00010AEC29F0050108EF91F023B10C
:1022300085EF91F0630E000187EC28F0630E87ECC8
:1022400028F005010E6B0D6B00016553D8A447EF14
:1022500091F005010D2BD8B40E2B0E510008D8B00B
:102260003FEF91F0FF0AD8A43BEF91F00D51F40835
:10227000D8B03FEF91F0000E016E87EF91F0020EA3
:102280000801D16F00010AEC29F025EF91F06553A8
:10229000D8B474EF91F0050E0501256F0F0E246F71
:1022A000140E266F0001CAEC36F0012C72EF91F08B
:1022B00005010F516308D8A471EF91F0105168081F
:1022C000D8A471EF91F00B513009115DD8A471EFD2
:1022D00091F00001BDEC36F0010E016E050187EFB3
:1022E00091F0000147EF91F005010C2B0C51020811
:1022F000D8B07CEF91F02381320E0801D16F00013C
:102300000AEC29F0050117EF91F0000E016E0001B3
